 RT2501USB

 Timestamp is 45c1fc21 (Thu Feb 01 22:41:37 2007)

 Preferred load address is 10000000

 Start         Length     Name                   Class
 0001:00000000 0000bdbcH .rdata                  CODE
 0001:0000bdbc 00000065H .rdata$debug            CODE
 0001:0000be30 000419d3H .text                   CODE
 0001:0004d804 0000003cH .idata$2                CODE
 0001:0004d840 00000014H .idata$3                CODE
 0001:0004d854 00000114H .idata$4                CODE
 0001:0004d968 000003b8H .idata$6                CODE
 0001:0004dd20 0000009eH .edata                  CODE
 0002:00000000 00000114H .idata$5                DATA
 0002:00000118 00005cccH .data                   DATA
 0002:00005e00 000013fdH .bss                    DATA

  Address         Publics by Value              Rva+Base     Lib:Object

 0000:00000000       ___safe_se_handler_count   00000000     <absolute>
 0000:00000000       ___safe_se_handler_table   00000000     <absolute>
 0001:0000001c       ??_C@_0N@BOOJCAPA@HW?5Diversity?$AA@ 1000101c     mlme.obj
 0001:0000002c       ??_C@_05LKLMIBEG@Ant?9B?$AA@ 1000102c     mlme.obj
 0001:00000034       ??_C@_05JBJBNCIF@Ant?9A?$AA@ 10001034     mlme.obj
 0001:0000003c       ??_C@_0N@ENCHDJIJ@SW?5Diversity?$AA@ 1000103c     mlme.obj
 0001:0000004c       ??_C@_0DC@DNIOBKKO@4?9way?5handshake?5IE?5diff?5among?5As@ 1000104c     mlme.obj
 0001:00000080       ??_C@_0CE@ODBDOOLB@2?9way?5?$CIgroup?5key?$CJ?5handshake?5time@ 10001080     mlme.obj
 0001:000000a4       ??_C@_0BI@IFDLABDB@4?9way?5handshake?5timeout?$AA@ 100010a4     mlme.obj
 0001:000000bc       ??_C@_09CJDAIAGP@MIC?5error?$AA@ 100010bc     mlme.obj
 0001:000000c8       ??_C@_0L@LCBPMDKI@invalid?5IE?$AA@ 100010c8     mlme.obj
 0001:000000d4       ??_C@_0CD@EMJAOFKL@require?5auth?5before?5assoc?1re?9ass@ 100010d4     mlme.obj
 0001:000000f8       ??_C@_0O@IBGJFIPI@class?53?5error?$AA@ 100010f8     mlme.obj
 0001:00000108       ??_C@_0O@ENMDFIGG@class?52?5error?$AA@ 10001108     mlme.obj
 0001:00000118       ??_C@_0CE@IOCPNGNK@AP?5unable?5to?5hanle?5all?5associati@ 10001118     mlme.obj
 0001:0000013c       ??_C@_0BM@OBHJDPBG@DIS?9ASSOC?5due?5to?5inactivity?$AA@ 1000113c     mlme.obj
 0001:00000158       ??_C@_0BK@BAGFOGKD@STA?5is?5leaving?5?1?5has?5left?$AA@ 10001158     mlme.obj
 0001:00000174       ??_C@_0BO@PEBKGJDA@Previous?5Auth?5no?5longer?5valid?$AA@ 10001174     mlme.obj
 0001:00000194       ??_C@_0BD@PBGFPAEA@Unspecified?5Reason?$AA@ 10001194     mlme.obj
 0001:000001a8       ??_C@_08NKCLJDKG@Reserved?$AA@ 100011a8     mlme.obj
 0001:000001b4       ??_C@_0BF@KFHIDKKF@?$DM?9?9?5MLME?5Initialize?6?$AA@ 100011b4     mlme.obj
 0001:000001cc       ??_C@_0BF@MBFCBGHE@?9?9?$DO?5MLME?5Initialize?6?$AA@ 100011cc     mlme.obj
 0001:000001e4       ??_C@_0BO@NALBCFMJ@MlmeHandler?3?5MlmeQueue?5empty?6?$AA@ 100011e4     mlme.obj
 0001:00000204       ??_C@_0BB@LJGKENIN@RT2501USB?5ERROR?3?$AA@ 10001204     mlme.obj
 0001:00000218       ??_C@_0CJ@GLPMGFH@ERROR?3?5Illegal?5machine?5in?5MlmeHa@ 10001218     mlme.obj
 0001:00000244       ??_C@_0CC@CLKIEPMO@?$CB?$CB?$CB?5reset?5MLME?5state?5machine?5?$CB?$CB?$CB@ 10001244     mlme.obj
 0001:00000268       ??_C@_0EK@EGLGGJEG@Device?5Halted?5or?5Removed?5or?5Mlme@ 10001268     mlme.obj
 0001:000002b4       ??_C@_0O@DPOFPIAE@?$DM?$DN?$DN?5MlmeHalt?6?$AA@ 100012b4     mlme.obj
 0001:000002c4       ??_C@_0O@NFHEMLIC@?$DN?$DN?$DO?5MlmeHalt?6?$AA@ 100012c4     mlme.obj
 0001:000002d4       ??_C@_0BA@FEFLNHKP@?$DM?$DN?$DNMlmeSuspend?6?$AA@ 100012d4     mlme.obj
 0001:000002e4       ??_C@_0CA@KBPCGKML@ERROR?3?5empty?5Elem?5in?5MlmeQueue?6?$AA@ 100012e4     mlme.obj
 0001:00000304       ??_C@_0BA@IGFCGDOF@?$DN?$DN?$DOMlmeSuspend?6?$AA@ 10001304     mlme.obj
 0001:00000314       ??_C@_0P@DEFOPNOP@?$DM?$DN?$DNMlmeResume?6?$AA@ 10001314     mlme.obj
 0001:00000324       ??_C@_0P@DAGPEKMJ@?$DN?$DN?$DOMlmeResume?6?$AA@ 10001324     mlme.obj
 0001:00000334       ??_C@_0CD@HEDBGBO@OneSecAggCnt?$DN?$CFd?0OneSecNoAggCnt?$DN?$CF@ 10001334     mlme.obj
 0001:00000358       ??_C@_0CH@BCKEIIKJ@NDIS_STATUS_MEDIA_DISCONNECT?5Eve@ 10001358     mlme.obj
 0001:00000380       ??_C@_0CE@ELOODNLJ@pAd?9?$DOStaCfg?4bAutoReconnect?5is?5TR@ 10001380     mlme.obj
 0001:000003a4       ??_C@_0DK@KINFKHLB@CNTL?5?9?5No?5matching?5BSS?0?5start?5a?5@ 100013a4     mlme.obj
 0001:000003e0       ??_C@_0CL@CGKOOPBI@MLME?5periodic?5exec?0?5no?5associati@ 100013e0     mlme.obj
 0001:00000410       ??_C@_0EP@LAOHBGHC@MMCHK?5?9?5excessive?5BEACON?5lost?0?5l@ 10001410     mlme.obj
 0001:00000460       ??_C@_0CL@KJDFOMDE@Not?5found?5radar?5signal?0?5start?5se@ 10001460     mlme.obj
 0001:0000048c       ??_C@_0BI@CKMGBLNE@Found?5radar?5signal?$CB?$CB?$CB?6?6?$AA@ 1000148c     mlme.obj
 0001:000004a4       ??_C@_0CN@GDCEANDO@MMCHK?5?9?5last?511B?5peer?5left?0?5upda@ 100014a4     mlme.obj
 0001:000004d4       ??_C@_0N@DLDNHFDI@RxSignal?5?$CFd?6?$AA@ 100014d4     mlme.obj
 0001:000004e4       ??_C@_0CM@GJLCIBAC@MMCHK?5?9?5Bad?5CQI?4?5Auto?5Recovery?5a@ 100014e4     mlme.obj
 0001:00000510       ??_C@_0DI@IJMMIEOH@MMCHK?5?9?5No?5BEACON?4?5Dead?5CQI?4?5Aut@ 10001510     mlme.obj
 0001:00000548       ??_C@_0DJ@CPNJNHAA@STAMlmePeriodicExec?5?9?5LastRssi?$DN?$CF@ 10001548     mlme.obj
 0001:00000584       ??_C@_0CB@HGLEIPIO@Ant?9realrssi0?$CI?$CFd?$CJ?0Lastrssi0?$CI?$CFd?$CJ?6@ 10001584     mlme.obj
 0001:000005a8       ??_C@_0DB@NLDAOOAH@MlmePeriodicExec?3?5no?5traffic?1bea@ 100015a8     mlme.obj
 0001:000005e0       ??_C@_0EF@HBMLNPIK@MMCHK?5?9?5CommonCfg?4Ssid?$FL?$CFd?$FN?$DN?$CFc?$CFc?$CF@ 100015e0     mlme.obj
 0001:00000628       ??_C@_0BK@GAJBDICC@MMCHK?5?9?5Driver?5auto?5scan?6?$AA@ 10001628     mlme.obj
 0001:00000648       ??_C@_0EG@NHNNNGNH@Driver?5auto?5reconnect?5to?5last?5OI@ 10001648     mlme.obj
 0001:00000690       ??_C@_0CN@GLNBGBEB@?$DM?$DN?$DN?5MlmeCheckForRoaming?$CI?$CD?5of?5can@ 10001690     mlme.obj
 0001:000006c0       ??_C@_0BN@DKOAEPAH@MMCHK?5?9?5Roaming?5attempt?5?$CD?$CFd?6?$AA@ 100016c0     mlme.obj
 0001:000006e0       ??_C@_0BJ@FIFPAOCP@?$DN?$DN?$DO?5MlmeCheckForRoaming?6?$AA@ 100016e0     mlme.obj
 0001:000006fc       ??_C@_0BN@CECCMCMI@?$DM?$DN?$DN?5MlmeCheckForFastRoaming?6?$AA@ 100016fc     mlme.obj
 0001:0000071c       ??_C@_0DD@LEDDAC@MMCHK?5?9?5Roaming?0?5No?5eligable?5ent@ 1000171c     mlme.obj
 0001:00000750       ??_C@_0CA@EIJLLNEB@LastRssi?5?$DN?5?$CFd?0?5pBss?9?$DORssi?5?$DN?5?$CFd?6?$AA@ 10001750     mlme.obj
 0001:00000770       ??_C@_0BN@PELBDGCP@?$DN?$DN?$DO?5MlmeCheckForFastRoaming?6?$AA@ 10001770     mlme.obj
 0001:00000790       ??_C@_0FC@FNIFIADK@MMCHK?5?9?5CQI?$DN?5?$CFd?5?$CITx?5Fail?$DN?$CFd?1Retr@ 10001790     mlme.obj
 0001:000007e4       ??_C@_0DA@CIDAAHMM@BEACON?5lost?5?$DO?5?$CFd?5msec?5with?5TxOkC@ 100017e4     mlme.obj
 0001:00000814       ??_C@_0CD@GBLMFGBJ@DRS?3?5?9?9TX?5rate?5from?5?$CFd?5to?5?$CFd?5Mbp@ 10001814     mlme.obj
 0001:00000838       ??_C@_0CD@HJJPMMLA@DRS?3?5?$CL?$CLTX?5rate?5from?5?$CFd?5to?5?$CFd?5Mbp@ 10001838     mlme.obj
 0001:0000085c       ??_C@_0CI@PEODENBM@DRS?3?52?5NULL?5frames?5at?5UpRate?5?$DN?5?$CF@ 1000185c     mlme.obj
 0001:00000888       ??_C@_0EA@CDOGDGBM@DRS?3?5?$CD?$CD?$CD?$CD?5leave?5Noisy?5environmen@ 10001888     mlme.obj
 0001:000008c8       ??_C@_0CI@CPKEAOJA@DRS?3?5?$CD?$CD?$CD?$CD?5enter?5Noisy?5environmen@ 100018c8     mlme.obj
 0001:000008f0       ??_C@_0GK@MJPAJKLK@?$CFd?3?5NDIS?5push?5BE?$DN?$CFd?0?5BK?$DN?$CFd?0?5VI?$DN?$CF@ 100018f0     mlme.obj
 0001:0000095c       ??_C@_0BE@BPMIFJNI@MlmeSetPsmBit?5?$DN?5?$CFd?6?$AA@ 1000195c     mlme.obj
 0001:00000970       ??_C@_0CG@EENPFOPN@MlmeSetTxPreamble?5?$CI?$DN?5SHORT?5PREAM@ 10001970     mlme.obj
 0001:00000998       ??_C@_0CF@GGJHLABL@MlmeSetTxPreamble?5?$CI?$DN?5LONG?5PREAMB@ 10001998     mlme.obj
 0001:000009c0       ??_C@_0EE@BANLCMAO@?5MlmeUpdateTxRates?5?$CITxRate?$DN?$CFd?0?5R@ 100019c0     mlme.obj
 0001:00000a08       ??_C@_0FE@EPLKFKCI@?5MlmeUpdateTxRates?5?$CIMaxDesire?$DN?$CFd@ 10001a08     mlme.obj
 0001:00000a5c       ??_C@_0DG@DBIFONLM@?5MlmeUpdateTxRates?5?$CIRssi?$DN?$CFd?0?5ini@ 10001a5c     mlme.obj
 0001:00000a94       ??_C@_0CC@NNNGGMIO@Exptected?5ACK?5rate?$FL?$CFd?$FN?5?$DN?5?$CFd?5Mbps@ 10001a94     mlme.obj
 0001:00000ab8       ??_C@_0BC@GONIMOIH@?$DM?$DN?$DN?5MlmeRadioOff?6?$AA@ 10001ab8     mlme.obj
 0001:00000acc       ??_C@_0BI@PDLIKBPL@BulkOut?5IRP?5Pending?$CB?$CB?$CB?6?$AA@ 10001acc     mlme.obj
 0001:00000ae4       ??_C@_0BH@HLFDJKDK@BulkIn?5IRP?5Pending?$CB?$CB?$CB?6?$AA@ 10001ae4     mlme.obj
 0001:00000afc       ??_C@_0BC@KIECMMJE@?$DN?$DN?$DO?5MlmeRadioOff?6?$AA@ 10001afc     mlme.obj
 0001:00000b10       ??_C@_0BB@CJNFNKA@?$DN?$DN?$DO?5MlmeRadioOn?6?$AA@ 10001b10     mlme.obj
 0001:00000b24       ??_C@_0DE@KFDCONOO@CommonCfg?4WepStatus?$DN?$CFd?0?5while?5pI@ 10001b24     mlme.obj
 0001:00000b58       ??_C@_0CD@KCHNKJHD@?$EA?$EA?$EA?5MlmeQueueInit?5Queue?9?$DOLock?5?$DN?$CF@ 10001b58     mlme.obj
 0001:00000b7c       ??_C@_0BF@MNDOIEEO@MlmeEnqueue?0?5num?$DN?$CFd?6?$AA@ 10001b7c     mlme.obj
 0001:00000b94       ??_C@_0DF@NAOONHPL@MlmeEnqueue?3?5full?0?5msg?5dropped?5a@ 10001b94     mlme.obj
 0001:00000bcc       ??_C@_0CI@ODKFEBBA@MlmeEnqueue?3?5msg?5too?5large?0?5size@ 10001bcc     mlme.obj
 0001:00000bf4       ??_C@_0BM@DNAMCAN@MlmeEnqueueForRecv?0?5num?$DN?$CFd?6?$AA@ 10001bf4     mlme.obj
 0001:00000c10       ??_C@_0DF@OGAGJABB@MlmeEnqueueForRecv?3?5un?9recongniz@ 10001c10     mlme.obj
 0001:00000c48       ??_C@_0CG@HKDBINCL@MlmeEnqueueForRecv?3?5full?5and?5dro@ 10001c48     mlme.obj
 0001:00000c70       ??_C@_0DB@BMOIKAPK@MlmeEnqueueForRecv?3?5frame?5too?5la@ 10001c70     mlme.obj
 0001:00000ca4       ??_C@_0BF@BAEDGELA@MlmeDequeue?0?5num?$DN?$CFd?6?$AA@ 10001ca4     mlme.obj
 0001:00000cbc       ??_C@_0BN@POPBCJAH@?$DM?$DN?$DN?5MlmeRestartStateMachine?6?$AA@ 10001cbc     mlme.obj
 0001:00000cdc       ??_C@_0BN@COGCNNOA@?$DN?$DN?$DO?5MlmeRestartStateMachine?6?$AA@ 10001cdc     mlme.obj
 0001:00000d00       ??_C@_0FJ@LGNHBPLH@AsicSwitchChannel?$CIRF?$DN?$CFd?$CJ?5to?5?$CD?$CFd?0@ 10001d00     mlme.obj
 0001:00000d5c       ??_C@_0CJ@GJAOJJKN@AsicAntennaSelect?$CIch?$DN?$CFd?$CJ?5?9?5Tx?$DN?$CFs@ 10001d5c     mlme.obj
 0001:00000d88       ??_C@_0BC@NJKCDFCM@Unkown?5RFIC?5Type?6?$AA@ 10001d88     mlme.obj
 0001:00000d9c       ??_C@_0CG@BJLCMOIA@AsicAdjustTxPower?5?$DN?5?$CFd?0?5AvgRssi?5@ 10001d9c     mlme.obj
 0001:00000dc4       ??_C@_0DM@DHCNECDC@?$CL?$CL?5Tx?5Power?0?5BBP?5R1?$DN?$CFx?0?5Tssi0?$DN?$CFx@ 10001dc4     mlme.obj
 0001:00000e00       ??_C@_0DO@EMNLCJBF@?9?9?5Tx?5Power?0?5BBP?5R1?$DN?$CFx?0?5TssiRef?$DN@ 10001e00     mlme.obj
 0001:00000e40       ??_C@_0EG@PFKDEGON@AsicAdjustTxPower?$CIcan?5find?5pAd?9?$DO@ 10001e40     mlme.obj
 0001:00000e88       ??_C@_0CM@DGJPKHEP@?$DO?$DO?$DOAsicSleepThenAutoWakeup?$CIsleep@ 10001e88     mlme.obj
 0001:00000eb4       ??_C@_0BG@NHDNBOHG@?$DO?$DO?$DOAsicForceSleep?$DM?$DM?$DM?6?$AA@ 10001eb4     mlme.obj
 0001:00000ecc       ??_C@_0BH@MEPPFOKP@?$DO?$DO?$DOAsicForceWakeup?$DM?$DM?$DM?6?$AA@ 10001ecc     mlme.obj
 0001:00000ee4       ??_C@_0BE@IPCIFFIC@?$DO?$DO?$DOAsicSetBssid?$DM?$DM?$DM?6?$AA@ 10001ee4     mlme.obj
 0001:00000ef8       ??_C@_0CB@KJJMMDE@?9?9?9?$DODisable?5TSF?5synchronization?6@ 10001ef8     mlme.obj
 0001:00000f1c       ??_C@_0CD@NNMMNNEG@?9?9?9?$DOAsicEnableBssSync?$CIINFRA?5mode@ 10001f1c     mlme.obj
 0001:00000f40       ??_C@_0BB@KHBJECDL@CSR9?5?$DN?50x?$CF08lx?5?6?$AA@ 10001f40     mlme.obj
 0001:00000f54       ??_C@_0CE@GMHJPLF@?9?9?9?$DOAsicEnableIbssSync?$CIADHOC?5mod@ 10001f54     mlme.obj
 0001:00000f78       ??_C@_0CP@CKBLJIJO@?5?5?5?5AC_VO?5?5?5?5?5?$CFd?5?5?5?5?5?$CFd?5?5?5?5?5?$CFd?5?5@ 10001f78     mlme.obj
 0001:00000fa8       ??_C@_0CP@FGFMKHCJ@?5?5?5?5AC_VI?5?5?5?5?5?$CFd?5?5?5?5?5?$CFd?5?5?5?5?5?$CFd?5?5@ 10001fa8     mlme.obj
 0001:00000fd8       ??_C@_0CP@OPCIPAFK@?5?5?5?5AC_BK?5?5?5?5?5?$CFd?5?5?5?5?5?$CFd?5?5?5?5?5?$CFd?5?5@ 10001fd8     mlme.obj
 0001:00001008       ??_C@_0CP@IKLEJIGG@?5?5?5?5AC_BE?5?5?5?5?5?$CFd?5?5?5?5?5?$CFd?5?5?5?5?5?$CFd?5?5@ 10002008     mlme.obj
 0001:00001038       ??_C@_0CO@EONIKGDE@EDCA?5?$FL?$CD?$CFd?$FN?3?5AIFSN?5CWmin?5CWmax?5?5T@ 10002038     mlme.obj
 0001:00001068       ??_C@_0BB@ENFHEMBH@AsicSetEdcaParm?6?$AA@ 10002068     mlme.obj
 0001:0000107c       ??_C@_0BJ@NALBBIL@AsicSetSlotTime?$CI?$DN?$CFd?5us?$CJ?6?$AA@ 1000207c     mlme.obj
 0001:00001098       ??_C@_0CJ@LHJPNECD@RSSI?$DN?$CFd?0?5CCA?$DN?$CFd?0?5R17?$DNR17UpperBou@ 10002098     mlme.obj
 0001:000010c4       ??_C@_0CI@HDEHACKO@mid?5RSSI?$DN?$CFd?0?5CCA?$DN?$CFd?0?5fixed?5R17?5a@ 100020c4     mlme.obj
 0001:000010ec       ??_C@_0CN@HLKNMFLL@3?5strong?5RSSI?$DN?$CFd?0?5CCA?$DN?$CFd?0?5fixed?5@ 100020ec     mlme.obj
 0001:0000111c       ??_C@_0CN@NIDLONPH@2?5strong?5RSSI?$DN?$CFd?0?5CCA?$DN?$CFd?0?5fixed?5@ 1000211c     mlme.obj
 0001:0000114c       ??_C@_0CD@OPPHFDIA@Avg?5RSSI?$DN?$CFd?0?5BbpRssiToDbmDelta?$DN?$CF@ 1000214c     mlme.obj
 0001:00001170       ??_C@_0CD@DDHMKIMO@RSSI?$DN?$CFd?0?5CCA?$DN?$CFd?0?5keep?5R17?5at?50x?$CF@ 10002170     mlme.obj
 0001:00001194       ??_C@_0BO@CEIJHPJM@RSSI?$DN?$CFd?0?5CCA?$DN?$CFd?0?5?9?9R17?$DN?50x?$CFx?6?$AA@ 10002194     mlme.obj
 0001:000011b4       ??_C@_0BO@GLFBAFKB@RSSI?$DN?$CFd?0?5CCA?$DN?$CFd?0?5?$CL?$CLR17?$DN?50x?$CFx?6?$AA@ 100021b4     mlme.obj
 0001:000011d4       ??_C@_0CN@OHPAJDGC@1?5strong?5RSSI?$DN?$CFd?0?5CCA?$DN?$CFd?0?5fixed?5@ 100021d4     mlme.obj
 0001:00001204       ??_C@_0DL@HEKIHOHH@?5?5?5?5?5Tx?5MIC?5Key?5?$DN?5?$CF02x?3?$CF02x?3?$CF02x@ 10002204     mlme.obj
 0001:00001240       ??_C@_0DL@HBHFILMD@?5?5?5?5?5Rx?5MIC?5Key?5?$DN?5?$CF02x?3?$CF02x?3?$CF02x@ 10002240     mlme.obj
 0001:00001280       ??_C@_0FM@LBEPCOLK@?5?5?5?5?5Key?5?$DN?5?$CF02x?3?$CF02x?3?$CF02x?3?$CF02x?3?$CF@ 10002280     mlme.obj
 0001:000012dc       ??_C@_0CD@PMFJLLCD@AsicAddSharedKeyEntry?3?5?$CFs?5key?5?$CD?$CF@ 100022dc     mlme.obj
 0001:00001300       ??_C@_1FK@FNONLNGN@?$AA?$CF?$AAs?$AA?3?$AA?5?$AAD?$AAE?$AAB?$AAU?$AAG?$AAC?$AAH?$AAK?$AA?5?$AAf?$AAa?$AAi?$AAl?$AAe?$AAd?$AA?5@ 10002300     mlme.obj
 0001:0000135c       ??_C@_1BA@LEPJIIOK@?$AAU?$AAn?$AAk?$AAn?$AAo?$AAw?$AAn?$AA?$AA@ 1000235c     mlme.obj
 0001:00001370       ??_C@_1HE@GFNMHAOC@?$AAC?$AA?3?$AA?2?$AAW?$AAI?$AAN?$AAC?$AAE?$AA5?$AA0?$AA0?$AA?2?$AAP?$AAB?$AAW?$AAo?$AAr?$AAk?$AAs?$AAp@ 10002370     mlme.obj
 0001:000013e4       ??_C@_0CA@GIKNBHP@AsicRemoveSharedKeyEntry?3?5?$CD?$CFd?5?6?$AA@ 100023e4     mlme.obj
 0001:00001404       ??_C@_0CE@HEALNGMG@?5?5pRxMic?5?$DN?5?$CF02x?3?$CF02x?3?$CF02x?3?$CF02x?3?4@ 10002404     mlme.obj
 0001:00001428       ??_C@_0CE@CKHLPKBD@?5?5TxMIC?5?5?$DN?5?$CF02x?3?$CF02x?3?$CF02x?3?$CF02x?3?4@ 10002428     mlme.obj
 0001:0000144c       ??_C@_0CE@MNKCACCJ@?5?5Key?5?5?5?5?$DN?5?$CF02x?3?$CF02x?3?$CF02x?3?$CF02x?3?4@ 1000244c     mlme.obj
 0001:00001470       ??_C@_0EM@JDBCJKOK@AsicAddPairwiseKeyEntry?3?5Entry?$CD?$CF@ 10002470     mlme.obj
 0001:000014bc       ??_C@_0CC@BOKOJPNL@AsicRemovePairwiseKeyEntry?3?5?$CD?$CFd?5@ 100024bc     mlme.obj
 0001:000014e0       ??_C@_0CC@NGCIDNIA@AsicSetRxAnt?0?5pair1?$DN?$CFd?0?5pair2?$DN?$CFd@ 100024e0     mlme.obj
 0001:00001504       ??_C@_0DP@BGOGKPAL@AntDiv?5?9?5before?5evaluate?5Pair1?9A@ 10002504     mlme.obj
 0001:00001544       ??_C@_0CA@KIEDFAGD@After?5Eval?9Pair1?5?$CD?$CFd?0Pair2?5?$CD?$CFd?6?$AA@ 10002544     mlme.obj
 0001:00001568       ??_C@_0EB@MGIGNCPH@After?5Eval?0RSSI?$FL0?01?02?03?$FN?$DN?$DM?$CFd?0?$CFd?0@ 10002568     mlme.obj
 0001:000015b0       ??_C@_0EP@GHPDNONO@StaQuickResponeForRateUpExec?3?5Be@ 100025b0     mlme.obj
 0001:00001600       ??_C@_0BJ@DIAPDBOF@RadarDetectionStart?9?9?9?$DO?6?$AA@ 10002600     mlme.obj
 0001:0000161c       ??_C@_0CP@BDGHPBED@?$DM?$DN?$DN?5MlmeFreeMemory?5?$FLIN?3?$CFd?$FN?$FLUN?3?$CFd@ 1000261c     mlme.obj
 0001:00001650       ??_C@_0FH@CDHFCHFF@MlmeFreeMemory?5Add?5it?5to?5the?5Unu@ 10002650     mlme.obj
 0001:000016a8       ??_C@_0HH@HGEKCKCA@?$DMWarning?$DOFree?5memory?5faild?$CB?$CB?5mem@ 100026a8     mlme.obj
 0001:00001720       ??_C@_0BE@IBOPMBON@?$DM?$DN?$DN?5MlmeFreeMemory?6?$AA@ 10002720     mlme.obj
 0001:00001738       ??_C@_0FI@ELLHFEGA@Mlme?5memory?5Handler?5Busy?$CB?$CB?5move?5@ 10002738     mlme.obj
 0001:00001790       ??_C@_0BE@OAOCHMJ@?$DN?$DN?$DO?5MlmeFreeMemory?6?$AA@ 10002790     mlme.obj
 0001:000017a4       ??_C@_0DC@IMDMGHCM@?$DM?$DN?$DN?5MlmeAllocateMemory?$FLIN?3?$CFd?$FN?$FLUN@ 100027a4     mlme.obj
 0001:000017d8       ??_C@_0DG@MJNLKOFL@MlmeAllocateMemory?5?$FLpMlmeMemoryS@ 100027d8     mlme.obj
 0001:00001810       ??_C@_0EG@KMAOJKEN@MlmeAllocateMemory?0?5failed?$CB?$CB?5?$CITh@ 10002810     mlme.obj
 0001:00001858       ??_C@_0BI@KKHFDPKB@?$DM?$DN?$DN?5MlmeAllocateMemory?6?$AA@ 10002858     mlme.obj
 0001:00001870       ??_C@_0DJ@DGPBIMOD@Mlme?5memory?5Handler?5Busy?$CB?$CB?0?5Mlme@ 10002870     mlme.obj
 0001:000018ac       ??_C@_0BI@BCCIPHMG@?$DN?$DN?$DO?5MlmeAllocateMemory?6?$AA@ 100028ac     mlme.obj
 0001:000018c4       ??_C@_0BE@PGBALOCM@?$DM?$DN?$DN?5MlmeInitMemory?6?$AA@ 100028c4     mlme.obj
 0001:000018d8       ??_C@_0DK@EAMLLFJN@MlmeInitMemory?5Initial?5failed?5?$FLR@ 100028d8     mlme.obj
 0001:00001914       ??_C@_0BE@HJPBFIAI@?$DN?$DN?$DO?5MlmeInitMemory?6?$AA@ 10002914     mlme.obj
 0001:00001928       ??_C@_0BJ@HJMABJMD@?$DM?9?9?9?9?9?5AironetMsgAction?6?$AA@ 10002928     aironet.obj
 0001:00001944       ??_C@_0N@DHDEPIEC@FR?5len?5?$DN?5?$CFd?6?$AA@ 10002944     aironet.obj
 0001:00001954       ??_C@_0DK@DKJHBNAA@Wrong?5IAPP?5SA?5for?5Cisco?5Aironet?5@ 10002954     aironet.obj
 0001:00001990       ??_C@_0DK@NOKMICGP@Wrong?5IAPP?5DA?5for?5Cisco?5Aironet?5@ 10002990     aironet.obj
 0001:000019cc       ??_C@_0DA@HINIAAEB@Wrong?5IAPP?5subtype?5for?5Cisco?5Air@ 100029cc     aironet.obj
 0001:000019fc       ??_C@_0CN@EHELCGHJ@Wrong?5IAPP?5type?5for?5Cisco?5Airone@ 100029fc     aironet.obj
 0001:00001a2c       ??_C@_0BM@OIPEIPBN@IAPP?5Measurement?5Offset?5?$CFx?6?$AA@ 10002a2c     aironet.obj
 0001:00001a48       ??_C@_0BK@ONGANIEC@IAPP?5Activation?5Delay?5?$CFx?6?$AA@ 10002a48     aironet.obj
 0001:00001a64       ??_C@_0BG@EJECLJKI@IAPP?5Dialog?5Token?5?$CFx?6?$AA@ 10002a64     aironet.obj
 0001:00001a7c       ??_C@_0BB@FPEIDLDD@IAPP?5SubType?5?$CFx?6?$AA@ 10002a7c     aironet.obj
 0001:00001a90       ??_C@_0O@HEPIDHDG@IAPP?5Type?5?$CFx?6?$AA@ 10002a90     aironet.obj
 0001:00001aa0       ??_C@_0BF@ILKJELFG@IAPP?5ID?5?$CG?5Length?5?$CFd?6?$AA@ 10002aa0     aironet.obj
 0001:00001ab8       ??_C@_0BJ@MLDDEIEM@?9?9?9?9?9?$DO?5AironetMsgAction?6?$AA@ 10002ab8     aironet.obj
 0001:00001ad4       ??_C@_0CB@ELJJOMEK@ChannelLoadRequestAction?5?$DM?9?9?9?9?9?6@ 10002ad4     aironet.obj
 0001:00001af8       ??_C@_0CI@NGCIHEFA@Send?5PSM?5Data?5frame?5for?5off?5chan@ 10002af8     aironet.obj
 0001:00001b20       ??_C@_0BK@LAICFHGC@Duration?5?$CFd?0?5Channel?5?$CFd?$CB?6?$AA@ 10002b20     aironet.obj
 0001:00001b3c       ??_C@_0CB@OFOIMANG@ChannelLoadRequestAction?5?9?9?9?9?9?$DO?6@ 10002b3c     aironet.obj
 0001:00001b60       ??_C@_0BP@LMHEGMDC@NoiseHistRequestAction?5?$DM?9?9?9?9?9?6?$AA@ 10002b60     aironet.obj
 0001:00001b80       ??_C@_0BP@BCAFEAKO@NoiseHistRequestAction?5?9?9?9?9?9?$DO?6?$AA@ 10002b80     aironet.obj
 0001:00001ba0       ??_C@_0BM@JHFJHGOL@BeaconRequestAction?5?$DM?9?9?9?9?9?6?$AA@ 10002ba0     aironet.obj
 0001:00001bbc       ??_C@_0BC@LBJBAFBB@Wrong?5Scan?5Mode?$CB?6?$AA@ 10002bbc     aironet.obj
 0001:00001bd0       ??_C@_0BF@NEBMODEP@Beacon?5Report?5Mode?$CB?6?$AA@ 10002bd0     aironet.obj
 0001:00001be8       ??_C@_0BD@HAAFBFOE@Active?5Scan?5Mode?$CB?6?$AA@ 10002be8     aironet.obj
 0001:00001bfc       ??_C@_0O@CMCIPBCP@Duration?5?$CFd?$CB?6?$AA@ 10002bfc     aironet.obj
 0001:00001c0c       ??_C@_0BE@FIFDBKHC@Passive?5Scan?5Mode?$CB?6?$AA@ 10002c0c     aironet.obj
 0001:00001c20       ??_C@_0BM@DJCIFKHH@BeaconRequestAction?5?9?9?9?9?9?$DO?6?$AA@ 10002c20     aironet.obj
 0001:00001c3c       ??_C@_0BM@EKJAGNG@AironetReportAction?5?$DM?9?9?9?9?9?6?$AA@ 10002c3c     aironet.obj
 0001:00001c58       ??_C@_0BM@KKNICKEK@AironetReportAction?5?9?9?9?9?9?$DO?6?$AA@ 10002c58     aironet.obj
 0001:00001c74       ??_C@_0CB@IDHHHOCN@AironetFinalReportAction?5?$DM?9?9?9?9?9?6@ 10002c74     aironet.obj
 0001:00001c98       ??_C@_0CB@CNAGFCLB@AironetFinalReportAction?5?9?9?9?9?9?$DO?6@ 10002c98     aironet.obj
 0001:00001cbc       ??_C@_0CA@PFKFHHJL@ChannelLoadReportAction?5?$DM?9?9?9?9?9?6?$AA@ 10002cbc     aironet.obj
 0001:00001cdc       ??_C@_0BD@JHBMOFCE@FrameReportLen?5?$CFd?6?$AA@ 10002cdc     aironet.obj
 0001:00001cf0       ??_C@_0CI@KLDDAJOL@CLBusyByte?5?$CFd?0?5Duration?5?$CFd?0?5Resu@ 10002cf0     aironet.obj
 0001:00001d18       ??_C@_0CA@FLNEFLAH@ChannelLoadReportAction?5?9?9?9?9?9?$DO?6?$AA@ 10002d18     aironet.obj
 0001:00001d38       ??_C@_0BO@HKHCFCAP@NoiseHistReportAction?5?$DM?9?9?9?9?9?6?$AA@ 10002d38     aironet.obj
 0001:00001d58       ??_C@_0BL@JFGNOGFD@Reported?5RPI?$FL0?$FN?5?5?$DN?50x?$CF02x?6?$AA@ 10002d58     aironet.obj
 0001:00001d74       ??_C@_0BM@KOCKFHAN@Reported?5RPI?$FL?$CFd?$FN?5?5?$DN?50x?$CF02x?6?$AA@ 10002d74     aironet.obj
 0001:00001d90       ??_C@_0BF@GCIGDMNE@Total?5RPI?5Conuts?5?$CFd?6?$AA@ 10002d90     aironet.obj
 0001:00001da8       ??_C@_0BC@MOKPKFAH@RPI?5?$CFd?5Conuts?5?$CFd?6?$AA@ 10002da8     aironet.obj
 0001:00001dbc       ??_C@_0BO@NEADHOJD@NoiseHistReportAction?5?9?9?9?9?9?$DO?6?$AA@ 10002dbc     aironet.obj
 0001:00001ddc       ??_C@_0BL@ODDCBJLF@BeaconReportAction?5?$DM?9?9?9?9?9?6?$AA@ 10002ddc     aironet.obj
 0001:00001df8       ??_C@_0BL@ENEDDFCJ@BeaconReportAction?5?9?9?9?9?9?$DO?6?$AA@ 10002df8     aironet.obj
 0001:00001e14       ??_C@_0BG@MEBFBIPF@RxPower?$FL?$CFd?$FN?0?5Rssi?5?$CFd?6?$AA@ 10002e14     aironet.obj
 0001:00001e2c       ??_C@_0BF@COBOCKCM@FrameReportLen?5?$DN?5?$CFd?6?$AA@ 10002e2c     aironet.obj
 0001:00001e44       ??_C@_0CC@JBLEHIHB@RxPower?$FL?$CFd?$FN?5Rssi?5?$CFd?0?5Avg?5Rssi?5?$CFd@ 10002e44     aironet.obj
 0001:00001e68       ??_C@_0CF@NFOOFABO@Bssid?5?$CF02x?3?$CF02x?3?$CF02x?3?$CF02x?3?$CF02x?3?$CF@ 10002e68     aironet.obj
 0001:00001e90       ??_C@_0CM@OKGHKGKF@Sniff2BytesFromNdisBuffer?$CIoffset@ 10002e90     rtusb_data.obj
 0001:00001ebc       ??_C@_0BI@HGBFLCFD@?$DO?$DO?$DO?5One?5Packet?5Pending?6?$AA@ 10002ebc     rtusb_data.obj
 0001:00001ed4       ??_C@_0BN@BDIMLFLK@Ad?9Hoc?5?9?$DO?5Enqueue?5one?5frame?6?$AA@ 10002ed4     rtusb_data.obj
 0001:00001ef4       ??_C@_0CF@OKLLCBGL@Infrastructure?5?9?$DO?5Enqueue?5one?5fr@ 10002ef4     rtusb_data.obj
 0001:00001f1c       ??_C@_0CF@NAOBINAP@Number?5of?5fragments?5include?5RTS?5@ 10002f1c     rtusb_data.obj
 0001:00001f44       ??_C@_0BF@GNHDENIC@?$DN?$DN?$DN?$DO?5RTMPSendPacket?6?$AA@ 10002f44     rtusb_data.obj
 0001:00001f60       ??_C@_0EA@OGBHPJKA@?9?9RTMPDeQueuePacket?5?$CFd?5queue?5ful@ 10002f60     rtusb_data.obj
 0001:00001fa0       ??_C@_0CP@BBDGDJCM@?9?9RTMPDeQueuePacket?5?$CFd?5reset?9in?9@ 10002fa0     rtusb_data.obj
 0001:00001fd0       ??_C@_0DC@OFGILKLA@?9?9RTMPDeQueuePacket?5?$CFd?5TxRingTot@ 10002fd0     rtusb_data.obj
 0001:00002004       ??_C@_0CL@MFGAFFNH@?9?9?9?$DORTUSBFreeDescriptorRequest?$CI?$CJ@ 10003004     rtusb_data.obj
 0001:00002030       ??_C@_0BK@BKJDMLJI@?$DM?9?9?9RejectPendingPackets?6?$AA@ 10003030     rtusb_data.obj
 0001:0000204c       ??_C@_0BK@CAELIJAG@?9?9?9?$DORejectPendingPackets?6?$AA@ 1000304c     rtusb_data.obj
 0001:00002068       ??_C@_0CJ@HMDNHMAK@SCANNING?0?5suspend?5MSDU?5transmiss@ 10003068     rtusb_data.obj
 0001:00002094       ??_C@_0CJ@MFMBHLOO@SCAN?5done?0?5resume?5MSDU?5transmiss@ 10003094     rtusb_data.obj
 0001:000020c0       ??_C@_0CL@FGBFFDHO@?5WMM?5in?5used?5but?5EDCA?5not?5valid?5@ 100030c0     rtusb_data.obj
 0001:000020f0       ??_C@_0FB@JAOHBPIG@MLME?5?9?5disassociate?5with?5current@ 100030f0     rtusb_data.obj
 0001:00002144       ??_C@_01EEMJAFIK@?6?$AA@   10003144     rtusb_data.obj
 0001:00002148       ??_C@_05JNBEKFOE@?$CF02x?3?$AA@ 10003148     rtusb_data.obj
 0001:00002150       ??_C@_0BK@OBKNGOKP@Calculated?5TX?5MIC?5value?5?$DN?$AA@ 10003150     rtusb_data.obj
 0001:0000216c       ??_C@_0CB@MKGPKADG@RTUSBHardTransmit?3?5TX?5RING?5full?6@ 1000316c     rtusb_data.obj
 0001:00002190       ??_C@_0CA@BDOPEKFM@?9?9TxringtotalNumber?5?$DN?5?$CFlx?5?$CB?$CB?9?9?6?$AA@ 10003190     rtusb_data.obj
 0001:000021b0       ??_C@_0CA@HHJAEKGO@?9?9?9?9?9?9ERROR?5TX?5RING?5FULL?5?$CFd?5?$CB?$CB?6?$AA@ 100031b0     rtusb_data.obj
 0001:000021d0       ??_C@_0DC@ELKPAKA@RTMPHardTransmit?$CIbEAP?$DN?$CFd?$CJ?5?9?5?$CFs?5k@ 100031d0     rtusb_data.obj
 0001:00002208       ??_C@_1IA@NGMEHGAA@?$AAC?$AA?3?$AA?2?$AAW?$AAI?$AAN?$AAC?$AAE?$AA5?$AA0?$AA0?$AA?2?$AAP?$AAB?$AAW?$AAo?$AAr?$AAk?$AAs?$AAp@ 10003208     rtusb_data.obj
 0001:00002288       ??_C@_0DJ@DBCNFLON@RTMPHardEncrypt?5?9?9?$DO?5Drop?5packet?5@ 10003288     rtusb_data.obj
 0001:000022c4       ??_C@_0DE@HLLDDOPB@RTUSBHardTransmit?5?9?9?$DO?5Ndis?5Packe@ 100032c4     rtusb_data.obj
 0001:000022f8       ??_C@_0BJ@GJFMDJBG@pVirtualAddress?5?$DN?$DN?5NULL?6?$AA@ 100032f8     rtusb_data.obj
 0001:00002314       ??_C@_0P@NEJNAILE@packetsize?3?$CFd?6?$AA@ 10003314     rtusb_data.obj
 0001:00002324       ??_C@_0DL@ONHKKFCJ@RTUSBHardTransmit?5?9?9?$DO?5radar?5dete@ 10003324     rtusb_data.obj
 0001:00002360       ??_C@_0BK@HDKMOMGN@?$DM?9?9?9USB_RxPacketComplete?6?$AA@ 10003360     rtusb_data.obj
 0001:0000237c       ??_C@_0BA@DAHLPGLN@Bulk?5In?5Failed?6?$AA@ 1000337c     rtusb_data.obj
 0001:0000238c       ??_C@_0DC@MJDCHCHB@?$CB?$CB?$CB?5report?5DATA?5?$CIfragmented?$CJ?5to?5@ 1000338c     rtusb_data.obj
 0001:000023c0       ??_C@_0BG@FDIJIFCM@Rx?5MIC?5Value?5error?52?6?$AA@ 100033c0     rtusb_data.obj
 0001:000023d8       ??_C@_0GE@LNANMIMO@?$CB?$CB?$CB?5report?5DATA?5?$CIno?5frag?$CJ?5to?5LLC@ 100033d8     rtusb_data.obj
 0001:00002440       ??_C@_0GG@NMMPCKNB@?$CB?$CB?$CB?5report?5segregated?5MSDU2?5to?5L@ 10003440     rtusb_data.obj
 0001:000024a8       ??_C@_0GG@JFHJPPNC@?$CB?$CB?$CB?5report?5segregated?5MSDU1?5to?5L@ 100034a8     rtusb_data.obj
 0001:00002510       ??_C@_0DE@FPBPLPBI@?$CB?$CB?$CB?5report?5EAPOL?1AIRONET?5DATA?5to@ 10003510     rtusb_data.obj
 0001:00002544       ??_C@_0CL@ELNBKLHP@?$CB?$CB?$CB?5report?5BCAST?5DATA?5to?5LLC?5?$CIle@ 10003544     rtusb_data.obj
 0001:00002570       ??_C@_0CC@NGPJBMOL@2?9Way?3?3RTMPSoftDecryptAES?5Failed@ 10003570     rtusb_data.obj
 0001:00002594       ??_C@_0CE@IGCIAGJB@2?9Way?3?3RTMPSoftDecryptAES?5Comple@ 10003594     rtusb_data.obj
 0001:000025b8       ??_C@_0CD@HPOFFKON@2?9Way?3?3RTMPSoftDecryptTKIP?5Faile@ 100035b8     rtusb_data.obj
 0001:000025dc       ??_C@_0CF@EPMNOMKO@2?9Way?3?3RTMPSoftDecryptTKIP?5Compl@ 100035dc     rtusb_data.obj
 0001:00002604       ??_C@_0BI@BFEENHKE@RTMPCkipDecrypt?5failed?6?$AA@ 10003604     rtusb_data.obj
 0001:0000261c       ??_C@_0CG@BAPGCLHG@RxDone?5?9?5drop?5NULL?5frame?$CIsubtype@ 1000361c     rtusb_data.obj
 0001:00002644       ??_C@_0DB@MLBBMJLG@RxDone?5?9?5drop?5DATA?5frame?5before?5@ 10003644     rtusb_data.obj
 0001:00002678       ??_C@_0BE@FNDAMPBP@duplicate?5frame?5?$CFd?6?$AA@ 10003678     rtusb_data.obj
 0001:0000268c       ??_C@_0BD@PFPOKPOF@?9?9?9?$DORTUSBRxPacket?6?$AA@ 1000368c     rtusb_data.obj
 0001:000026a0       ??_C@_0IA@POPBAFCN@RTUSBDequeueMLMEPacket?3?3PrioRing@ 100036a0     rtusb_data.obj
 0001:00002720       ??_C@_0DK@KCGIBGDJ@not?5enough?5space?5in?5PrioRing?$FLpAd@ 10003720     rtusb_data.obj
 0001:0000275c       ??_C@_0BK@MKFDOFDK@?$DM?9?9?9CleanUpMLMEWaitQueue?6?$AA@ 1000375c     rtusb_data.obj
 0001:00002778       ??_C@_0BK@PAILKHKE@?9?9?9?$DOCleanUpMLMEWaitQueue?6?$AA@ 10003778     rtusb_data.obj
 0001:00002794       ??_C@_0BI@BACCDPCM@?$DM?9?9?9?5MiniportMMRequest?6?$AA@ 10003794     rtusb_data.obj
 0001:000027ac       ??_C@_0CG@FHEFMLON@MiniportMMRequest?5?$CIerror?3?3?5NULL?5@ 100037ac     rtusb_data.obj
 0001:000027d4       ??_C@_0CL@PAFEGNOE@MiniportMMRequest?5?$CIerror?3?3?5MgmtR@ 100037d4     rtusb_data.obj
 0001:00002800       ??_C@_0BI@NOJGLFDJ@?9?9?9?$DO?5MiniportMMRequest?6?$AA@ 10003800     rtusb_data.obj
 0001:00002818       ??_C@_0EA@OOFLGLOH@DUPCHECK?5?9?5replace?5Entry?5?$CFd?0?5MAC@ 10003818     rtusb_data.obj
 0001:00002858       ??_C@_0DM@DAOJGCKM@DUPCHECK?5?9?5Add?5Entry?5?$CFd?0?5MAC?$DN?$CF02@ 10003858     rtusb_data.obj
 0001:00002894       ??_C@_0BD@CDLHMEBF@not?9to?9me?5unicast?6?$AA@ 10003894     rtusb_data.obj
 0001:000028a8       ??_C@_0DA@JIGHBGOJ@Accept?5multicast?5?$CF02x?3?$CF02x?3?$CF02x?3@ 100038a8     rtusb_data.obj
 0001:000028d8       ??_C@_0DN@EJDAJKJM@Rx?5MCAST?5?$CF02x?3?$CF02x?3?$CF02x?3?$CF02x?3?$CF02@ 100038d8     rtusb_data.obj
 0001:00002918       ??_C@_0BP@LDCLPLJJ@Rx?5MCAST?5dropped?5by?5RX_FILTER?6?$AA@ 10003918     rtusb_data.obj
 0001:00002938       ??_C@_0BP@LKINOACC@Rx?5BCAST?5dropped?5by?5RX_FILTER?6?$AA@ 10003938     rtusb_data.obj
 0001:00002958       ??_C@_0BN@PJJLECKM@Rx?5U2M?5dropped?5by?5RX_FILTER?6?$AA@ 10003958     rtusb_data.obj
 0001:00002978       ??_C@_0CC@CLIOIPBG@Rx?5dropped?5by?5MIC?5countermeasure@ 10003978     rtusb_data.obj
 0001:0000299c       ??_C@_0BE@EPBKBMD@Rx?5MIC?5Value?5error?6?$AA@ 1000399c     rtusb_data.obj
 0001:000029b0       ??_C@_0FD@BOJCHIFE@?$CF02x?3?$CF02x?3?$CF02x?3?$CF02x?3?$CF02x?3?$CF02x?3?$CF0@ 100039b0     rtusb_data.obj
 0001:00002a08       ??_C@_0EK@CDOKHMDE@ERROR?3?5CRC?5ok?5but?5CipherErr?5?$CFd?5?$CI@ 10003a08     rtusb_data.obj
 0001:00002a54       ??_C@_0BK@GHKAJGCP@received?5packet?5too?5long?6?$AA@ 10003a54     rtusb_data.obj
 0001:00002a70       ??_C@_0BG@NMJIJKNE@?$DM?9?9?9MlmeHardTransmit?6?$AA@ 10003a70     rtusb_data.obj
 0001:00002a88       ??_C@_0DP@KMMFANBM@RTUSBMlmeHardTransmit?5?9?9?$DO?5radar?5@ 10003a88     rtusb_data.obj
 0001:00002ac8       ??_C@_0BO@CGCMKIBP@?$DM?9?9?9MlmeRate?5?$CFd?5?5?5Channel?5?$CFd?6?$AA@ 10003ac8     rtusb_data.obj
 0001:00002ae8       ??_C@_0BG@NCFDAJPG@?9?9?9?$DOMlmeHardTransmit?6?$AA@ 10003ae8     rtusb_data.obj
 0001:00002b00       ??_C@_0CE@LEPBJPAD@SYNC?5?9?5send?5NULL?5Frame?5?$EA?$CFd?5Mbps?4@ 10003b00     rtusb_data.obj
 0001:00002b24       ??_C@_0BK@PGAIOLJD@Making?5CTS?9to?9self?5Frame?6?$AA@ 10003b24     rtusb_data.obj
 0001:00002b40       ??_C@_0BC@MEPIBLEM@Making?5RTS?5Frame?6?$AA@ 10003b40     rtusb_data.obj
 0001:00002b54       ??_C@_0CJ@FPDCCLCP@Not?5use?5RTS?5Frame?5to?5proect?5MCAS@ 10003b54     rtusb_data.obj
 0001:00002b80       ??_C@_0DA@EAJDKMPL@Making?5RTS?1CTS?5Frame?5failed?0?5typ@ 10003b80     rtusb_data.obj
 0001:00002bb0       ??_C@_19DICJPJO@?$AAT?$AAE?$AAS?$AAT?$AA?$AA@ 10003bb0     rtmp_init.obj
 0001:00002bbc       ??_C@_1BG@IINBLCLB@?$AAD?$AAt?$AAi?$AAm?$AAP?$AAe?$AAr?$AAi?$AAo?$AAd?$AA?$AA@ 10003bbc     rtmp_init.obj
 0001:00002bd4       ??_C@_1CE@PCANMBOM@?$AAA?$AAu?$AAt?$AAo?$AAC?$AAh?$AAa?$AAn?$AAn?$AAe?$AAl?$AAS?$AAe?$AAl?$AAe?$AAc?$AAt?$AA?$AA@ 10003bd4     rtmp_init.obj
 0001:00002bf8       ??_C@_1BC@GBGBNBCD@?$AAC?$AAL?$AAF?$AAa?$AAc?$AAt?$AAo?$AAr?$AA?$AA@ 10003bf8     rtmp_init.obj
 0001:00002c0c       ??_C@_1BC@EGPLFCEP@?$AAN?$AAH?$AAF?$AAa?$AAc?$AAt?$AAo?$AAr?$AA?$AA@ 10003c0c     rtmp_init.obj
 0001:00002c20       ??_C@_1BI@GKAHDKBF@?$AAC?$AAC?$AAX?$AA2?$AAC?$AAo?$AAn?$AAt?$AAr?$AAo?$AAl?$AA?$AA@ 10003c20     rtmp_init.obj
 0001:00002c38       ??_C@_1O@LPLILBCD@?$AAP?$AAS?$AAM?$AAo?$AAd?$AAe?$AA?$AA@ 10003c38     rtmp_init.obj
 0001:00002c48       ??_C@_1BE@KABNOABI@?$AAA?$AAd?$AAh?$AAo?$AAc?$AAO?$AAf?$AAd?$AAm?$AA?$AA@ 10003c48     rtmp_init.obj
 0001:00002c5c       ??_C@_1BI@FJLDDKCH@?$AAN?$AAe?$AAt?$AAw?$AAo?$AAr?$AAk?$AAT?$AAy?$AAp?$AAe?$AA?$AA@ 10003c5c     rtmp_init.obj
 0001:00002c74       ??_C@_1BM@EFMHHLJG@?$AAA?$AAu?$AAt?$AAo?$AAR?$AAe?$AAc?$AAo?$AAn?$AAn?$AAe?$AAc?$AAt?$AA?$AA@ 10003c74     rtmp_init.obj
 0001:00002c90       ??_C@_1BO@MJECKBG@?$AAS?$AAh?$AAo?$AAw?$AAH?$AAi?$AAd?$AAd?$AAe?$AAn?$AAS?$AAS?$AAI?$AAD?$AA?$AA@ 10003c90     rtmp_init.obj
 0001:00002cb0       ??_C@_1M@HCFAIFML@?$AAR?$AAa?$AAd?$AAi?$AAo?$AA?$AA@ 10003cb0     rtmp_init.obj
 0001:00002cbc       ??_C@_1BI@HGMLCLKI@?$AAM?$AAu?$AAl?$AAt?$AAi?$AAp?$AAl?$AAe?$AAI?$AAR?$AAP?$AA?$AA@ 10003cbc     rtmp_init.obj
 0001:00002cd4       ??_C@_1BG@HGDCKNNC@?$AAW?$AAM?$AAM?$AAC?$AAa?$AAp?$AAa?$AAb?$AAl?$AAe?$AA?$AA@ 10003cd4     rtmp_init.obj
 0001:00002cec       ??_C@_1BA@FANIFMBI@?$AAT?$AAX?$AAB?$AAu?$AAr?$AAs?$AAt?$AA?$AA@ 10003cec     rtmp_init.obj
 0001:00002cfc       ??_C@_1BG@BPJAKMMA@?$AAI?$AAE?$AAE?$AAE?$AA8?$AA0?$AA2?$AA1?$AA1?$AAH?$AA?$AA@ 10003cfc     rtmp_init.obj
 0001:00002d14       ??_C@_1CC@CENNGNJ@?$AAF?$AAr?$AAa?$AAm?$AAe?$AAA?$AAg?$AAg?$AAr?$AAe?$AAg?$AAa?$AAt?$AAi?$AAo?$AAn?$AA?$AA@ 10003d14     rtmp_init.obj
 0001:00002d38       ??_C@_1BE@CJFJGBPC@?$AAS?$AAh?$AAo?$AAr?$AAt?$AAS?$AAl?$AAo?$AAt?$AA?$AA@ 10003d38     rtmp_init.obj
 0001:00002d4c       ??_C@_1BK@KPPOILKG@?$AAB?$AAG?$AAP?$AAr?$AAo?$AAt?$AAe?$AAc?$AAt?$AAi?$AAo?$AAn?$AA?$AA@ 10003d4c     rtmp_init.obj
 0001:00002d68       ??_C@_1BO@HGPPFMIN@?$AAN?$AAe?$AAt?$AAw?$AAo?$AAr?$AAk?$AAA?$AAd?$AAd?$AAr?$AAe?$AAs?$AAs?$AA?$AA@ 10003d68     rtmp_init.obj
 0001:00002d88       ??_C@_1BA@HCLACGFM@?$AAW?$AAE?$AAP?$AAK?$AAe?$AAy?$AA4?$AA?$AA@ 10003d88     rtmp_init.obj
 0001:00002d98       ??_C@_1BA@OPGHBOOF@?$AAW?$AAE?$AAP?$AAK?$AAe?$AAy?$AA3?$AA?$AA@ 10003d98     rtmp_init.obj
 0001:00002da8       ??_C@_1BA@FHNLHJIA@?$AAW?$AAE?$AAP?$AAK?$AAe?$AAy?$AA2?$AA?$AA@ 10003da8     rtmp_init.obj
 0001:00002db8       ??_C@_1BA@EFGONGGO@?$AAW?$AAE?$AAP?$AAK?$AAe?$AAy?$AA1?$AA?$AA@ 10003db8     rtmp_init.obj
 0001:00002dc8       ??_C@_1BG@OIMBEMPB@?$AAV?$AAe?$AAn?$AAd?$AAo?$AAr?$AAD?$AAe?$AAs?$AAc?$AA?$AA@ 10003dc8     rtmp_init.obj
 0001:00002de0       ??_C@_19KJNOMKCJ@?$AAS?$AAS?$AAI?$AAD?$AA?$AA@ 10003de0     rtmp_init.obj
 0001:00002dec       ??_C@_1BE@HKNKOMJL@?$AAW?$AAE?$AAP?$AAK?$AAe?$AAy?$AAU?$AAs?$AAe?$AA?$AA@ 10003dec     rtmp_init.obj
 0001:00002e00       ??_C@_1BG@CLENCLJC@?$AAA?$AAu?$AAt?$AAh?$AAe?$AAn?$AAT?$AAy?$AAp?$AAe?$AA?$AA@ 10003e00     rtmp_init.obj
 0001:00002e18       ??_C@_1BG@MHEIMMBG@?$AAE?$AAn?$AAc?$AAr?$AAy?$AAp?$AAt?$AAi?$AAo?$AAn?$AA?$AA@ 10003e18     rtmp_init.obj
 0001:00002e30       ??_C@_1BG@CPCOBECG@?$AAF?$AAr?$AAa?$AAg?$AAT?$AAh?$AAr?$AAe?$AAs?$AAh?$AA?$AA@ 10003e30     rtmp_init.obj
 0001:00002e48       ??_C@_1BE@NCNOFIOB@?$AAR?$AAt?$AAs?$AAT?$AAh?$AAr?$AAe?$AAs?$AAh?$AA?$AA@ 10003e48     rtmp_init.obj
 0001:00002e5c       ??_C@_1BA@DLAHBHMC@?$AAC?$AAh?$AAa?$AAn?$AAn?$AAe?$AAl?$AA?$AA@ 10003e5c     rtmp_init.obj
 0001:00002e6c       ??_C@_1BK@CMGABJAK@?$AAW?$AAi?$AAr?$AAe?$AAl?$AAe?$AAs?$AAs?$AAM?$AAo?$AAd?$AAe?$AA?$AA@ 10003e6c     rtmp_init.obj
 0001:00002e88       ??_C@_1CG@FHJPKHBD@?$AAC?$AAo?$AAu?$AAn?$AAt?$AAr?$AAy?$AAR?$AAe?$AAg?$AAi?$AAo?$AAn?$AAA?$AAB?$AAa?$AAn?$AAd?$AA?$AA@ 10003e88     rtmp_init.obj
 0001:00002eb0       ??_C@_1BM@PHDEHLBE@?$AAC?$AAo?$AAu?$AAn?$AAt?$AAr?$AAy?$AAR?$AAe?$AAg?$AAi?$AAo?$AAn?$AA?$AA@ 10003eb0     rtmp_init.obj
 0001:00002ecc       ??_C@_1O@OADBDALB@?$AAO?$AAp?$AAM?$AAo?$AAd?$AAe?$AA?$AA@ 10003ecc     rtmp_init.obj
 0001:00002ee0       _ccitt_16Table             10003ee0     rtmp_init.obj
 0001:000030e0       ??_C@_07BDGAECLF@CKIP128?$AA@ 100040e0     rtmp_init.obj
 0001:000030e8       ??_C@_06HHMNOKIF@CKIP64?$AA@ 100040e8     rtmp_init.obj
 0001:000030f0       ??_C@_03BKNEFOAH@AES?$AA@  100040f0     rtmp_init.obj
 0001:000030f4       ??_C@_04HNKLFFMO@TKIP?$AA@ 100040f4     rtmp_init.obj
 0001:000030fc       ??_C@_06JCFAKCMD@wep128?$AA@ 100040fc     rtmp_init.obj
 0001:00003104       ??_C@_05PJDLFBFB@wep64?$AA@ 10004104     rtmp_init.obj
 0001:0000310c       ??_C@_04CGFJFPFD@none?$AA@ 1000410c     rtmp_init.obj
 0001:00003114       ??_C@_0CG@OCNACBOC@?$DM?9?9?5RTMPAllocAdapterBlock?0?5Statu@ 10004114     rtmp_init.obj
 0001:0000313c       ??_C@_0CF@OKIAKFAA@Failed?5to?5allocate?5memory?5?9?5ADAP@ 1000413c     rtmp_init.obj
 0001:00003164       ??_C@_0BL@JGKILNFB@?9?9?$DO?5RTMPAllocAdapterBlock?6?$AA@ 10004164     rtmp_init.obj
 0001:00003180       ??_C@_0BF@MLMMNDCF@?$DM?9?9?5NICInitTransmit?6?$AA@ 10004180     rtmp_init.obj
 0001:00003198       ??_C@_0DD@ONNCDAOJ@?$DM?9?9?5ERROR?5in?5Alloc?5TX?5PsPollCont@ 10004198     rtmp_init.obj
 0001:000031cc       ??_C@_0DA@KGPAPHEL@?$DM?9?9?5ERROR?5in?5Alloc?5TX?5RTSContext@ 100041cc     rtmp_init.obj
 0001:000031fc       ??_C@_0DB@GHKDFEHD@?$DM?9?9?5ERROR?5in?5Alloc?5TX?5NullContex@ 100041fc     rtmp_init.obj
 0001:00003230       ??_C@_0DH@OMLLOEPG@?$DM?9?9?5ERROR?5in?5Alloc?5TX?5BeaconCont@ 10004230     rtmp_init.obj
 0001:00003268       ??_C@_0DF@CLCCHGFA@?$DM?9?9?5ERROR?5in?5Alloc?5TX?5MLMEContex@ 10004268     rtmp_init.obj
 0001:000032a0       ??_C@_0DD@JKNKBBIM@?$DM?9?9?5ERROR?5in?5Alloc?5TX?5TxContext?$FL@ 100042a0     rtmp_init.obj
 0001:000032d4       ??_C@_0BF@KPOGPPPE@?9?9?$DO?5NICInitTransmit?6?$AA@ 100042d4     rtmp_init.obj
 0001:000032ec       ??_C@_0BB@CKDCGDNO@?$DM?9?9?5NICInitRecv?6?$AA@ 100042ec     rtmp_init.obj
 0001:00003300       ??_C@_0BB@OPNKMENG@?9?9?$DO?5NICInitRecv?6?$AA@ 10004300     rtmp_init.obj
 0001:00003314       ??_C@_0CF@BPCDNDPB@?$DM?9?9?5RTMPInitAdapterBlock?0?5Status@ 10004314     rtmp_init.obj
 0001:0000333c       ??_C@_0BK@DJIKAFOI@?9?9?$DO?5RTMPInitAdapterBlock?6?$AA@ 1000433c     rtmp_init.obj
 0001:00003358       ??_C@_0BF@BGEGKJLJ@?$DM?9?9?9?5ReleaseAdapter?6?$AA@ 10004358     rtmp_init.obj
 0001:00003370       ??_C@_0BF@GFNLJLB@?9?9?9?$DO?5ReleaseAdapter?6?$AA@ 10004370     rtmp_init.obj
 0001:00003388       ??_C@_0BF@PDOKGADN@?$DM?9?9?5RTMPFreeAdapter?6?$AA@ 10004388     rtmp_init.obj
 0001:000033a0       ??_C@_1HO@HOJMPALM@?$AAC?$AA?3?$AA?2?$AAW?$AAI?$AAN?$AAC?$AAE?$AA5?$AA0?$AA0?$AA?2?$AAP?$AAB?$AAW?$AAo?$AAr?$AAk?$AAs?$AAp@ 100043a0     rtmp_init.obj
 0001:00003420       ??_C@_0BF@JHMAEMOM@?9?9?$DO?5RTMPFreeAdapter?6?$AA@ 10004420     rtmp_init.obj
 0001:00003438       ??_C@_0BD@CKMOPGMM@NumOfBulkInIRP?$DN?$CFd?6?$AA@ 10004438     rtmp_init.obj
 0001:0000344c       ??_C@_0P@NJDHNJBG@WmmCapable?$DN?$CFd?6?$AA@ 1000444c     rtmp_init.obj
 0001:0000345c       ??_C@_0CL@FCFMHIIM@Local?5MAC?5?$DN?5?$CF02x?3?$CF02x?3?$CF02x?3?$CF02x?3@ 1000445c     rtmp_init.obj
 0001:00003488       ??_C@_0BO@OJJINGMM@NHFactori?5?$DN?$CFd?0?5CLFactor?5?$DN?5?$CFd?6?$AA@ 10004488     rtmp_init.obj
 0001:000034a8       ??_C@_0BF@IEPLGABF@CCX2Control?5is?5?$CF08x?6?$AA@ 100044a8     rtmp_init.obj
 0001:000034c0       ??_C@_0BI@IKJPMJHO@WindowsPowerMode?5is?5?$CFd?6?$AA@ 100044c0     rtmp_init.obj
 0001:000034d8       ??_C@_0BG@MEHMEPLP@Software?5Radio?5is?5on?6?$AA@ 100044d8     rtmp_init.obj
 0001:000034f0       ??_C@_0BH@CFIMCAHD@Software?5Radio?5is?5off?6?$AA@ 100044f0     rtmp_init.obj
 0001:00003508       ??_C@_0CP@MKHFOGKI@Vendor?5Description?5?$CILen?$DN?$CFd?0?5Vend@ 10004508     rtmp_init.obj
 0001:00003538       ??_C@_0BL@CNHLFECN@SSID?5?$CILen?$DN?$CFd?0?5ssid?$DN?$CFs?4?4?4?$CJ?6?$AA@ 10004538     rtmp_init.obj
 0001:00003558       ??_C@_0FN@BHMFPOI@AP?5Mode?$DN?$CFd?0?5Channel?$DN?$CFd?0?5Rts?$DN?$CFd?0?5@ 10004558     rtmp_init.obj
 0001:000035b8       ??_C@_0BF@PHFIBNDC@Bogus?5field?5size?5?$CFd?6?$AA@ 100045b8     rtmp_init.obj
 0001:000035d0       ??_C@_0BC@FICEFMOJ@?$DN?50x?$CFx?5?$CIdefault?$CJ?6?$AA@ 100045d0     rtmp_init.obj
 0001:000035e4       ??_C@_0M@BIPEIMIP@?5?9?9?5failed?6?$AA@ 100045e4     rtmp_init.obj
 0001:000035f0       ??_C@_0CF@LBJHNGKL@?$DM?9?9?5NICReadRegParameters?0?5Status@ 100045f0     rtmp_init.obj
 0001:00003618       ??_C@_0BO@DPMOFAFD@NdisOpenConfiguration?5failed?6?$AA@ 10004618     rtmp_init.obj
 0001:00003638       ??_C@_0BK@PGIONEIM@?9?9?$DO?5NICReadRegParameters?6?$AA@ 10004638     rtmp_init.obj
 0001:00003654       ??_C@_0BN@NAMNKJBM@?$DM?9?9?5NICReadEEPROMParameters?6?$AA@ 10004654     rtmp_init.obj
 0001:00003674       ??_C@_0BN@NOKEAOOO@E2PROM?3?5RF?5freq?5offset?$DN0x?$CFx?6?$AA@ 10004674     rtmp_init.obj
 0001:00003698       ??_C@_0EN@LGHBPPJL@E2PROM?3?5A?5Tssi?$FL?94?5?4?4?5?$CL4?$FN?5?$DN?5?$CFd?5?$CFd@ 10004698     rtmp_init.obj
 0001:000036e8       ??_C@_0EN@CFPNPMFA@E2PROM?3?5G?5Tssi?$FL?94?5?4?4?5?$CL4?$FN?5?$DN?5?$CFd?5?$CFd@ 100046e8     rtmp_init.obj
 0001:00003738       ??_C@_0BP@BFNJOEGK@Tx?5power?5for?5channel?5?$CFd?5?3?5?$CF0x?6?$AA@ 10004738     rtmp_init.obj
 0001:00003758       ??_C@_0CH@IMCJKMIN@E2PROM?3?5Version?5?$DN?5?$CFd?0?5FAE?5releas@ 10004758     rtmp_init.obj
 0001:00003780       ??_C@_0BN@NIOCHLKL@?9?9?$DO?5NICReadEEPROMParameters?6?$AA@ 10004780     rtmp_init.obj
 0001:000037a0       ??_C@_0BL@DMFFKKPO@?$DM?9?9?5NICInitAsicFromEEPROM?6?$AA@ 100047a0     rtmp_init.obj
 0001:000037bc       ??_C@_0BG@NCOOFBOB@RFIC?$DN?$CFd?0?5LED?5mode?$DN?$CFd?6?$AA@ 100047bc     rtmp_init.obj
 0001:000037d4       ??_C@_0CO@FKEBOFFH@Use?5Hw?5Radio?5Control?5Pin?$DN?$CFd?$DL?5if?5@ 100047d4     rtmp_init.obj
 0001:00003804       ??_C@_0BE@KNOEGBCE@pAd?9?$DORfIcType?5?$DN?5?$CFd?6?$AA@ 10004804     rtmp_init.obj
 0001:00003818       ??_C@_0CD@EOKJGJHI@E2PROM?5error?0?5hard?5code?5as?50x?$CF04@ 10004818     rtmp_init.obj
 0001:0000383c       ??_C@_0BL@GBFHILNH@?9?9?$DO?5NICInitAsicFromEEPROM?6?$AA@ 1000483c     rtmp_init.obj
 0001:00003858       ??_C@_0BH@DHLGCAAF@?$DM?9?9?5NICInitializeAsic?6?$AA@ 10004858     rtmp_init.obj
 0001:00003870       ??_C@_0BC@LPJHJHGI@BBP?5version?5?$DN?5?$CFd?6?$AA@ 10004870     rtmp_init.obj
 0001:00003884       ??_C@_0CB@JFLFHMHB@MAC?5ASIC?5Version?5number?5?$DN?50x?$CFx?$AN?6@ 10004884     rtmp_init.obj
 0001:000038a8       ??_C@_0BI@OBDMEBLL@?9?9?$DO?5NICInitializeAsic?$AN?6?$AA@ 100048a8     rtmp_init.obj
 0001:000038c0       ??_C@_0BP@DCLOKFHD@?$DM?$DN?$DN?$DN?$DN?5NICLoadFirmware?$CILen?$DN?$CFd?$CJ?6?$AA@ 100048c0     rtmp_init.obj
 0001:000038e0       ??_C@_0CL@JGLJOCGF@NICLoadFirmware?5Failed?$CB?5?$CIntStatu@ 100048e0     rtmp_init.obj
 0001:00003910       ??_C@_0EK@PECDNKPD@NICLoadFirmware?3?5NdisOpenFile?$CI?$CJ?5@ 10004910     rtmp_init.obj
 0001:00003960       ??_C@_0EP@BBNCDKNB@NICLoadFirmware?3?5Ver?$DN?$CFd?4?$CFd?0?5loca@ 10004960     rtmp_init.obj
 0001:000039b0       ??_C@_0DG@BHFAFCBE@NICLoadFirmware?5from?5File?5OK?3?5CR@ 100049b0     rtmp_init.obj
 0001:000039e8       ??_C@_0GH@JGEKOIJM@NICLoadFirmware?3?5CRC?5?$DN?50x?$CF02x?50x@ 100049e8     rtmp_init.obj
 0001:00003a50       ??_C@_0FC@DDCOPDKB@NICLoadFirmware?3?5NdisOpenFile?$CIrt@ 10004a50     rtmp_init.obj
 0001:00003aa4       ??_C@_08FDDFGJNM@rt73?4bin?$AA@ 10004aa4     rtmp_init.obj
 0001:00003ab0       ??_C@_0BH@IHIDDODK@?$DN?$DN?$DN?$DN?$DO?5NICLoadFirmware?6?$AA@ 10004ab0     rtmp_init.obj
 0001:00003ac8       ??_C@_0BB@PHIIJONB@?$DM?9?9?5UserCfgInit?6?$AA@ 10004ac8     rtmp_init.obj
 0001:00003adc       ??_C@_0BB@DCGADJNJ@?9?9?$DO?5UserCfgInit?6?$AA@ 10004adc     rtmp_init.obj
 0001:00003af0       ??_C@_0DE@CCCAEEKK@RTMPSetTimer?5failed?0?5Timer?5hasn?8@ 10004af0     rtmp_init.obj
 0001:00003b24       ??_C@_0DI@GHCOIHIK@NdisMCancelTimer?5failed?0?5Timer?5h@ 10004b24     rtmp_init.obj
 0001:00003b5c       ??_C@_0BP@LEONMOCE@RTMPSetLED?3?3Unknown?5Status?5?$CFd?6?$AA@ 10004b5c     rtmp_init.obj
 0001:00003b80       ??_C@_1FG@GMNPDMHK@?$AAR?$AAT?$AA2?$AA5?$AA0?$AA1?$AAU?$AAS?$AAB?$AA?3?$AA?5?$AA?$DM?$AA?$DN?$AA?$DN?$AA?$DN?$AA?$DN?$AA?$DN?$AA?5?$AAD?$AAr@ 10004b80     rtmp_main.obj
 0001:00003bd8       ??_C@_0CC@OMMKENOM@Calling?5NdisMRegisterMiniport?4?4?4@ 10004bd8     rtmp_main.obj
 0001:00003bfc       ??_C@_0DE@ILKGMENG@?$DM?$DN?$DN?$DN?$DN?5DriverEntry?5failed?5to?5Init@ 10004bfc     rtmp_main.obj
 0001:00003c30       ??_C@_0BE@EHIOEMCA@?$CGStatus?5?$DN?5?$CFc0x?$CF08x?6?$AA@ 10004c30     rtmp_main.obj
 0001:00003c44       ??_C@_0CI@NGCPLDBL@Build?5Date?3?5Feb?5?51?52007?5Time?3?522@ 10004c44     rtmp_main.obj
 0001:00003c6c       ??_C@_0DC@OEKGBEFC@?$DN?$DN?$DN?$DN?$DN?$DN?$DN?$DN?$DN?$DN?$DN?$DN?$DN?$DN?$DN?$DN?$DN?$DN?$DN?$DN?$DN?$DN?$DN?$DN?$DN?$DN?$DN?$DN?$DN?$DN?$DN?$DN@ 10004c6c     rtmp_main.obj
 0001:00003ca0       ??_C@_1EA@KDPAJHGG@?$AAR?$AAT?$AA2?$AA5?$AA0?$AA1?$AAU?$AAS?$AAB?$AA?3?$AA?5?$AA?$DN?$AA?$DN?$AA?$DN?$AA?$DN?$AA?$DN?$AA?$DO?$AA?5?$AAD?$AAr@ 10004ca0     rtmp_main.obj
 0001:00003ce0       ??_C@_0CB@IJCDNANJ@?$DM?$DN?$DN?$DN?$DN?5RTMPInitialize?0?5Status?$DN?$CFx?6@ 10004ce0     rtmp_main.obj
 0001:00003d04       ??_C@_0CD@INENLHOK@RxThread?5handle?$DN0x?$CFx?0?5Priority?$DN?$CF@ 10004d04     rtmp_main.obj
 0001:00003d28       ??_C@_1HO@PINPMNDF@?$AAC?$AA?3?$AA?2?$AAW?$AAI?$AAN?$AAC?$AAE?$AA5?$AA0?$AA0?$AA?2?$AAP?$AAB?$AAW?$AAo?$AAr?$AAk?$AAs?$AAp@ 10004d28     rtmp_main.obj
 0001:00003da8       ??_C@_0CC@FDCOMGPL@MlmeInit?5failed?0?5Status?$FL?$DN0x?$CF08x?$FN@ 10004da8     rtmp_main.obj
 0001:00003dcc       ??_C@_0CL@KGGEDADG@NICInitializeAsic?5failed?0?5Status@ 10004dcc     rtmp_main.obj
 0001:00003df8       ??_C@_0CJ@CDNEOMCG@NICLoadFirmware?5failed?0?5Status?$FL?$DN@ 10004df8     rtmp_main.obj
 0001:00003e24       ??_C@_0CO@JBPFLHDN@NICReadRegParameters?5failed?0?5Sta@ 10004e24     rtmp_main.obj
 0001:00003e54       ??_C@_0CG@OKBKNBGD@RT2501USB?3?5USB_InterfaceStart?5fa@ 10004e54     rtmp_main.obj
 0001:00003e7c       ??_C@_0CO@GCEAKGBJ@RTMPInitAdapterBlock?5failed?0?5Sta@ 10004e7c     rtmp_main.obj
 0001:00003eac       ??_C@_0BP@MLFMABFF@NdisMGetDeviceProperty?5failed?6?$AA@ 10004eac     rtmp_main.obj
 0001:00003ecc       ??_C@_0CP@LFACBFEF@RTMPAllocAdapterBlock?5failed?0?5St@ 10004ecc     rtmp_main.obj
 0001:00003efc       ??_C@_0DH@KNFEHFGD@RT2501USB?3?5Expected?5media?5?$CI?$CFx?$CJ?5i@ 10004efc     rtmp_main.obj
 0001:00003f34       ??_C@_0BG@NIGEMMBH@?$DN?$DN?$DN?$DN?$DO?5RTMPInitialize?6?$AA@ 10004f34     rtmp_main.obj
 0001:00003f4c       ??_C@_0BI@NBHGOOHL@?$DN?$DN?$DN?$DN?$DO?5RTMPCheckForHang?6?$AA@ 10004f4c     rtmp_main.obj
 0001:00003f64       ??_C@_0BA@LJBIDOBK@?$DM?$DN?$DN?$DN?$DN?5RTMPHalt?6?$AA@ 10004f64     rtmp_main.obj
 0001:00003f74       ??_C@_0CL@JKGIAEDF@Halt?5wait?5for?5SCAN_CHANNEL_IN_PR@ 10004f74     rtmp_main.obj
 0001:00003fa0       ??_C@_0CJ@BOGICMLC@Halt?5wait?5for?5RESET_PIPE_IN_PROG@ 10004fa0     rtmp_main.obj
 0001:00003fcc       ??_C@_0BA@BAJOCMCN@PendingRx?5?$DN?5?$CFd?6?$AA@ 10004fcc     rtmp_main.obj
 0001:00003fdc       ??_C@_0BN@IKMIGDBD@Halt?5wait?5for?5MlmeThread?$CB?$CB?$CB?6?$AA@ 10004fdc     rtmp_main.obj
 0001:00003ffc       ??_C@_0CA@OHIIGJIG@Halt?5wait?5for?5ControlThread?$CB?$CB?$CB?6?$AA@ 10004ffc     rtmp_main.obj
 0001:0000401c       ??_C@_0BD@ELKKCIOH@Terminate?5Threads?6?$AA@ 1000501c     rtmp_main.obj
 0001:00004030       ??_C@_0BA@GAOOHNHL@?$DN?$DN?$DN?$DN?$DO?5RTMPHalt?6?$AA@ 10005030     rtmp_main.obj
 0001:00004040       ??_C@_0P@LEBEILCN@?$DM?9?9?9RTMPReset?6?$AA@ 10005040     rtmp_main.obj
 0001:00004050       ??_C@_0P@DCALPAIG@?9?9?9?$DORTMPReset?6?$AA@ 10005050     rtmp_main.obj
 0001:00004060       ??_C@_0BI@NBOMLCPL@?$DM?$DN?$DN?$DN?$DN?5RTMPTransferData?6?$AA@ 10005060     rtmp_main.obj
 0001:00004078       ??_C@_0FB@CEHGILL@?$DN?$DN?$DN?$DN?$DO?5RTMPTransferData?5Ops?$CB?5pAda@ 10005078     rtmp_main.obj
 0001:000040cc       ??_C@_0BI@PPGAJKBG@?$DN?$DN?$DN?$DN?$DO?5RTMPTransferData?6?$AA@ 100050cc     rtmp_main.obj
 0001:000040e4       ??_C@_0BK@MOOEFMFE@?$DM?$DN?$DN?$DN?$DN?5RTMPPnPEventNotify?6?$AA@ 100050e4     rtmp_main.obj
 0001:00004100       ??_C@_0CP@GPELIKKA@RTMPPnPEventNotify?3?5unsupported?5@ 10005100     rtmp_main.obj
 0001:00004130       ??_C@_0CO@CFIHJMCN@RTMPPnPEventNotify?3?5NdisPowerPro@ 10005130     rtmp_main.obj
 0001:00004160       ??_C@_0CN@MLNPNADH@RTMPPnPEventNotify?3?5NdisPowerPro@ 10005160     rtmp_main.obj
 0001:00004190       ??_C@_0DL@EJJFAAF@RTMPPnPEventNotify?3?5NdisDevicePn@ 10005190     rtmp_main.obj
 0001:000041cc       ??_C@_0DH@GADDADJI@RTMPPnPEventNotify?3?5NdisDevicePn@ 100051cc     rtmp_main.obj
 0001:00004204       ??_C@_0BK@BAIBFHID@?$DN?$DN?$DN?$DN?$DO?5RTMPPnPEventNotify?6?$AA@ 10005204     rtmp_main.obj
 0001:00004220       ??_C@_0BC@OCCJCLCM@?$DM?$DN?$DN?$DN?$DN?5MPShutdown?6?$AA@ 10005220     rtmp_main.obj
 0001:00004234       ??_C@_0BC@HBBKLIBG@?$DN?$DN?$DN?$DN?$DO?5MPShutdown?6?$AA@ 10005234     rtmp_main.obj
 0001:00004248       ??_C@_0DD@CAABHMGK@Query?3?3RT_OID_802_11_QUERY_FIRMW@ 10005248     rtmp_info.obj
 0001:00004280       ??_C@_0EF@GHHECJJM@Query?3?3RT_OID_802_11_QUERY_HARDW@ 10005280     rtmp_info.obj
 0001:000042c8       ??_C@_0CP@NIMCLFDE@Query?3?3RT_OID_802_11_QUERY_MULTI@ 100052c8     rtmp_info.obj
 0001:000042f8       ??_C@_0CG@MADDCMLA@Query?3?3RT_OID_802_11_QUERY_WMM?5?$CI@ 100052f8     rtmp_info.obj
 0001:00004320       ??_C@_0CO@OMCLKKIN@Query?3?3RT_OID_802_11_QUERY_AGGRE@ 10005320     rtmp_info.obj
 0001:00004350       ??_C@_0CN@EKNPFEBE@Query?3?3RT_OID_802_11_QUERY_IEEE8@ 10005350     rtmp_info.obj
 0001:00004380       ??_C@_0CK@CNDKPKCI@Query?3?3RT_OID_802_11_QUERY_PREAM@ 10005380     rtmp_info.obj
 0001:000043ac       ??_C@_0DD@HPHAPBAG@Query?3?3RT_OID_802_11_QUERY_TX_PO@ 100053ac     rtmp_info.obj
 0001:000043e0       ??_C@_0DF@NJJHAHOJ@Query?3?3RT_OID_802_11_QUERY_CURRE@ 100053e0     rtmp_info.obj
 0001:00004418       ??_C@_0CL@JJPLDIB@Query?3?3RT_OID_802_11_QUERY_PHY_M@ 10005418     rtmp_info.obj
 0001:00004444       ??_C@_0DP@EODMLAJG@Query?3?3RT_OID_802_11_QUERY_COUNT@ 10005444     rtmp_info.obj
 0001:00004484       ??_C@_0CJ@MFEJFBDC@Query?3?3RT_OID_802_11_QUERY_LINK_@ 10005484     rtmp_info.obj
 0001:000044b0       ??_C@_0CM@KHLEIBOI@Query?3?3OID_802_11_TX_ANTENNA_SEL@ 100054b0     rtmp_info.obj
 0001:000044dc       ??_C@_0CM@JIGKFMFJ@Query?3?3OID_802_11_RX_ANTENNA_SEL@ 100054dc     rtmp_info.obj
 0001:00004508       ??_C@_0CL@OPCGEINM@Query?3?3OID_802_11_NUMBER_OF_ANTE@ 10005508     rtmp_info.obj
 0001:00004534       ??_C@_0CL@OAKNOPEF@Query?3?3OID_802_11_NETWORK_TYPES_@ 10005534     rtmp_info.obj
 0001:00004560       ??_C@_0BP@IEDDLOCD@Query?3?3OID_802_11_STATISTICS?5?6?$AA@ 10005560     rtmp_info.obj
 0001:00004580       ??_C@_0CH@FMGGFNCO@Query?3?3OID_802_11_TX_POWER_LEVEL@ 10005580     rtmp_info.obj
 0001:000045a8       ??_C@_0DA@NLFPODLE@Query?3?3OID_802_11_FRAGMENTATION_@ 100055a8     rtmp_info.obj
 0001:000045d8       ??_C@_0CG@CDOKGMJL@Query?3?3OID_802_11_RTS_THRESHOLD?$CI@ 100055d8     rtmp_info.obj
 0001:00004600       ??_C@_0CM@JIDKLGLC@Query?3?3OID_802_11_NETWORK_TYPE_I@ 10005600     rtmp_info.obj
 0001:00004630       ??_C@_0EH@DKNOICMH@Query?3?3OID_802_11_CONFIGURATION?$CI@ 10005630     rtmp_info.obj
 0001:00004678       ??_C@_0DL@BMOALMIA@Query?3?3OID_802_11_DESIRED_RATES?5@ 10005678     rtmp_info.obj
 0001:000046b4       ??_C@_0CM@LPIHDPBN@Query?3?3OID_802_11_SUPPORTED_RATE@ 100056b4     rtmp_info.obj
 0001:000046e0       ??_C@_0CM@OOENDMPG@Query?3?3OID_802_11_AUTHENTICATION@ 100056e0     rtmp_info.obj
 0001:0000470c       ??_C@_0CH@OBIPKPML@Query?3?3OID_802_11_PRIVACY_FILTER@ 1000570c     rtmp_info.obj
 0001:00004734       ??_C@_0CD@JIHCFKKH@Query?3?3OID_802_11_WEP_STATUS?$CI?$DN?$CFd@ 10005734     rtmp_info.obj
 0001:00004758       ??_C@_0BH@DFBEKOCK@RT_OID_VENDOR_FLIP_IQ?6?$AA@ 10005758     rtmp_info.obj
 0001:00004770       ??_C@_0CD@KOPMNEJE@RT_OID_USB_VENDOR_SWITCH_FUNCTIO@ 10005770     rtmp_info.obj
 0001:00004794       ??_C@_0BK@KDFIGBIJ@RT_OID_USB_VENDOR_UNPLUG?6?$AA@ 10005794     rtmp_info.obj
 0001:000047b0       ??_C@_0BJ@NFGJLEBE@RT_OID_USB_VENDOR_RESET?6?$AA@ 100057b0     rtmp_info.obj
 0001:000047cc       ??_C@_0CJ@OBNEAIFP@Set?3?3RT_OID_802_11_RESET_COUNTER@ 100057cc     rtmp_info.obj
 0001:000047f8       ??_C@_0BI@FPJIPKEB@RT_OID_VENDOR_WRITE_RF?6?$AA@ 100057f8     rtmp_info.obj
 0001:00004810       ??_C@_0BI@LHKEGDFF@RT_OID_VENDOR_READ_BBP?6?$AA@ 10005810     rtmp_info.obj
 0001:00004828       ??_C@_0BJ@HFMCKKMF@RT_OID_VENDOR_WRITE_BBP?6?$AA@ 10005828     rtmp_info.obj
 0001:00004844       ??_C@_0DB@BFJLDGBK@Query?3?3RT_OID_802_11_QUERY_EEPRO@ 10005844     rtmp_info.obj
 0001:00004878       ??_C@_0BM@IMCMMFGP@RT_OID_USB_GET_DEVICE_DESC?6?$AA@ 10005878     rtmp_info.obj
 0001:00004894       ??_C@_0CB@LIIMLHED@RT_OID_USB_VENDOR_EXIT_TESTMODE?6@ 10005894     rtmp_info.obj
 0001:000048b8       ??_C@_0BP@ICFJPPBE@RT_OID_USB_VENDOR_EEPROM_READ?6?$AA@ 100058b8     rtmp_info.obj
 0001:000048d8       ??_C@_0CA@LHPDKOCP@RT_OID_USB_VENDOR_EEPROM_WRITE?6?$AA@ 100058d8     rtmp_info.obj
 0001:000048f8       ??_C@_0CC@DDIKILAH@offset?5?$DN?50x?$CF04x?0?5length?5?$DN?50x?$CF04x@ 100058f8     rtmp_info.obj
 0001:0000491c       ??_C@_0BM@MJFAGCN@RT_OID_VENDOR_GET_COUNTERS?6?$AA@ 1000591c     rtmp_info.obj
 0001:00004938       ??_C@_0DB@GGGKDHOH@Query?3?3OID_802_3_XMIT_MORE_COLLI@ 10005938     rtmp_info.obj
 0001:0000496c       ??_C@_0CP@NDLBBAAK@Query?3?3OID_802_3_XMIT_ONE_COLLIS@ 1000596c     rtmp_info.obj
 0001:0000499c       ??_C@_0DA@ECMCLLK@Query?3?3OID_802_3_RCV_ERROR_ALIGN@ 1000599c     rtmp_info.obj
 0001:000049cc       ??_C@_0CI@OANAMALP@Query?3?3OID_GEN_RCV_NO_BUFFER?5COU@ 100059cc     rtmp_info.obj
 0001:000049f4       ??_C@_0CE@GBJOOJHE@Query?3?3OID_GEN_RCV_ERROR?5COUNTER@ 100059f4     rtmp_info.obj
 0001:00004a18       ??_C@_0CF@GPADPILI@Query?3?3OID_GEN_XMIT_ERROR?5COUNTE@ 10005a18     rtmp_info.obj
 0001:00004a40       ??_C@_0CB@EPMEBIOM@Query?3?3OID_GEN_RCV_OK?5COUNTERS?5?6@ 10005a40     rtmp_info.obj
 0001:00004a64       ??_C@_0CC@CGPDHM@Query?3?3OID_GEN_XMIT_OK?5COUNTERS?5@ 10005a64     rtmp_info.obj
 0001:00004a88       ??_C@_0CC@PKKLEHMG@Query?3?3OID_802_3_MULTICAST_LIST?5@ 10005a88     rtmp_info.obj
 0001:00004aac       ??_C@_0BP@IGHBJLLG@Query?3?3OID_802_3_MAC_OPTIONS?5?6?$AA@ 10005aac     rtmp_info.obj
 0001:00004acc       ??_C@_0CF@JPMDLHOL@Query?3?3OID_802_3_MAXIMUM_LIST_SI@ 10005acc     rtmp_info.obj
 0001:00004af4       ??_C@_0CD@PEMJGHCN@Query?3?3OID_802_3_CURRENT_ADDRESS@ 10005af4     rtmp_info.obj
 0001:00004b18       ??_C@_0CF@GNAHHEHP@Query?3?3OID_802_3_PERMANENT_ADDRE@ 10005b18     rtmp_info.obj
 0001:00004b40       ??_C@_0BN@NEMEENHB@Query?3?3OID_PNP_QUERY_POWER?5?6?$AA@ 10005b40     rtmp_info.obj
 0001:00004b60       ??_C@_0CB@MJGNDIAP@Query?3?3OID_GEN_PHYSICAL_MEDIUM?5?6@ 10005b60     rtmp_info.obj
 0001:00004b84       ??_C@_0CB@KHBFDFFE@Query?3?3OID_GEN_SUPPORTED_GUIDS?5?6@ 10005b84     rtmp_info.obj
 0001:00004ba8       ??_C@_0CG@IAABCDAP@Query?3?3OID_GEN_MAXIMUM_SEND_PACK@ 10005ba8     rtmp_info.obj
 0001:00004bd0       ??_C@_0CG@OGPNBFIA@Query?3?3OID_GEN_MEDIA_CONNECT_STA@ 10005bd0     rtmp_info.obj
 0001:00004bf8       ??_C@_0BN@EGEMJNPE@Query?3?3OID_GEN_MAC_OPTIONS?5?6?$AA@ 10005bf8     rtmp_info.obj
 0001:00004c18       ??_C@_0CH@KDNCIEMI@Query?3?3OID_GEN_CURRENT_PACKET_FI@ 10005c18     rtmp_info.obj
 0001:00004c40       ??_C@_0CA@PFBDKNOM@Query?3?3OID_GEN_DRIVER_VERSION?5?6?$AA@ 10005c40     rtmp_info.obj
 0001:00004c60       ??_C@_0CH@KOCBBIAE@Query?3?3OID_GEN_VENDOR_DRIVER_VER@ 10005c60     rtmp_info.obj
 0001:00004c88       ??_C@_0CE@JJDNJIPD@Query?3?3OID_GEN_VENDOR_DESCRIPTIO@ 10005c88     rtmp_info.obj
 0001:00004cac       ??_C@_0BL@GCGACEMA@Query?3?3OID_GEN_VENDOR_ID?5?6?$AA@ 10005cac     rtmp_info.obj
 0001:00004cc8       ??_C@_0CG@KMOOMODH@Query?3?3OID_GEN_RECEIVE_BUFFER_SP@ 10005cc8     rtmp_info.obj
 0001:00004cf0       ??_C@_0CH@CPGJOFMN@Query?3?3OID_GEN_TRANSMIT_BUFFER_S@ 10005cf0     rtmp_info.obj
 0001:00004d18       ??_C@_0BM@EGKOOEEB@Query?3?3OID_GEN_LINK_SPEED?5?6?$AA@ 10005d18     rtmp_info.obj
 0001:00004d34       ??_C@_0CA@LMLLKGG@Query?3?3OID_GEN_XXX_BLOCK_SIZE?5?6?$AA@ 10005d34     rtmp_info.obj
 0001:00004d54       ??_C@_0CE@HOFCFHAM@Query?3?3OID_GEN_MAXIMUM_FRAME_SIZ@ 10005d54     rtmp_info.obj
 0001:00004d78       ??_C@_0BP@HMEMEIFG@Query?3?3OID_GEN_XXX_LOOKAHEAD?5?6?$AA@ 10005d78     rtmp_info.obj
 0001:00004d98       ??_C@_0BL@NHJAAPPD@Query?3?3OID_GEN_MEDIA_XXX?5?6?$AA@ 10005d98     rtmp_info.obj
 0001:00004db4       ??_C@_0CB@FAIKJOBI@Query?3?3OID_GEN_HARDWARE_STATUS?5?6@ 10005db4     rtmp_info.obj
 0001:00004dd8       ??_C@_0DN@DGDMMALP@Set?3?3RT_OID_802_11_SET_MULTIPLE_@ 10005dd8     rtmp_info.obj
 0001:00004e18       ??_C@_0CD@LNJDNOOH@Set?3?3RT_OID_802_11_SET_WMM?5?$CI?$DN?$CFd?$CJ@ 10005e18     rtmp_info.obj
 0001:00004e3c       ??_C@_0CL@EAFDFCMG@Set?3?3RT_OID_802_11_SET_AGGREGATI@ 10005e3c     rtmp_info.obj
 0001:00004e68       ??_C@_0BO@EHBACENO@InformationBufferLength?5?$DN?5?$CFd?6?$AA@ 10005e68     rtmp_info.obj
 0001:00004e88       ??_C@_0EB@GFIJMLDI@Set?3?3RT_OID_802_11_SET_HARDWARE_@ 10005e88     rtmp_info.obj
 0001:00004ecc       ??_C@_0CB@COKKJBEK@Set?3?3RT_OID_802_11_SET_PREAMBLE?6@ 10005ecc     rtmp_info.obj
 0001:00004ef0       ??_C@_0DG@HDAJJGEE@Set?3?3RT_OID_802_11_SET_COUNTRY_R@ 10005ef0     rtmp_info.obj
 0001:00004f28       ??_C@_0CH@FIJBBKNH@Set?3?3OID_802_11_TX_POWER_LEVEL?5?$CI@ 10005f28     rtmp_info.obj
 0001:00004f50       ??_C@_0DA@OHCGBPIP@Set?3?3OID_802_11_FRAGMENTATION_TH@ 10005f50     rtmp_info.obj
 0001:00004f80       ??_C@_0CF@PPEHBBHG@Set?3?3OID_802_11_RTS_THRESHOLD?5?$CI?$DN@ 10005f80     rtmp_info.obj
 0001:00004fa8       ??_C@_0CA@LENPKACJ@Set?3?3OID_PNP_SET_POWER?0?5?$CFd?5?$CB?$CB?$CB?6?$AA@ 10005fa8     rtmp_info.obj
 0001:00004fc8       ??_C@_0CA@OLCOHIMB@Set?3?3OID_GEN_PROTOCOL_OPTIONS?5?6?$AA@ 10005fc8     rtmp_info.obj
 0001:00004fe8       ??_C@_0FA@MDKNEKCJ@Set?3?3OID_GEN_CURRENT_PACKET_FILT@ 10005fe8     rtmp_info.obj
 0001:00005038       ??_C@_0CB@HIJBKCIP@Set?3?3OID_GEN_CURRENT_LOOKAHEAD?5?6@ 10006038     rtmp_info.obj
 0001:0000505c       ??_C@_0CD@MPEGFFOA@?$CFd?$CJ?5?$CF02x?3?$CF02x?3?$CF02x?3?$CF02x?3?$CF02x?3?$CF02@ 1000605c     rtmp_info.obj
 0001:00005080       ??_C@_0CA@OFBOEBLA@Set?3?3OID_802_3_MULTICAST_LIST?5?6?$AA@ 10006080     rtmp_info.obj
 0001:000050a0       ??_C@_0BH@CNLJEJGO@Query?3?3Size?5too?5short?6?$AA@ 100060a0     rtmp_info.obj
 0001:000050b8       ??_C@_0BM@NMDBEABN@Query?3?3unknown?5OID?50x?$CF08x?5?6?$AA@ 100060b8     rtmp_info.obj
 0001:000050d4       ??_C@_0CJ@IGGABC@Query?3?3RT_OID_802_11_QUERY_OP_MO@ 100060d4     rtmp_info.obj
 0001:00005100       ??_C@_0CM@LJADHKCI@Query?3?3RT_OID_802_11_QUERY_AIRON@ 10006100     rtmp_info.obj
 0001:0000512c       ??_C@_0CG@DKGPFJKC@Query?3?3OID_MH_802_1X_SUPPORTED?5?$CI@ 1000612c     rtmp_info.obj
 0001:00005154       ??_C@_0BI@IPFENO@Query?3?3OID_802_11_TEST?6?$AA@ 10006154     rtmp_info.obj
 0001:0000516c       ??_C@_0CH@CDMOABJI@Query?3?3RT_OID_802_11_EXTRA_INFO?5@ 1000616c     rtmp_info.obj
 0001:00005194       ??_C@_0CH@LOPFFCBD@Query?3?3RT_OID_802_11_QUERY_STA_C@ 10006194     rtmp_info.obj
 0001:000051bc       ??_C@_0CP@LMAAECFI@Query?3?3RT_OID_802_11_QUERY_LAST_@ 100061bc     rtmp_info.obj
 0001:000051ec       ??_C@_0CO@NGAJJALN@Query?3?3RT_OID_802_11_QUERY_NOISE@ 100061ec     rtmp_info.obj
 0001:0000521c       ??_C@_0CI@NOBHOFHJ@Query?3?3RT_OID_802_11_QUERY_RADIO@ 1000621c     rtmp_info.obj
 0001:00005244       ??_C@_0DP@HCEPDJKE@Query?3?3OID_802_11_ASSOCIATION_IN@ 10006244     rtmp_info.obj
 0001:00005288       ??_C@_0EA@BHHDCCMB@Query?3?3OID_802_11_ASSOCIATION_IN@ 10006288     rtmp_info.obj
 0001:000052c8       ??_C@_0DB@OJAJAGCA@BSS?$CD?$CFd?5?9?5?$CFs?0?5Ch?5?$CFd?5?$DN?5?$CFd?5Khz?0?5Sup@ 100062c8     rtmp_info.obj
 0001:000052fc       ??_C@_0CI@PDDIHPPG@Query?3?3?5BssTable?5total?5byte?5coun@ 100062fc     rtmp_info.obj
 0001:00005324       ??_C@_0CE@KLLGDLJC@?$CK?$CK?$CK?$CK?5BssTable?5too?5large?5?$CI?$CFd?5byte@ 10006324     rtmp_info.obj
 0001:00005348       ??_C@_0DA@HAHFKKNK@Query?3?3OID_802_11_BSSID_LIST?5?$CI?$CFd@ 10006348     rtmp_info.obj
 0001:00005378       ??_C@_0EM@KFHGFKCO@Query?3?3OID_802_11_BSSID_LIST?5?$CI?$CFd@ 10006378     rtmp_info.obj
 0001:000053c4       ??_C@_0CD@BLOIIOOA@Query?3?3OID_802_11_POWER_MODE?$CI?$DN?$CFd@ 100063c4     rtmp_info.obj
 0001:000053e8       ??_C@_0CM@HFEMKMIN@Query?3?3OID_802_11_INFRASTRUCTURE@ 100063e8     rtmp_info.obj
 0001:00005414       ??_C@_0CF@KJBKKMNK@Query?3?3OID_802_11_RSSI_TRIGGER?$CI?$DN@ 10006414     rtmp_info.obj
 0001:0000543c       ??_C@_0CF@ODHPKKBM@Query?3?3OID_802_11_RSSI?$CI?$DN?$CFd?5?$DN?$CFd?5?$DN@ 1000643c     rtmp_info.obj
 0001:00005464       ??_C@_0CK@HHECPPIH@Query?3?3OID_802_11_SSID?5?$CILen?$DN?$CFd?0?5@ 10006464     rtmp_info.obj
 0001:00005490       ??_C@_0CB@OAKIBHLA@Query?3?3OID_802_11_BSSID?$CI?$DNEMPTY?$CJ?6@ 10006490     rtmp_info.obj
 0001:000054b4       ??_C@_0DJ@IDKNAJBP@Query?3?3OID_802_11_BSSID?$CI?$DN?$CF02x?3?$CF0@ 100064b4     rtmp_info.obj
 0001:000054f0       ??_C@_0CA@KHEAIIHN@Query?3?3OID_GEN_SUPPORTED_LIST?5?6?$AA@ 100064f0     rtmp_info.obj
 0001:00005510       ??_C@_0BN@CNMNLKDJ@Set?3?3?$CB?$CB?$CB?5unknown?5OID?50x?$CF08x?6?$AA@ 10006510     rtmp_info.obj
 0001:00005530       ??_C@_0CG@EDILLKLA@Set?3?3RT_OID_802_11_SET_OP_MODE?5?$CI@ 10006530     rtmp_info.obj
 0001:00005558       ??_C@_0CP@FKCBNEPE@Set?3?3RT_OID_802_11_LEAP_AUTH_INF@ 10006558     rtmp_info.obj
 0001:00005588       ??_C@_0CP@MDABCIBC@Set?3?3RT_OID_802_11_SET_TX_POWER_@ 10006588     rtmp_info.obj
 0001:000055b8       ??_C@_0EN@FFMPEDHJ@Set?3?3RT_OID_802_11_SET_STA_CONFI@ 100065b8     rtmp_info.obj
 0001:00005608       ??_C@_0CH@PHDOBFHD@Set?3?3RT_OID_802_11_SET_PHY_MODE?5@ 10006608     rtmp_info.obj
 0001:00005630       ??_C@_0CE@PEMBMJJI@Set?3?3RT_OID_802_11_SET_RADIO?5?$CI?$DN?$CF@ 10006630     rtmp_info.obj
 0001:00005654       ??_C@_0CF@EACDIMLE@Set?3?3RT_OID_802_11_CCX20_INFO?5?$CI?$DN@ 10006654     rtmp_info.obj
 0001:0000567c       ??_C@_0CF@GNOAPIHF@Set?3?3RT_OID_802_11_SET_AC_CAM?5?$CI?$DN@ 1000667c     rtmp_info.obj
 0001:000056a4       ??_C@_0CC@PFJIKHAG@Set?3?3OID_802_11_POWER_MODE?5?$CI?$DN?$CFd?$CJ@ 100066a4     rtmp_info.obj
 0001:000056c8       ??_C@_0DP@EOKAOKDM@Set?3?3OID_802_11_CONFIGURATION?5?$CIB@ 100066c8     rtmp_info.obj
 0001:00005708       ??_C@_0EJ@JFEAGLFK@Set?3?3OID_802_11_DESIRED_RATES?5?$CI?$CF@ 10006708     rtmp_info.obj
 0001:00005754       ??_C@_0CE@PNEDDMJM@Set?3?3OID_802_11_RSSI_TRIGGER?5?$CI?$DN?$CF@ 10006754     rtmp_info.obj
 0001:00005778       ??_C@_0CL@FMJJGPLE@Set?3?3OID_802_11_NETWORK_TYPE_IN_@ 10006778     rtmp_info.obj
 0001:000057a4       ??_C@_0DE@DFNNFCDB@Set?3?3OID_802_11_RELOAD_DEFAULTS?5@ 100067a4     rtmp_info.obj
 0001:000057d8       ??_C@_0CC@BNKDOJOB@Set?3?3OID_802_11_WEP_STATUS?5?$CI?$DN?$CFd?$CJ@ 100067d8     rtmp_info.obj
 0001:00005800       ??_C@_0EM@OJFEKMBG@?$CB?$CB?$CB?5Link?5UP?0?5Port?5Not?5Secured?$CB?5i@ 10006800     rtmp_info.obj
 0001:00005850       ??_C@_0EE@LJCODEHF@Heavy?5traffic?5on?5TX?1RX?5ignore?5th@ 10006850     rtmp_info.obj
 0001:00005894       ??_C@_0CO@PKNFCNOA@Set?3?3OID_802_11_BSSID_LIST_SCAN?0@ 10006894     rtmp_info.obj
 0001:000058c4       ??_C@_0CH@CICLDDKH@Set?3?3OID_802_11_PRIVACY_FILTER?5?$CI@ 100068c4     rtmp_info.obj
 0001:000058ec       ??_C@_0CM@JKBNFDAO@Set?3?3OID_802_11_AUTHENTICATION_M@ 100068ec     rtmp_info.obj
 0001:00005918       ??_C@_0BP@KHNLCAOO@Set?3?3OID_802_11_DISASSOCIATE?5?6?$AA@ 10006918     rtmp_info.obj
 0001:00005938       ??_C@_0CD@MCEDEGKD@EnqueueCmd?3?3OID_802_11_REMOVE_WE@ 10006938     rtmp_info.obj
 0001:0000595c       ??_C@_0BM@LAOPJNO@Set?3?3OID_802_11_REMOVE_WEP?6?$AA@ 1000695c     rtmp_info.obj
 0001:00005978       ??_C@_0CA@MCHCILNG@EnqueueCmd?3?3OID_802_11_ADD_WEP?6?$AA@ 10006978     rtmp_info.obj
 0001:00005998       ??_C@_0DA@DILJNKCA@Set?3?3OID_802_11_ADD_WEP?5failed?0?5@ 10006998     rtmp_info.obj
 0001:000059c8       ??_C@_0BJ@CHKDJABG@Set?3?3OID_802_11_ADD_WEP?6?$AA@ 100069c8     rtmp_info.obj
 0001:000059e4       ??_C@_0BG@IJEMAHAJ@Set?3?3OID_802_11_TEST?6?$AA@ 100069e4     rtmp_info.obj
 0001:000059fc       ??_C@_0CM@JLPHGGOJ@Set?3?3OID_802_11_ASSOCIATION_INFO@ 100069fc     rtmp_info.obj
 0001:00005a28       ??_C@_0DD@JIGMCONL@Set?3?3OID_802_11_REMOVE_KEY?5?$CIid?$DN0@ 10006a28     rtmp_info.obj
 0001:00005a5c       ??_C@_0CN@IPAADAFF@Set?3?3OID_802_11_REMOVE_KEY?0?5?5INV@ 10006a5c     rtmp_info.obj
 0001:00005a8c       ??_C@_0BN@CGBBMFOO@RT_OID_802_11_ADD_WPA?5Key?5?$DN?5?$AA@ 10006a8c     rtmp_info.obj
 0001:00005aac       ??_C@_0DD@JEIFOMLD@Set?3?3RT_OID_802_11_ADD_WPA?5?$CIid?$DN0@ 10006aac     rtmp_info.obj
 0001:00005ae0       ??_C@_0DA@LOFBOOKB@Set?3?3OID_802_11_ADD_KEY?5?$CIid?$DN0x?$CFx@ 10006ae0     rtmp_info.obj
 0001:00005b10       ??_C@_0CE@LFLJLKNA@EnqueueCmd?3?3OID_802_11_ADD_KEY_W@ 10006b10     rtmp_info.obj
 0001:00005b34       ??_C@_0CA@GILDMKNK@EnqueueCmd?3?3OID_802_11_ADD_KEY?6?$AA@ 10006b34     rtmp_info.obj
 0001:00005b54       ??_C@_0CI@EAMLODAD@Set?3?3OID_802_11_ADD_KEY?0?5?5INVALI@ 10006b54     rtmp_info.obj
 0001:00005b7c       ??_C@_0CP@DINLEMIF@Set?3?3OID_802_11_INFRASTRUCTURE_M@ 10006b7c     rtmp_info.obj
 0001:00005bac       ??_C@_0CN@JPHDHPDB@Set?3?3OID_802_11_INFRASTRUCTURE_M@ 10006bac     rtmp_info.obj
 0001:00005bdc       ??_C@_0CO@HLOKENEC@Set?3?3OID_802_11_INFRASTRUCTURE_M@ 10006bdc     rtmp_info.obj
 0001:00005c0c       ??_C@_0CI@EIHMKGKC@NDIS_STATUS_MEDIA_DISCONNECT?5Eve@ 10006c0c     rtmp_info.obj
 0001:00005c34       ??_C@_0CH@PHIBEFAD@Set?3?3OID_802_11_SSID?5?$CILen?$DN?$CFd?0Ssi@ 10006c34     rtmp_info.obj
 0001:00005c5c       ??_C@_0CI@FMFFNGEJ@Set?3?3OID_802_11_SSID?5?$CILen?$DN?$CFd?0Ssi@ 10006c5c     rtmp_info.obj
 0001:00005c84       ??_C@_0DM@PCPGCEPG@Set?3?3OID_802_11_SSID?5?$CILen?$DN?$CFd?0Ssi@ 10006c84     rtmp_info.obj
 0001:00005cc0       ??_C@_0DI@KPKKMGFK@Set?3?3RT_OID_802_11_BSSID?5?$CF02x?3?$CF0@ 10006cc0     rtmp_info.obj
 0001:00005cf8       ??_C@_0CJ@LNDELJGC@pAd?9?$DOSharedKey?$FLBSS0?$FN?$FL?$CFd?$FN?4CipherA@ 10006cf8     rtmp_info.obj
 0001:00005d24       ??_C@_0CB@ILBMEPKL@RTMPWPARemoveKeyProc?$CIKeyIdx?$DN?$CFd?$CJ?6@ 10006d24     rtmp_info.obj
 0001:00005d48       ??_C@_0BL@NPGAOOHN@?9?9?9?$DO?5RTMPWPARemoveKeyProc?6?$AA@ 10006d48     rtmp_info.obj
 0001:00005d64       ??_C@_0BD@FHDILJKC@remove?5?$CFs?5key?5?$CD?$CFd?6?$AA@ 10006d64     rtmp_info.obj
 0001:00005d78       ??_C@_0DB@BFBIEKN@RTMPWPARemoveAllKeys?$CIAuthMode?$DN?$CFd@ 10006d78     rtmp_info.obj
 0001:00005dac       ??_C@_0BF@GJCEOIB@RTMPSetPhyMode?$CI?$DN?$CFx?$CJ?6?$AA@ 10006dac     rtmp_info.obj
 0001:00005dc4       ??_C@_0BI@HAKILBDH@RFIC?$FL?$CFd?$FN?0?5Phymode?$CI?$DN?$CFd?$CJ?6?$AA@ 10006dc4     rtmp_info.obj
 0001:00005ddc       ??_C@_0BF@BMFNKGKG@RTMPSetPhyMode?$CI?$DN?$CFd?$CJ?6?$AA@ 10006ddc     rtmp_info.obj
 0001:00005df4       ??_C@_0BI@BNDFFBGF@?$CB?5WEP?5Data?5CRC?5Error?5?$CB?6?$AA@ 10006df4     rtmp_wep.obj
 0001:00005e0c       ??_C@_0BH@MJMAGBCI@Calculated?5MIC?5value?5?$DN?$AA@ 10006e0c     rtmp_tkip.obj
 0001:00005e24       ??_C@_0BB@DICCCLEK@Orig?5MIC?5value?5?$DN?$AA@ 10006e24     rtmp_tkip.obj
 0001:00005e38       ??_C@_0BE@CBHOODBL@?$CB?5TKIP?5MIC?5Error?5?$CB?6?$AA@ 10006e38     rtmp_tkip.obj
 0001:00005e4c       ??_C@_0CE@HFPCFLAC@RTMPSoftDecryptTKIP?5Decript?5done@ 10006e4c     rtmp_tkip.obj
 0001:00005e70       ??_C@_0CL@NEMBPOHF@RTMPSoftDecryptTKIP?0?5WEP?5Data?5MI@ 10006e70     rtmp_tkip.obj
 0001:00005e9c       ??_C@_0CL@CBOOBEAL@RTMPSoftDecryptTKIP?0?5WEP?5Data?5IC@ 10006e9c     rtmp_tkip.obj
 0001:00005ec8       ??_C@_0DM@MOHMDDKB@RTMPSoftDecryptTKIP?5failed?$CB?$CIKeyI@ 10006ec8     rtmp_tkip.obj
 0001:00005f04       ??_C@_0CK@PAGKAPFG@RTMPSoftDecryptAES?0?5WEP?5Data?5MIC@ 10006f04     rtmp_tkip.obj
 0001:00005f30       ??_C@_0CE@NPBEAIGG@ASSOC?5?9?5enqueue?5MT2_ASSOC_TIMEOU@ 10006f30     assoc.obj
 0001:00005f54       ??_C@_0CG@GMHNAAIK@ASSOC?5?9?5enqueue?5MT2_REASSOC_TIME@ 10006f54     assoc.obj
 0001:00005f7c       ??_C@_0CH@INCOHEHM@ASSOC?5?9?5enqueue?5MT2_DISASSOC_TIM@ 10006f7c     assoc.obj
 0001:00005fa4       ??_C@_0DO@GIHLKBMM@ASSOC?5?9?5MlmeAssocReqAction?$CI?$CJ?5san@ 10006fa4     assoc.obj
 0001:00005fe4       ??_C@_0BP@HAMHFODL@ASSOC?5?9?5Send?5ASSOC?5request?4?4?4?6?$AA@ 10006fe4     assoc.obj
 0001:00006004       ??_C@_0DG@DLEENDGL@ASSOC?5?9?5MlmeAssocReqAction?$CI?$CJ?5all@ 10007004     assoc.obj
 0001:0000603c       ??_C@_0DH@GNPKKAFJ@ASSOC?5?9?5Block?5Assoc?5request?5durn@ 1000703c     assoc.obj
 0001:00006074       ??_C@_0DO@JIHAFOIG@ASSOC?5?9?5MlmeReassocReqAction?$CI?$CJ?5s@ 10007074     assoc.obj
 0001:000060b4       ??_C@_0CC@NIANDMMK@ASSOC?5?9?5Send?5RE?9ASSOC?5request?4?4?4@ 100070b4     assoc.obj
 0001:000060d8       ??_C@_0DI@OLCLJDEK@ASSOC?5?9?5MlmeReassocReqAction?$CI?$CJ?5a@ 100070d8     assoc.obj
 0001:00006110       ??_C@_0DJ@IKPPOPCA@ASSOC?5?9?5Block?5ReAssoc?5request?5du@ 10007110     assoc.obj
 0001:00006150       ??_C@_0EE@DGPNBCDD@ASSOC?5?9?5Send?5DISASSOC?5request?$FLBS@ 10007150     assoc.obj
 0001:00006194       ??_C@_0DI@CDNFMMAA@ASSOC?5?9?5MlmeDisassocReqAction?$CI?$CJ?5@ 10007194     assoc.obj
 0001:000061cc       ??_C@_0DA@NLMEEBCP@ASSOC?5?9?5PeerAssocRspAction?$CI?$CJ?5san@ 100071cc     assoc.obj
 0001:000061fc       ??_C@_0CF@GPOCPJOK@?$DMCCX?$DO?5pAd?9?$DOStaCfg?4CkipFlag?5?$DN?50x?$CF@ 100071fc     assoc.obj
 0001:00006224       ??_C@_0CN@JCABFGDO@ASSOC?5?9?5receive?5ASSOC_RSP?5to?5me?5@ 10007224     assoc.obj
 0001:00006254       ??_C@_0DC@INILAGHG@ASSOC?5?9?5PeerReassocRspAction?$CI?$CJ?5s@ 10007254     assoc.obj
 0001:00006288       ??_C@_0DA@GBGOHMON@ASSOC?5?9?5CCKMAssocRspSanity?$CI?$CJ?5san@ 10007288     assoc.obj
 0001:000062b8       ??_C@_0CP@PMPOKCNK@ASSOC?5?9?5receive?5REASSOC_RSP?5to?5m@ 100072b8     assoc.obj
 0001:000062e8       ??_C@_0DH@MOGOHJDP@ASSOC?5?9?5Can?8t?5find?5BSS?5after?5rec@ 100072e8     assoc.obj
 0001:00006320       ??_C@_0DA@ODDHDAFC@ASSOC?5?9?5PeerDisassocAction?$CI?$CJ?5san@ 10007320     assoc.obj
 0001:00006350       ??_C@_0BM@CEEKGCPG@ASSOC?5?9?5AssocTimeoutAction?6?$AA@ 10007350     assoc.obj
 0001:0000636c       ??_C@_0BO@JNNPCJJM@ASSOC?5?9?5ReassocTimeoutAction?6?$AA@ 1000736c     assoc.obj
 0001:0000638c       ??_C@_0BP@KEFGKFCG@ASSOC?5?9?5DisassocTimeoutAction?6?$AA@ 1000738c     assoc.obj
 0001:000063b0       ??_C@_0EE@MIINLNBE@ASSOC?5?9?5InvalidStateWhenAssoc?$CIst@ 100073b0     assoc.obj
 0001:000063f8       ??_C@_0EG@MMEHINEH@ASSOC?5?9?5InvalidStateWhenReassoc?$CI@ 100073f8     assoc.obj
 0001:00006440       ??_C@_0EH@OEFLDGLE@ASSOC?5?9?5InvalidStateWhenDisassoc@ 10007440     assoc.obj
 0001:00006488       ??_C@_0CM@EJEDBDPE@ASSOC?5?9?5Class?53?5Error?0?5Send?5DISA@ 10007488     assoc.obj
 0001:000064b4       ??_C@_0DD@OPEAGCBM@SwitchBetweenWepAndCkip?3?5modify?5@ 100074b4     assoc.obj
 0001:000064e8       ??_C@_0BE@KGNKGALE@AUTH?5?9?5AuthTimeout?6?$AA@ 100074e8     auth.obj
 0001:000064fc       ??_C@_0DA@FNHIJCI@AUTH?5?9?5MlmeAuthReqAction?$CI?$CJ?5sanit@ 100074fc     auth.obj
 0001:0000652c       ??_C@_0DA@MPOCIDDM@AUTH?5?9?5Send?5AUTH?5request?5seq?$CD1?5?$CI@ 1000752c     auth.obj
 0001:0000655c       ??_C@_0DD@KECJJMAM@AUTH?5?9?5MlmeAuthReqAction?$CI?$CJ?5alloc@ 1000755c     auth.obj
 0001:00006590       ??_C@_0DF@GEFOMOIC@AUTH?5?9?5Block?5Auth?5request?5durnin@ 10007590     auth.obj
 0001:000065c8       ??_C@_0CL@EGHBHPJ@AUTH?5?9?5PeerAuthSanity?$CI?$CJ?5sanity?5c@ 100075c8     auth.obj
 0001:000065f4       ??_C@_0CD@MHBJFLCM@AUTH?5?9?5Send?5AUTH?5request?5seq?$CD3?4?4@ 100075f4     auth.obj
 0001:00006618       ??_C@_0DH@POGCGJBJ@AUTH?5?9?5PeerAuthRspAtSeq2Action?$CI?$CJ@ 10007618     auth.obj
 0001:00006650       ??_C@_0DJ@HMHGLDLL@AUTH?5?9?5Receive?5AUTH_RSP?5seq?$CD2?5to@ 10007650     auth.obj
 0001:0000668c       ??_C@_0DE@IELPEDCO@AUTH?5?9?5PeerAuthRspAtSeq4Action?$CI?$CJ@ 1000768c     auth.obj
 0001:000066c0       ??_C@_0CF@KBAGKPNP@AUTH?5?9?5Receive?5AUTH_RSP?5seq?$CD4?5to@ 100076c0     auth.obj
 0001:000066e8       ??_C@_0CM@IGJEBLAE@AUTH?5?9?5Send?5DE?9AUTH?5request?5?$CIRea@ 100076e8     auth.obj
 0001:00006714       ??_C@_0DD@PCPDANEG@AUTH?5?9?5MlmeDeauthReqAction?$CI?$CJ?5all@ 10007714     auth.obj
 0001:00006748       ??_C@_0BK@JNKOGFNM@AUTH?5?9?5AuthTimeoutAction?6?$AA@ 10007748     auth.obj
 0001:00006768       ??_C@_0EC@JIGOAOAF@AUTH?5?9?5InvalidStateWhenAuth?5?$CIsta@ 10007768     auth.obj
 0001:000067ac       ??_C@_0CM@MJJCHKFC@AUTH?5?9?5Class?52?5error?0?5Send?5DEAUT@ 100077ac     auth.obj
 0001:000067d8       ??_C@_0BP@OAFJBIFG@Send?5AUTH?5response?5?$CIseq?$CD2?$CJ?4?4?4?6?$AA@ 100077d8     auth_rsp.obj
 0001:000067f8       ??_C@_0BD@FPHMAHJL@Peer?5AUTH?5fail?4?4?4?6?$AA@ 100077f8     auth_rsp.obj
 0001:0000680c       ??_C@_0DB@IHPPNNAH@AUTH_RSP?5?9?5PeerDeauthAction?$CI?$CJ?5sa@ 1000780c     auth_rsp.obj
 0001:00006840       ??_C@_0DE@KHKHNOPK@AUTH_RSP?5?9?5receive?5DE?9AUTH?5from?5@ 10007840     auth_rsp.obj
 0001:00006874       ??_C@_0BG@OKHOMMNN@SYNC?5?9?5BeaconTimeout?6?$AA@ 10007874     sync.obj
 0001:0000688c       ??_C@_0BG@HLPCBHKO@SYNC?5?9?5Scan?5Timeout?5?6?$AA@ 1000788c     sync.obj
 0001:000068a4       ??_C@_0CO@OPEIFMNL@SYNC?5?9?5MlmeScanReqAction?$CI?$CJ?5sanit@ 100078a4     sync.obj
 0001:000068d4       ??_C@_0DN@GPFBCMLM@MlmeScanReqAction?5?9?9?5Send?5PSM?5Da@ 100078d4     sync.obj
 0001:00006914       ??_C@_0BK@JCBMFILD@SYNC?5?9?5MlmeScanReqAction?6?$AA@ 10007914     sync.obj
 0001:00006930       ??_C@_0EI@JIDFLIDB@SYNC?5?9?5Switch?5to?5ch?5?$CFd?0?5Wait?5BEA@ 10007930     sync.obj
 0001:00006978       ??_C@_0CD@HIEFMEBE@SYNC?5?9?5MlmeJoinReqAction?$CIBSS?5?$CD?$CFd@ 10007978     sync.obj
 0001:0000699c       ??_C@_0DA@NGBBKGMA@SYNC?5?9?5MlmeStartReqAction?$CI?$CJ?5sani@ 1000799c     sync.obj
 0001:000069cc       ??_C@_0DP@NACCAHKL@SYNC?5?9?5MlmeStartReqAction?$CIch?$DN?5?$CFd@ 100079cc     sync.obj
 0001:00006a0c       ??_C@_0DB@DECJICF@SYNC?5?9?5after?5JOIN?0?5SupRateLen?$DN?$CFd@ 10007a0c     sync.obj
 0001:00006a40       ??_C@_0EB@MBFGCIM@SYNC?5?9?5receive?5desired?5BEACON?5at@ 10007a40     sync.obj
 0001:00006a84       ??_C@_0CL@OHGONHHD@SYNC?5?9?5PHY?5sleeps?5for?5?$CFd?5TBTT?0?5D@ 10007a84     sync.obj
 0001:00006ab0       ??_C@_0DD@LJHIBKDP@SYNC?5?9?5AP?5backlog?5broadcast?1mult@ 10007ab0     sync.obj
 0001:00006ae4       ??_C@_0DK@IMBEEHE@SYNC?5?9?5AP?5backlog?5unicast?9to?9me?0@ 10007ae4     sync.obj
 0001:00006b20       ??_C@_0DB@POMPAEFO@SYNC?5?9?5AP?5change?5EDCA?5parameters@ 10007b20     sync.obj
 0001:00006b54       ??_C@_0CH@LMIDECJO@SYNC?5?9?5AP?5forced?5to?5use?5LONG?5pre@ 10007b54     sync.obj
 0001:00006b7c       ??_C@_0CI@NKMHKFBH@SYNC?5?9?5AP?5changed?5B?1G?5protection@ 10007b7c     sync.obj
 0001:00006ba8       ??_C@_0EL@DHFGBJJH@SYNC?5?9?5NdisMIndicateStatus?5?$CK?$CK?$CK?5R@ 10007ba8     sync.obj
 0001:00006bf8       ??_C@_0EI@CKCLGNNN@SYNC?5?9?5NdisMIndicateStatus?5?$CK?$CK?$CK?5R@ 10007bf8     sync.obj
 0001:00006c40       ??_C@_0DF@HNHJMJLG@SYNC?5?9?511b?5peer?5joined?4?5down?9gra@ 10007c40     sync.obj
 0001:00006c78       ??_C@_0O@GANGOBDF@Rx?5My?5BEACON?6?$AA@ 10007c78     sync.obj
 0001:00006c88       ??_C@_0EO@CJMLMEDG@SYNC?5?9?5PeerBeacon?5from?5?$CF02x?3?$CF02x@ 10007c88     sync.obj
 0001:00006cd8       ??_C@_0EK@HECKCKCK@SYNC?5?9?5merge?5to?5the?5IBSS?5with?5bi@ 10007cd8     sync.obj
 0001:00006d24       ??_C@_0CF@LDKJHFHA@SYNC?5?9?5Not?5matched?5wep?5status?5?$CFd@ 10007d24     sync.obj
 0001:00006d4c       ??_C@_0DL@HIDLGPHM@PeerBeacon?$CIcan?5not?5find?5New?5Chan@ 10007d4c     sync.obj
 0001:00006d88       ??_C@_0EL@BLHDMLMA@PeerBeacon?5?9?5STA?5receive?5channel@ 10007d88     sync.obj
 0001:00006dd8       ??_C@_0FD@NMKEIBMC@SYNC?5?9?5New?5AP?5added?5to?5SsidBssTa@ 10007dd8     sync.obj
 0001:00006e2c       ??_C@_0DL@KHEEAHKC@SYNC?5?9?5Send?5PROBE_RSP?5to?5?$CF02x?3?$CF0@ 10007e2c     sync.obj
 0001:00006e68       ??_C@_0CC@HKMEIBBD@SYNC?5?9?5BeaconTimeoutAtJoinAction@ 10007e68     sync.obj
 0001:00006e8c       ??_C@_0CL@CELIKACI@SYNC?5?9?5send?5ProbeReq?5?$EA?5channel?$DN?$CF@ 10007e8c     sync.obj
 0001:00006eb8       ??_C@_0CP@DFNCKPDJ@SYNC?5?9?5ScanNextChannel?$CI?$CJ?5allocat@ 10007eb8     sync.obj
 0001:00006ee8       ??_C@_0CK@JKDMHFEO@MlmeScanReqAction?5?9?9?5Send?5PSM?5Da@ 10007ee8     sync.obj
 0001:00006f14       ??_C@_0DM@CLGDNDLE@SYNC?5?9?5End?5of?5SCAN?0?5restore?5to?5c@ 10007f14     sync.obj
 0001:00006f50       ??_C@_0BI@CKNKHNCA@ScanNextChannel?$CIch?$DN?$CFd?$CJ?6?$AA@ 10007f50     sync.obj
 0001:00006f68       ??_C@_0DL@DPPLBMBC@AYNC?5?9?5InvalidStateWhenScan?$CIstat@ 10007f68     sync.obj
 0001:00006fa4       ??_C@_0DE@DGDDDOIA@InvalidStateWhenJoin?$CIstate?$DN?$CFd?$CJ?4?5@ 10007fa4     sync.obj
 0001:00006fd8       ??_C@_0DF@GOPKNNOJ@InvalidStateWhenStart?$CIstate?$DN?$CFd?$CJ?4@ 10007fd8     sync.obj
 0001:00007010       ??_C@_0BI@LMCMJIBL@SYNC?5?9?5send?5PsPoll?5?4?4?4?6?$AA@ 10008010     sync.obj
 0001:00007028       ??_C@_0CJ@BDIPLDPB@EnqueueBeaconFrame?5allocate?5memo@ 10008028     sync.obj
 0001:00007054       ??_C@_0CH@NBEFGGIA@SYNC?5?9?5driver?5sent?5BEACON?5?$CIlen?$DN?$CF@ 10008054     sync.obj
 0001:0000707c       ??_C@_0BO@BLKMMEKG@force?5out?5a?5ProbeRequest?5?4?4?4?6?$AA@ 1000807c     sync.obj
 0001:0000709c       ??_C@_0N@NADEDOMA@channel?5?$CD?$CFd?6?$AA@ 1000809c     sync.obj
 0001:000070ac       ??_C@_0DP@CLKBLMHF@country?5code?$DN?$CFd?1?$CFd?0?5RFIC?$DN?$CFd?0?5PHY@ 100080ac     sync.obj
 0001:000070ec       ??_C@_0BN@POGCCCPH@countryregion?$DN?$CFd?5not?5support?$AA@ 100080ec     sync.obj
 0001:0000710c       ??_C@_0CN@EHJLKIDP@BuildChannelList?$CIpAd?9?$DOCommonCfg?4@ 1000810c     sync.obj
 0001:0000713c       ??_C@_0CJ@HJHHJFCL@?$CBERROR?$CB?5CNTL?5?9?5Illegal?5message?5t@ 1000813c     connect.obj
 0001:00007168       ??_C@_0DE@OGKJMNPD@CNTL?5?9?5Illegal?5message?5in?5CntlId@ 10008168     connect.obj
 0001:0000719c       ??_C@_00CNPNBAHC@?$AA@     1000819c     connect.obj
 0001:000071a0       ??_C@_0DA@NEDAEIOI@SCAN_PROTECTION?5CNTL?5?9?5Bss?5Table@ 100081a0     connect.obj
 0001:000071d0       ??_C@_0CO@FAOCDMCC@SCAN_PROTECTION?5CNTL?5?9?5Bss?5Table@ 100081d0     connect.obj
 0001:00007200       ??_C@_0BE@JOPIIDIP@CNTL?5?9?5SCAN?5starts?6?$AA@ 10008200     connect.obj
 0001:00007214       ??_C@_0CK@PCPNCK@CNTL?5?9?5No?5matching?5BSS?0?5start?5a?5@ 10008214     connect.obj
 0001:00007240       ??_C@_0CH@KKBIOPMM@NDIS_STATUS_MEDIA_DISCONNECT?5Eve@ 10008240     connect.obj
 0001:00007268       ??_C@_0BL@PPKLHBBN@CNTL?5?9?5drop?5current?5ADHOC?6?$AA@ 10008268     connect.obj
 0001:00007284       ??_C@_0DO@POLPKGPG@CNTL?5?9?5already?5with?5this?5BSSID?4?5@ 10008284     connect.obj
 0001:000072c4       ??_C@_0DP@IAJGDLGN@CNTL?5?9?5disassociate?5with?5current@ 100082c4     connect.obj
 0001:00007304       ??_C@_0CI@GKCIGOMK@CNTL?5?9?5disassociate?5with?5current@ 10008304     connect.obj
 0001:0000732c       ??_C@_0DE@GLCCLOHP@CNTL?5?9?5?$CFd?5BSS?5of?5?$CFd?5BSS?5match?5th@ 1000832c     connect.obj
 0001:00007360       ??_C@_0DC@IICPANIA@CNTL?5?9?5joining?5?$CF02x?3?$CF02x?3?$CF02x?3?$CF0@ 10008360     connect.obj
 0001:00007394       ??_C@_0CJ@IEHKGEAG@CNTL?5?9?5disassociate?5with?5current@ 10008394     connect.obj
 0001:000073c0       ??_C@_0DN@NAOPGFPP@CNTL?5?9?5already?5in?5this?5BSSID?4?5ig@ 100083c0     connect.obj
 0001:00007400       ??_C@_0DI@KNCMOGFJ@CNTL?5?9?5BSSID?5not?5found?4?5reply?5ND@ 10008400     connect.obj
 0001:00007438       ??_C@_0BP@JPMBCMNP@CNTL?5?9?5CntlOidRTBssidProc?5?4?4?4?6?$AA@ 10008438     connect.obj
 0001:00007458       ??_C@_0CG@DPLPNMHD@CNTL?5?9?5Roaming?5in?5MlmeAux?4RoamTa@ 10008458     connect.obj
 0001:00007480       ??_C@_0DI@EOEOHJBD@CNTL?5?9?5No?5matching?5BSS?0?5start?5a?5@ 10008480     connect.obj
 0001:000074b8       ??_C@_0CB@MMEFCBNJ@CNTL?5?9?5Dis?9associate?5successful?6@ 100084b8     connect.obj
 0001:000074dc       ??_C@_0DK@GNDGOIM@CNTL?5?9?5join?5the?5IBSS?5?$DN?5?$CF02x?3?$CF02x@ 100084dc     connect.obj
 0001:00007518       ??_C@_0CC@BKCKLCJK@CNTL?5?9?5Start?5IBSS?5fail?4?5BUG?$CB?$CB?$CB?$CB?$CB@ 10008518     connect.obj
 0001:0000753c       ??_C@_0DN@JKJJHMJO@CNTL?5?9?5start?5a?5new?5IBSS?5?$DN?5?$CF02x?3?$CF@ 1000853c     connect.obj
 0001:0000757c       ??_C@_0CA@NKDBKPGJ@CNTL?5?9?5AUTH?5FAIL?0?5try?5again?4?4?4?6?$AA@ 1000857c     connect.obj
 0001:0000759c       ??_C@_0BA@FEKGKBAD@CNTL?5?9?5AUTH?5OK?6?$AA@ 1000859c     connect.obj
 0001:000075ac       ??_C@_0CJ@OHJNPGKE@CNTL?5?9?5AUTH?5FAIL?0?5give?5up?$DL?5try?5n@ 100085ac     connect.obj
 0001:000075d8       ??_C@_0CG@PPGIBJDF@CNTL?5?9?5AUTH?5FAIL?0?5try?5OPEN?5syste@ 100085d8     connect.obj
 0001:00007600       ??_C@_0BJ@OOEBLIPI@Total?5match?5BSSID?5?$FL?$DN?$CFd?$FN?6?$AA@ 10008600     connect.obj
 0001:0000761c       ??_C@_0DA@MIGPPFMC@CNTL?5?9?5?$CKLEAP?$CK?5AUTH?5FAIL?0?5give?5up@ 1000861c     connect.obj
 0001:0000764c       ??_C@_0CF@LMFEBJPF@CNTL?5?9?5Association?5fails?5on?5BSS?5@ 1000864c     connect.obj
 0001:00007674       ??_C@_0CK@DNGMGINB@CNTL?5?9?5Association?5successful?5on@ 10008674     connect.obj
 0001:000076a0       ??_C@_0CH@NPFFEDFO@CNTL?5?9?5Re?9assocition?5fails?5on?5BS@ 100086a0     connect.obj
 0001:000076c8       ??_C@_0CM@NBDJHLMD@CNTL?5?9?5Re?9assocition?5successful?5@ 100086c8     connect.obj
 0001:000076f4       ??_C@_0BI@DDFADDLO@CCX?3?5CWMax?5CWMin?5?$CFd?5?$CFd?6?$AA@ 100086f4     connect.obj
 0001:0000770c       ??_C@_0CE@KMIEAHPI@NDIS_STATUS_MEDIA_CONNECT?5Event?5@ 1000870c     connect.obj
 0001:00007730       ??_C@_0CI@BNGJHDJM@NDIS_STATUS_MEDIA_DISCONNECT?5Eve@ 10008730     connect.obj
 0001:00007758       ??_C@_0CF@DEEKMBCH@CNTL?5?9?5?$CB?$CB?$CB?5Set?5to?5short?5preamble@ 10008758     connect.obj
 0001:00007780       ??_C@_0CN@BDLKFCMG@?$CB?$CB?$CB?5LINK?5UP?5?$CB?$CB?$CB?5?$CIInfra?$DN?$CFd?0?5AID?$DN?$CF@ 10008780     connect.obj
 0001:000077b0       ??_C@_0CH@BBCHEH@NDIS_STATUS_MEDIA_DISCONNECT?5Eve@ 100087b0     connect.obj
 0001:000077d8       ??_C@_0BD@MFBGAHKA@?$CB?$CB?$CB?5LINK?5DOWN?5?$CB?$CB?$CB?6?$AA@ 100087d8     connect.obj
 0001:000077ec       ??_C@_0CK@DLNELIG@CNTL?5?9?5All?5roaming?5failed?0?5stay?5@ 100087ec     connect.obj
 0001:00007818       ??_C@_0DF@FJJFLKBJ@CNTL?5?9?5All?5BSS?5fail?$DL?5start?5a?5new@ 10008818     connect.obj
 0001:00007850       ??_C@_0BN@NABCMPNC@CNTL?5?9?5iterate?5BSS?5?$CFd?5of?5?$CFd?6?$AA@ 10008850     connect.obj
 0001:00007870       ??_C@_0DA@LFKHACKM@CNTL?5?9?5All?5fast?5roaming?5failed?0?5@ 10008870     connect.obj
 0001:000078a0       ??_C@_0BJ@GPJLADNN@MakeIbssBeacon?5?$CIlen?$DN?$CFd?$CJ?6?$AA@ 100088a0     connect.obj
 0001:000078bc       ??_C@_0DE@FHCBIKLJ@MlmeScanReqSanity?5fail?5?9?5wrong?5B@ 100088bc     sanity.obj
 0001:000078f0       ??_C@_0CN@EEOAAFHE@MlmeStartReqSanity?5fail?5?9?5wrong?5@ 100088f0     sanity.obj
 0001:00007920       ??_C@_0CK@GILPPNOI@MlmeAuthReqSanity?5fail?5?9?5wrong?5a@ 10008920     sanity.obj
 0001:0000794c       ??_C@_0DD@DHNIMLGH@PeerAssocRspSanity?5?9?5ignore?5unre@ 1000894c     sanity.obj
 0001:00007980       ??_C@_0DD@BAJFBEKN@PeerAssocRspSanity?5fail?5?9?5wrong?5@ 10008980     sanity.obj
 0001:000079b4       ??_C@_0CH@BIPFCJDM@PeerAuthSanity?5fail?5?9?5wrong?5algo@ 100089b4     sanity.obj
 0001:000079dc       ??_C@_0CC@DDNHAIDK@PeerAuthSanity?5fail?5?9?5wrong?5Seg?$CD@ 100089dc     sanity.obj
 0001:00007a00       ??_C@_0EB@IMPCBFEO@PeerProbeReqSanity?5fail?5?9?5wrong?5@ 10008a00     sanity.obj
 0001:00007a44       ??_C@_0DJ@FMKPGFHG@PeerProbeReqSanity?5fail?5?9?5wrong?5@ 10008a44     sanity.obj
 0001:00007a80       ??_C@_0DM@KELBNLBJ@PeerBeaconAndProbeRspSanity?5?9?5mi@ 10008a80     sanity.obj
 0001:00007abc       ??_C@_0DF@ENLIANNN@PeerBeaconAndProbeRspSanity?5?9?5un@ 10008abc     sanity.obj
 0001:00007af4       ??_C@_0BE@JGMOOONG@IE_RSN?5length?5?$DN?5?$CFd?6?$AA@ 10008af4     sanity.obj
 0001:00007b08       ??_C@_0CO@GGNNNAAG@PeerBeaconAndProbeRspSanity?5?9?5Re@ 10008b08     sanity.obj
 0001:00007b38       ??_C@_0DC@HFLCAEOC@PeerBeaconAndProbeRspSanity?5?9?5wr@ 10008b38     sanity.obj
 0001:00007b6c       ??_C@_0DA@PMMJHGGB@PeerBeaconAndProbeRspSanity?5?9?5wr@ 10008b6c     sanity.obj
 0001:00007b9c       ??_C@_0DJ@BBLNEPEJ@PeerBeaconAndProbeRspSanity?5?9?5wr@ 10008b9c     sanity.obj
 0001:00007bd8       ??_C@_0DI@NLKPHPBJ@PeerBeaconAndProbeRspSanity?5?9?5wr@ 10008bd8     sanity.obj
 0001:00007c10       ??_C@_0CK@HBCJAKBG@PeerBeaconAndProbeRspSanity?$CIIE_F@ 10008c10     sanity.obj
 0001:00007c3c       ??_C@_0DM@OJHKFFDL@PeerBeaconAndProbeRspSanity?5?9?5wr@ 10008c3c     sanity.obj
 0001:00007c78       ??_C@_0DG@EACFIODC@PeerBeaconAndProbeRspSanity?5?9?5wr@ 10008c78     sanity.obj
 0001:00007cb0       ??_C@_0FK@IFKNOOMO@PeerBeaconAndProbeRspSanity?5?9?5Va@ 10008cb0     sanity.obj
 0001:00007d0c       ??_C@_0CC@FBIOIOKB@WpaMsgTypeSubst?5?3?5return?5FALSE?$DL?5@ 10008d0c     wpa.obj
 0001:00007d30       ??_C@_0BK@FCFKDKFN@?$DM?9?9?9?9?9?5WpaEAPOLKeyAction?6?$AA@ 10008d30     wpa.obj
 0001:00007d4c       ??_C@_0CD@NEKIIEKD@Receive?5EAPOL?5Key?5Group?5Message?5@ 10008d4c     wpa.obj
 0001:00007d70       ??_C@_0CG@MOEKGKHL@Receive?5EAPOL?5Key?5Pairwise?5Messa@ 10008d70     wpa.obj
 0001:00007d98       ??_C@_0CG@MNMOLOBF@Receive?5EAPOL?5Key?5Pairwise?5Messa@ 10008d98     wpa.obj
 0001:00007dc0       ??_C@_0CK@NJMGNMDI@?7?5Key?5descripter?7version?7not?7mat@ 10008dc0     wpa.obj
 0001:00007dec       ??_C@_0CJ@CMKNHCCA@?7?5Key?5descripter?7version?7not?5mat@ 10008dec     wpa.obj
 0001:00007e18       ??_C@_0DA@DABEDLHK@?7?5Key?5descripter?7does?5not?5match?5@ 10008e18     wpa.obj
 0001:00007e48       ??_C@_0P@CLMDLOPL@KeyInfo?5DL?5?$CFd?6?$AA@ 10008e48     wpa.obj
 0001:00007e58       ??_C@_0BE@NLFFPJBE@KeyInfo?5Request?5?$CFd?6?$AA@ 10008e58     wpa.obj
 0001:00007e6c       ??_C@_0BC@EDNACAIN@KeyInfo?5Error?5?$CFd?6?$AA@ 10008e6c     wpa.obj
 0001:00007e80       ??_C@_0BD@EKMAOFCC@KeyInfo?5Secure?5?$CFd?6?$AA@ 10008e80     wpa.obj
 0001:00007e94       ??_C@_0BE@FOAJNOFO@KeyInfo?5Key?5MIC?5?$CFd?6?$AA@ 10008e94     wpa.obj
 0001:00007ea8       ??_C@_0BE@IJJECKJI@KeyInfo?5Key?5Ack?5?$CFd?6?$AA@ 10008ea8     wpa.obj
 0001:00007ebc       ??_C@_0BE@GMCJJBPH@KeyInfo?5Install?5?$CFd?6?$AA@ 10008ebc     wpa.obj
 0001:00007ed0       ??_C@_0BG@BPKLHODP@KeyInfo?5Key?5Index?5?$CFd?6?$AA@ 10008ed0     wpa.obj
 0001:00007ee8       ??_C@_0BF@JMNDEIOC@KeyInfo?5Key?5Type?5?$CFd?6?$AA@ 10008ee8     wpa.obj
 0001:00007f00       ??_C@_0CE@EGIDKOC@KeyInfo?5Key?5Description?5Version?5@ 10008f00     wpa.obj
 0001:00007f24       ??_C@_0BK@CPOPFHLN@?9?9?9?9?9?$DO?5WpaEAPOLKeyAction?6?$AA@ 10008f24     wpa.obj
 0001:00007f40       ??_C@_0BK@JAFFONEP@WpaPairMsg1Action?5?$DM?9?9?9?9?9?6?$AA@ 10008f40     wpa.obj
 0001:00007f5c       ??_C@_0BB@HHEOGBJL@?6?5FrameLen?5?$DN?5?$CFd?6?$AA@ 10008f5c     wpa.obj
 0001:00007f70       ??_C@_08PHECDEMI@?6?5PTK?5?$DN?5?$AA@ 10008f70     wpa.obj
 0001:00007f7c       ??_C@_04BABGPLLL@?$CF2x?9?$AA@ 10008f7c     wpa.obj
 0001:00007f84       ??_C@_07MFJOCGMC@?5PMK?5?$DN?5?$AA@ 10008f84     wpa.obj
 0001:00007f8c       ??_C@_0BK@DOCEMBND@WpaPairMsg1Action?5?9?9?9?9?9?$DO?6?$AA@ 10008f8c     wpa.obj
 0001:00007fa8       ??_C@_0BK@BHPFMICM@WpaPairMsg3Action?5?$DM?9?9?9?9?9?6?$AA@ 10008fa8     wpa.obj
 0001:00007fc4       ??_C@_0DD@LFNKAODL@?5MIC?5VALID?5in?5msg?53?5of?54?9way?5han@ 10008fc4     wpa.obj
 0001:00007ff8       ??_C@_0DH@FFNOHOGI@?5MIC?5Different?5in?5msg?53?5of?54?9way@ 10008ff8     wpa.obj
 0001:00008030       ??_C@_0DI@KIDEAJOH@?5RSN?5IE?5matched?5in?5msg?53?5of?54?9wa@ 10009030     wpa.obj
 0001:00008068       ??_C@_0DI@LNMJCNFK@?5RSN?5IE?5mismatched?5msg?53?5of?54?9wa@ 10009068     wpa.obj
 0001:000080a0       ??_C@_0BK@LJIEOELA@WpaPairMsg3Action?5?9?9?9?9?9?$DO?6?$AA@ 100090a0     wpa.obj
 0001:000080bc       ??_C@_0BL@HNEAFNIJ@WpaGroupMsg1Action?5?$DM?9?9?9?9?9?6?$AA@ 100090bc     wpa.obj
 0001:000080d8       ??_C@_06OAHPBHNA@PTK?5?$DN?5?$AA@ 100090d8     wpa.obj
 0001:000080e0       ??_C@_0DJ@HCPLAPHD@?5MIC?5VALID?5in?5group?5msg?51?5of?52?9w@ 100090e0     wpa.obj
 0001:0000811c       ??_C@_0DN@CHLDNCBC@?5MIC?5Different?5in?5group?5msg?51?5of@ 1000911c     wpa.obj
 0001:0000815c       ??_C@_0BL@NDDBHBBF@WpaGroupMsg1Action?5?9?9?9?9?9?$DO?6?$AA@ 1000915c     wpa.obj
 0001:00008178       ??_C@_0CD@OEBOOBJF@WpaGroupMsg1Action?5?9?9?9?9?9?$DOlen?5?$DN?5?$CF@ 10009178     wpa.obj
 0001:0000819c       ??_C@_0BO@IICCGDDE@?$DM?$DN?$DN?5LeapMachinePerformAction?6?$AA@ 1000919c     leap.obj
 0001:000081bc       ??_C@_0BL@HJOGHDEG@?5LEAP?5EAP?5Message?5Unknown?6?$AA@ 100091bc     leap.obj
 0001:000081d8       ??_C@_0BO@LGJMIHBL@?$DN?$DN?$DO?5LeapMachinePerformAction?6?$AA@ 100091d8     leap.obj
 0001:000081f8       ??_C@_0DK@IKFHLHKJ@LEAP?5?9?5Send?5EAPOL?9Start?5to?5?$CF02x?3@ 100091f8     leap.obj
 0001:00008234       ??_C@_0BF@BEOKAMA@?$DM?$DN?$DN?5LeapStartAction?6?$AA@ 10009234     leap.obj
 0001:0000824c       ??_C@_0DL@PNLBLNDL@Send?5EAPOL?9Start?5Frame?5failed?0?5c@ 1000924c     leap.obj
 0001:00008288       ??_C@_0BF@DNMCKFPH@?$DN?$DN?$DO?5LeapStartAction?6?$AA@ 10009288     leap.obj
 0001:000082a0       ??_C@_0BL@JGGBMCHH@EAPOL?5Frame?5can?8t?5be?5NULL?6?$AA@ 100092a0     leap.obj
 0001:000082bc       ??_C@_0BI@INEGAIKO@?$DM?$DN?$DN?5LeapIdentityAction?6?$AA@ 100092bc     leap.obj
 0001:000082d4       ??_C@_0DL@LHKMGJPJ@Send?5Identify?5response?5failed?0?5c@ 100092d4     leap.obj
 0001:00008310       ??_C@_0BI@DFBLMAMJ@?$DN?$DN?$DO?5LeapIdentityAction?6?$AA@ 10009310     leap.obj
 0001:00008328       ??_C@_0BN@EJEPMPHP@?$DM?$DN?$DN?5LeapPeerChallengeAction?6?$AA@ 10009328     leap.obj
 0001:00008348       ??_C@_0DM@KIOGKBLI@Send?5Challenge?5response?5failed?0?5@ 10009348     leap.obj
 0001:00008384       ??_C@_0BN@JJNMDLJI@?$DN?$DN?$DO?5LeapPeerChallengeAction?6?$AA@ 10009384     leap.obj
 0001:000083a4       ??_C@_0BG@GLHLHILP@?$DM?$DN?$DN?5LeapNakeResponse?6?$AA@ 100093a4     leap.obj
 0001:000083bc       ??_C@_0BG@NDPKFBLF@?$DN?$DN?$DO?5LeapNakeResponse?6?$AA@ 100093bc     leap.obj
 0001:000083d4       ??_C@_0CA@DDODIAFM@?$DM?$DN?$DN?5LeapNetworkChallengeAction?6?$AA@ 100093d4     leap.obj
 0001:000083f4       ??_C@_0DL@PHLLGPLI@Send?5Challenge?5request?5failed?0?5c@ 100093f4     leap.obj
 0001:00008430       ??_C@_0CA@IGJIKAOO@?$DN?$DN?$DO?5LeapNetworkChallengeAction?6?$AA@ 10009430     leap.obj
 0001:00008450       ??_C@_0CC@BOHCDPKJ@?$DM?$DN?$DN?5LeapNetworkChallengeResponse@ 10009450     leap.obj
 0001:00008478       ??_C@_0FD@HPKIKMPD@LEAP?5SessionKey?$FL?$CF02X?3?$CF02X?3?$CF02X?3?$CF@ 10009478     leap.obj
 0001:000084d0       ??_C@_0EF@DHAJOKNM@Verify?5Authenticator?8s?5challenge@ 100094d0     leap.obj
 0001:00008518       ??_C@_0CC@PDOPGGCA@?$DN?$DN?$DO?5LeapNetworkChallengeResponse@ 10009518     leap.obj
 0001:0000853c       ??_C@_0BI@DKOMKJKL@?$DM?$DN?$DN?5LeapEapolKeyAction?6?$AA@ 1000953c     leap.obj
 0001:00008554       ??_C@_0BK@OAAMMFDD@Signature?5verify?5failed?5?6?$AA@ 10009554     leap.obj
 0001:00008570       ??_C@_0BI@ICLBGBMM@?$DN?$DN?$DO?5LeapEapolKeyAction?6?$AA@ 10009570     leap.obj
 0001:00008588       ??_C@_0DF@NAHJKOKC@Add?3Rogue?5AP?$FL?$CF02X?3?$CF02X?3?$CF02X?3?$CF02X@ 10009588     leap.obj
 0001:000085c0       ??_C@_0BF@DABPLDEI@?$DM?$DN?$DN?5LeapAuthTimeout?6?$AA@ 100095c0     leap.obj
 0001:000085d8       ??_C@_0BM@JDCIEHNJ@Enqueue?5LINK?5DOWN?5command?5?6?$AA@ 100095d8     leap.obj
 0001:000085f4       ??_C@_0BF@MJDLGHP@?$DN?$DN?$DO?5LeapAuthTimeout?6?$AA@ 100095f4     leap.obj
 0001:0000860c       ??_C@_0BL@MEIODHBJ@?$DM?$DN?$DN?5LeapSendRogueAPReport?6?$AA@ 1000960c     leap.obj
 0001:00008628       ??_C@_0DI@NDEOMDGJ@Report?5RogueAP?3?$FL?$CF02X?3?$CF02X?3?$CF02X?3?$CF@ 10009628     leap.obj
 0001:00008660       ??_C@_0EK@FNMHFOHD@LeapSendRogueAPReport?$CD1588?3?5Can?8@ 10009660     leap.obj
 0001:000086ac       ??_C@_0BP@OGNGAEAG@Using?5Ckip?5encrypt?5DDP?5packet?6?$AA@ 100096ac     leap.obj
 0001:000086cc       ??_C@_0DH@OEGBEBEK@Send?5DDP?5RogueAP?5list?5failed?0?5ca@ 100096cc     leap.obj
 0001:00008704       ??_C@_0BL@JPOPJKAL@?$DN?$DN?$DO?5LeapSendRogueAPReport?6?$AA@ 10009704     leap.obj
 0001:00008720       ??_C@_0BP@MOCONIDN@?$DM?$DN?$DN?5CCKMAssocRspSanity?5Failed?6?$AA@ 10009720     leap.obj
 0001:00008740       ??_C@_0BL@GPKAJAKD@?$DM?$DN?$DN?5CCKMAssocRspSanity?5OK?6?$AA@ 10009740     leap.obj
 0001:0000875c       ??_C@_0CF@POHOIHBD@?$DN?$DN?$DO?52nd?5time?5CCKM?5MIC?5check?5succ@ 1000975c     leap.obj
 0001:00008784       ??_C@_0CC@KJJMLIOE@?$DN?$DN?$DO?52nd?5time?5CCKM?5MIC?5check?5fail@ 10009784     leap.obj
 0001:000087a8       ??_C@_0BH@MJOKNACO@?$DN?$DN?$DO?51st?5time?5CCKM?5MIC?6?$AA@ 100097a8     leap.obj
 0001:000087c0       ??_C@_0BI@NBEMBPGA@?$DN?$DN?$DO?5CCKMAssocRspSanity?6?$AA@ 100097c0     leap.obj
 0001:000087d8       ??_C@_0EO@FDLNOAPM@Report?5Adjacent?5Previous?5AP?$FL?$CF02X@ 100097d8     leap.obj
 0001:00008828       ??_C@_0EI@FFEPBKGC@CCXAdjacentAPReport?$CD1918?3?5Can?8t?5@ 10009828     leap.obj
 0001:00008a70       ??_C@_0EK@MODKFNNA@RTMPCkipInsertCMIC?0?5Before?5to?5fo@ 10009a70     rtmp_ckipmic.obj
 0001:00008abc       ??_C@_0DI@JBJNPANB@Decrypt?5ERROR?5?3?3?5SN?5?$DN?5?$CFd?0?5KeyIdx@ 10009abc     rtmp_ckipmic.obj
 0001:00008af8       ??_C@_0EJ@IJMAIDDJ@U2M?5Can?8t?5process?5Ckip?5key?0?5Pair@ 10009af8     rtmp_ckipmic.obj
 0001:00008b44       ??_C@_0BG@JMFDLJBE@keylen?5can?8t?5be?5zero?6?$AA@ 10009b44     rtmp_ckipmic.obj
 0001:00008b60       ??_C@_0FJ@PNPKFNG@RTUSBBulkOutDataPacket?5failed?0?5p@ 10009b60     wince_bulk.obj
 0001:00008bbc       ??_C@_0CO@IJEAEDLL@?9?9?9?$DORTUSBBulkOutDataPacket?0?5Bulk@ 10009bbc     wince_bulk.obj
 0001:00008bec       ??_C@_0DF@LODFJEMK@?9?9?9?$DORTUSBBulkOutDataPacket?0?5Bulk@ 10009bec     wince_bulk.obj
 0001:00008c24       ??_C@_0BO@PADIBOMJ@?9?9?9?$DORTUSBBulkOutDataPacket?0?5?6?$AA@ 10009c24     wince_bulk.obj
 0001:00008c44       ??_C@_0CE@PGEKMKFL@?$DM?9?9?9RTUSBBulkOutDataPacketComple@ 10009c44     wince_bulk.obj
 0001:00008c68       ??_C@_0CL@JBEEBDPB@BulkOutDataPacketComplete?$CISTATUS@ 10009c68     wince_bulk.obj
 0001:00008c94       ??_C@_0BM@KOOHGLKG@?$DM?9?9?9RTUSBBulkOutNullFrame?5?6?$AA@ 10009c94     wince_bulk.obj
 0001:00008cb0       ??_C@_0BM@NJPHNGFG@?9?9?9?$DORTUSBBulkOutNullFrame?5?6?$AA@ 10009cb0     wince_bulk.obj
 0001:00008ccc       ??_C@_0CD@IEOAJDHL@?$DM?9?9?9RTUSBBulkOutNullFrameComplet@ 10009ccc     wince_bulk.obj
 0001:00008cf0       ??_C@_0CD@NAMCKGKO@?9?9?9?$DORTUSBBulkOutNullFrameComplet@ 10009cf0     wince_bulk.obj
 0001:00008d14       ??_C@_0BJ@HBKBJBNL@?$DM?9?9?9RTUSBBulkOutBeacon?5?6?$AA@ 10009d14     wince_bulk.obj
 0001:00008d30       ??_C@_0BJ@BMLCMBLK@?9?9?9?$DORTUSBBulkOutBeacon?5?6?$AA@ 10009d30     wince_bulk.obj
 0001:00008d4c       ??_C@_0CB@HJBKGHP@?$DM?9?9?9?5RTUSBBulkOutBeaconComplete?6@ 10009d4c     wince_bulk.obj
 0001:00008d70       ??_C@_0CB@NMOFCMCE@?9?9?9?$DO?5RTUSBBulkOutBeaconComplete?6@ 10009d70     wince_bulk.obj
 0001:00008d94       ??_C@_0BM@EBEMPMOB@?$DM?9?9?9RTUSBBulkOutMLMEPacket?6?$AA@ 10009d94     wince_bulk.obj
 0001:00008db0       ??_C@_0IA@ICCJFKDP@RTUSBBulkOutMLMEPacket?3?3PrioRing@ 10009db0     wince_bulk.obj
 0001:00008e30       ??_C@_0BM@DGFMEBBB@?9?9?9?$DORTUSBBulkOutMLMEPacket?6?$AA@ 10009e30     wince_bulk.obj
 0001:00008e4c       ??_C@_0CE@MJBECIHE@?$DM?9?9?9RTUSBBulkOutMLMEPacketComple@ 10009e4c     wince_bulk.obj
 0001:00008e70       ??_C@_0II@NHBAPID@RTUSBBulkOutMLMEPacketComplete?3?3@ 10009e70     wince_bulk.obj
 0001:00008ef8       ??_C@_0CE@DPPJCMBK@?9?9?9?$DORTUSBBulkOutMLMEPacketComple@ 10009ef8     wince_bulk.obj
 0001:00008f1c       ??_C@_0BJ@NNDMBPEG@?$DM?9?9?9RTUSBBulkOutPsPoll?5?6?$AA@ 10009f1c     wince_bulk.obj
 0001:00008f38       ??_C@_0BJ@LACPEPCH@?9?9?9?$DORTUSBBulkOutPsPoll?5?6?$AA@ 10009f38     wince_bulk.obj
 0001:00008f54       ??_C@_0CA@JAFMDLIB@?$DM?9?9?9RTUSBBulkOutPsPollComplete?6?$AA@ 10009f54     wince_bulk.obj
 0001:00008f74       ??_C@_0CA@FPBPLGKL@?9?9?9?$DORTUSBBulkOutPsPollComplete?6?$AA@ 10009f74     wince_bulk.obj
 0001:00008f98       ??_C@_0EP@EHPACLBJ@RT2501USB?3?5dwTransferLength?$DM24?0?5@ 10009f98     wince_bulk.obj
 0001:00008fe8       ??_C@_0FE@KEJIJBAF@RT2501USB?3?5dwTransferLength?$DN1080@ 10009fe8     wince_bulk.obj
 0001:0000903c       ??_C@_0CK@PIFFPFJK@RT2501USB?3?5TransferStatus?5dwUsbE@ 1000a03c     wince_bulk.obj
 0001:00009068       ??_C@_0CE@NNAAGJ@RT2501USB?3?5USB_TRANSFER?5is?5NULL?$CB@ 1000a068     wince_bulk.obj
 0001:0000908c       ??_C@_1DG@PKFMJANK@?$AAB?$AAO?$AAT?$AA_?$AAD?$AAa?$AAt?$AAa?$AAT?$AAr?$AAa?$AAn?$AAs?$AAf?$AAe?$AAr?$AA?5?$AAe?$AAr?$AAr@ 1000a08c     wince_bulk.obj
 0001:000090c4       ??_C@_0CI@BCFLKEFF@?9?9?9?$DOcan?8t?5RTUSBKickBulkOut?4?5Flag@ 1000a0c4     wince_bulk.obj
 0001:000090ec       ??_C@_0BO@HGDOBABA@MLMEPacket?5?5BulkOutSize?5?$DN?5?$CFd?6?$AA@ 1000a0ec     wince_bulk.obj
 0001:00009110       ??_C@_1EE@IMFIBEFL@?$AAR?$AAT?$AA2?$AA5?$AA0?$AA1?$AAU?$AAS?$AAB?$AA?3?$AA?5?$AAD?$AAa?$AAt?$AAa?$AAT?$AAr?$AAa?$AAn?$AAs@ 1000a110     wince_bulk.obj
 0001:00009154       ??_C@_0BN@GDHDOJHH@?$DM?9?9?9CleanUpDataBulkOutQueue?6?$AA@ 1000a154     wince_bulk.obj
 0001:00009174       ??_C@_0BN@NOLJALNG@?9?9?9?$DOCleanUpDataBulkOutQueue?6?$AA@ 1000a174     wince_bulk.obj
 0001:00009194       ??_C@_0BN@IJLHHALC@?$DM?9?9?9CleanUpMLMEBulkOutQueue?6?$AA@ 1000a194     wince_bulk.obj
 0001:000091b4       ??_C@_0BN@DEHNJCBD@?9?9?9?$DOCleanUpMLMEBulkOutQueue?6?$AA@ 1000a1b4     wince_bulk.obj
 0001:000091d4       ??_C@_0BC@HIOBNOIP@Retry?5count?5?$DN?5?$CFd?6?$AA@ 1000a1d4     wince_io.obj
 0001:000091e8       ??_C@_0EC@HOIIODJO@RTUSBReadBBPRegister?3?5Retry?5coun@ 1000a1e8     wince_io.obj
 0001:00009230       ??_C@_0ED@LDMLPKOK@RTUSBWriteBBPRegister?3?5Retry?5cou@ 1000a230     wince_io.obj
 0001:00009278       ??_C@_0EC@MNDCPFFJ@RTUSBWriteRFRegister?3?5Retry?5coun@ 1000a278     wince_io.obj
 0001:000092bc       ??_C@_0BN@BALDHKEF@?$DM?9?9?9RTUSBEnqueueInternalCmd?6?$AA@ 1000a2bc     wince_io.obj
 0001:000092dc       ??_C@_0BN@KNHJJIOE@?9?9?9?$DORTUSBEnqueueInternalCmd?6?$AA@ 1000a2dc     wince_io.obj
 0001:00009300       ??_C@_1EC@KEFNNBMO@?$AA?5?$AAR?$AAe?$AAs?$AAe?$AAt?$AAD?$AAe?$AAf?$AAa?$AAu?$AAl?$AAt?$AAE?$AAn?$AAd?$AAp?$AAo?$AAi?$AAn@ 1000a300     wince_io.obj
 0001:00009348       ??_C@_1II@CKLGPFDF@?$AAV?$AAe?$AAn?$AAd?$AAe?$AAr?$AAR?$AAe?$AAq?$AA?4?$AAb?$AAm?$AAR?$AAe?$AAq?$AAu?$AAe?$AAs?$AAt?$AAT@ 1000a348     wince_io.obj
 0001:000093d0       ??_C@_1LO@JGAKIAI@?$AAR?$AAT?$AA2?$AA5?$AA0?$AA1?$AAU?$AAS?$AAB?$AA?3?$AA?5?$AA?5?$AAC?$AAB?$AAI?$AAT?$AA_?$AAD?$AAa?$AAt@ 1000a3d0     wince_io.obj
 0001:00009490       ??_C@_1GO@FJAJHAGN@?$AA?9?$AA?$DN?$AA?9?$AA?$DN?$AA?9?$AA?$DN?$AA?9?$AA?$DN?$AA?9?$AA?$DN?$AA?9?$AA?$DN?$AA?9?$AA?$DN?$AA?9?$AA?$DN?$AA?9?$AA?$DN?$AA?9?$AA?$DN@ 1000a490     wince_io.obj
 0001:00009500       ??_C@_1GA@IEJFCPAO@?$AA?5?$AAR?$AAT?$AAU?$AAS?$AAB?$AA_?$AAV?$AAe?$AAn?$AAd?$AAo?$AAr?$AAR?$AAe?$AAq?$AAu?$AAe?$AAs?$AAt@ 1000a500     wince_io.obj
 0001:00009560       ??_C@_1FE@OMABFLBO@?$AAR?$AAT?$AA2?$AA5?$AA0?$AA1?$AAU?$AAS?$AAB?$AA?5?$AAi?$AAs?$AA?5?$AAc?$AAo?$AAn?$AAf?$AAi?$AAg?$AAr@ 1000a560     wince_io.obj
 0001:000095b8       ??_C@_1FA@MDEEMIBE@?$AAR?$AAT?$AA2?$AA5?$AA0?$AA1?$AAU?$AAS?$AAB?$AA?5?$AAi?$AAs?$AA?5?$AAc?$AAo?$AAn?$AAf?$AAi?$AAg?$AAr@ 1000a5b8     wince_io.obj
 0001:00009608       ??_C@_1FE@FEJEEJIL@?$AAR?$AAT?$AA2?$AA5?$AA0?$AA1?$AAU?$AAS?$AAB?$AA?5?$AAi?$AAs?$AA?5?$AAc?$AAo?$AAn?$AAf?$AAi?$AAg?$AAr@ 1000a608     wince_io.obj
 0001:00009660       ??_C@_1FA@MHENDLEH@?$AAR?$AAT?$AA2?$AA5?$AA0?$AA1?$AAU?$AAS?$AAB?$AA?5?$AAi?$AAs?$AA?5?$AAc?$AAo?$AAn?$AAf?$AAi?$AAg?$AAr@ 1000a660     wince_io.obj
 0001:000096b0       ??_C@_0CK@NKDMJHNC@BulkIn?5bIndex?5?$DN?5?$CFd?3?5wMaxPacketSi@ 1000a6b0     wince_io.obj
 0001:000096e0       ??_C@_1EG@FJPBIAJD@?$AAR?$AAT?$AA2?$AA5?$AA0?$AA1?$AAU?$AAS?$AAB?$AA?3?$AA?5?$AAC?$AAr?$AAe?$AAa?$AAt?$AAe?$AAT?$AAh?$AAr@ 1000a6e0     wince_io.obj
 0001:00009728       ??_C@_1EE@CDGFEHAA@?$AAR?$AAT?$AA2?$AA5?$AA0?$AA1?$AAU?$AAS?$AAB?$AA?3?$AA?5?$AAO?$AAp?$AAe?$AAn?$AA?5?$AAB?$AAu?$AAl?$AAk@ 1000a728     wince_io.obj
 0001:0000976c       ??_C@_1DO@FMCOPJPE@?$AAR?$AAT?$AA2?$AA5?$AA0?$AA1?$AAU?$AAS?$AAB?$AA?3?$AA?5?$AAO?$AAp?$AAe?$AAn?$AAP?$AAi?$AAp?$AAe?$AA?5@ 1000a76c     wince_io.obj
 0001:000097ac       ??_C@_0CL@HPIEOPD@BulkOut?5bIndex?5?$DN?5?$CFd?3?5wMaxPacketS@ 1000a7ac     wince_io.obj
 0001:000097d8       ??_C@_1EE@KIMKNOOI@?$AAR?$AAT?$AA2?$AA5?$AA0?$AA1?$AAU?$AAS?$AAB?$AA?3?$AA?5?$AAC?$AAr?$AAe?$AAa?$AAt?$AAe?$AAE?$AAv?$AAe@ 1000a7d8     wince_io.obj
 0001:00009820       ??_C@_1EM@CAJPJOOJ@?$AAR?$AAT?$AA2?$AA5?$AA0?$AA1?$AAU?$AAS?$AAB?$AA?3?$AA?5?$AAO?$AAp?$AAe?$AAn?$AA?5?$AAB?$AAu?$AAl?$AAk@ 1000a820     wince_io.obj
 0001:00009870       ??_C@_1FC@IBBLPNJD@?$AA?$CF?$AAs?$AA?3?$AA?5?$AAC?$AAo?$AAd?$AAe?$AA?5?$AAC?$AAo?$AAv?$AAe?$AAr?$AAa?$AAg?$AAe?$AA?5?$AAT?$AAr@ 1000a870     wince_io.obj
 0001:000098c4       ??_C@_1BM@HKBLIFGJ@?$AAR?$AAT?$AA2?$AA5?$AA0?$AA1?$AAU?$AAS?$AAB?$AA?4?$AAD?$AAL?$AAL?$AA?$AA@ 1000a8c4     wince_io.obj
 0001:000098e0       ??_C@_1HM@JKGEABJJ@?$AAC?$AA?3?$AA?2?$AAW?$AAI?$AAN?$AAC?$AAE?$AA5?$AA0?$AA0?$AA?2?$AAP?$AAB?$AAW?$AAo?$AAr?$AAk?$AAs?$AAp@ 1000a8e0     wince_io.obj
 0001:0000995c       ??_C@_1DM@OMHFKLJC@?$AAR?$AAT?$AA2?$AA5?$AA0?$AA1?$AAU?$AAS?$AAB?$AA?3?$AA?5?$AAO?$AAp?$AAe?$AAn?$AAP?$AAi?$AAp?$AAe?$AA?5@ 1000a95c     wince_io.obj
 0001:00009998       ??_C@_1EM@BDENEPM@?$AAR?$AAT?$AA2?$AA5?$AA0?$AA1?$AAU?$AAS?$AAB?$AA?3?$AA?5?$AAS?$AAe?$AAt?$AAU?$AAs?$AAb?$AAI?$AAn?$AAt@ 1000a998     wince_io.obj
 0001:000099e4       ??_C@_0DC@PLDICDGE@pUsbInterface?9?$DODescriptor?4bInter@ 1000a9e4     wince_io.obj
 0001:00009a18       ??_C@_1DO@CAICHHPB@?$AAR?$AAT?$AA2?$AA5?$AA0?$AA1?$AAU?$AAS?$AAB?$AA?3?$AA?5?$AAI?$AAn?$AAv?$AAa?$AAl?$AAi?$AAd?$AA?5?$AAp@ 1000aa18     wince_io.obj
 0001:00009a58       ??_C@_1DM@KALFKCMM@?$AA?9?$AA?9?$AA?$DO?$AA?5?$AAR?$AAT?$AAU?$AAS?$AAB?$AAC?$AAE?$AA_?$AAC?$AAo?$AAn?$AAf?$AAi?$AAg?$AAu?$AAr@ 1000aa58     wince_io.obj
 0001:00009a98       ??_C@_1EE@IKBLFBPD@?$AAR?$AAT?$AA2?$AA5?$AA0?$AA1?$AAU?$AAS?$AAB?$AA?3?$AA?5?$AA?$DM?$AA?9?$AA?9?$AA?9?$AA?5?$AAR?$AAe?$AAs?$AAe@ 1000aa98     wince_io.obj
 0001:00009ae0       ??_C@_1FG@MGAIOKHC@?$AAR?$AAT?$AA2?$AA5?$AA0?$AA1?$AAU?$AAS?$AAB?$AA?3?$AA?5?$AAR?$AAe?$AAs?$AAe?$AAt?$AAD?$AAe?$AAf?$AAa@ 1000aae0     wince_io.obj
 0001:00009b38       ??_C@_1DO@PFBBFEBO@?$AAR?$AAT?$AA2?$AA5?$AA0?$AA1?$AAU?$AAS?$AAB?$AA?3?$AA?5?$AA?9?$AA?9?$AA?9?$AA?$DO?$AA?5?$AAR?$AAe?$AAs?$AAe@ 1000ab38     wince_io.obj
 0001:00009b78       ??_C@_0BD@KCPOAHFH@?$DM?9?9Command?5Thread?6?$AA@ 1000ab78     wince_io.obj
 0001:00009b8c       ??_C@_0BJ@BELCHNHN@Command?5Thread?5Finished?6?$AA@ 1000ab8c     wince_io.obj
 0001:00009ba8       ??_C@_0CO@HJOIIIGI@?9?9?$DO?5Control?5Thread?5?$CB?$CB?5ERROR?5?$CB?$CB?5d@ 1000aba8     wince_io.obj
 0001:00009bd8       ??_C@_0CI@FLEPJCPM@CmdThread?3?3OID_802_11_POWER_MODE@ 1000abd8     wince_io.obj
 0001:00009c00       ??_C@_0DA@PLOIOHOD@CmdThread?3?3AsicRemoveSharedKeyEn@ 1000ac00     wince_io.obj
 0001:00009c30       ??_C@_0DJ@EFBAEIOP@CmdThread?3?3OID_802_11_REMOVE_KEY@ 1000ac30     wince_io.obj
 0001:00009c6c       ??_C@_0CB@JCEACAEE@CmdThread?3?3RTMPWPARemoveKeyProc?6@ 1000ac6c     wince_io.obj
 0001:00009c90       ??_C@_0BP@FJJJFOOO@CmdThread?3?3OID_802_11_ADD_KEY?6?$AA@ 1000ac90     wince_io.obj
 0001:00009cb0       ??_C@_0EI@OJGHFCDO@CmdThread?3?3OID_802_11_ADD_KEY_WE@ 1000acb0     wince_io.obj
 0001:00009cf8       ??_C@_0DK@BCMPHKKK@CmdThread?3?3OID_802_11_ADD_KEY_WE@ 1000acf8     wince_io.obj
 0001:00009d34       ??_C@_0CO@MDNHJEFM@CmdThread?3?3OID_802_11_REMOVE_WEP@ 1000ad34     wince_io.obj
 0001:00009d64       ??_C@_0DJ@OHADAOII@CmdThread?3?3OID_802_11_REMOVE_WEP@ 1000ad64     wince_io.obj
 0001:00009da0       ??_C@_0DC@MIAFOFP@CmdThread?3?3OID_802_11_REMOVE_WEP@ 1000ada0     wince_io.obj
 0001:00009dd4       ??_C@_0DI@OMKJEDIG@CmdThread?3?3OID_802_11_ADD_WEP?5?$CIK@ 1000add4     wince_io.obj
 0001:00009e0c       ??_C@_0CP@JDCJONPA@CmdThread?3?3OID_802_11_ADD_WEP?0?5I@ 1000ae0c     wince_io.obj
 0001:00009e3c       ??_C@_0CB@OMGNIOPD@CmdThread?3?3OID_802_11_ADD_WEP?5?5?6@ 1000ae3c     wince_io.obj
 0001:00009e60       ??_C@_0CK@PEGEDMKG@SetCMD?3?3RT_OID_802_11_SET_PHY_MO@ 1000ae60     wince_io.obj
 0001:00009e8c       ??_C@_0CH@OLGPNPC@Set?3?3RT_OID_802_11_SET_PREAMBLE?5@ 1000ae8c     wince_io.obj
 0001:00009eb4       ??_C@_0O@PNBKBNAD@I?1Q?5Not?5Flip?6?$AA@ 1000aeb4     wince_io.obj
 0001:00009ec4       ??_C@_09BIFAHHDL@I?1Q?5Flip?6?$AA@ 1000aec4     wince_io.obj
 0001:00009ed0       ??_C@_0DB@IIOOOMJF@RT_OID_VENDOR_SWITCH_FUNCTION?5?9?9@ 1000aed0     wince_io.obj
 0001:00009f04       ??_C@_0BA@HFIMNODF@value?5?$DN?50x?$CF08x?6?$AA@ 1000af04     wince_io.obj
 0001:00009f14       ??_C@_0BA@BKDBDOFB@value?5?$DN?50x?$CF02x?6?$AA@ 1000af14     wince_io.obj
 0001:00009f24       ??_C@_0BB@OELIFODF@offset?5?$DN?50x?$CF02x?6?$AA@ 1000af24     wince_io.obj
 0001:00009f38       ??_C@_0CA@PPNMHDPK@offset?5?$DN?50x?$CF02x?7value?5?$DN?50x?$CF02x?6?$AA@ 1000af38     wince_io.obj
 0001:00009f58       ??_C@_0BM@PGBKONNJ@LinkDown?$CIRT_OID_LINK_DOWN?$CJ?6?$AA@ 1000af58     wince_io.obj
 0001:00009f78       ??_C@_0GB@FJAPGFLD@CmdThread?3?3RT_OID_802_11_SET_STA@ 1000af78     wince_io.obj
 0001:00009fdc       ??_C@_0CM@PECMKDNC@Bulk?5In?5Reset?5Failed?$CB?5Card?5must?5@ 1000afdc     wince_io.obj
 0001:0000a008       ??_C@_0BJ@HGAHBILG@Bulk?5In?5Reset?5Successed?6?$AA@ 1000b008     wince_io.obj
 0001:0000a024       ??_C@_0BK@KINMDOLD@RT_OID_USB_RESET_BULK_IN?6?$AA@ 1000b024     wince_io.obj
 0001:0000a040       ??_C@_0BK@LPDFAGGM@Bulk?5Out?5Reset?5Successed?6?$AA@ 1000b040     wince_io.obj
 0001:0000a05c       ??_C@_0BL@MGFFPAAG@RT_OID_USB_RESET_BULK_OUT?6?$AA@ 1000b05c     wince_io.obj
 0001:0000a078       ??_C@_0DB@FEJPAACB@CmdThread?3?3OID_802_11_TX_ANTENNA@ 1000b078     wince_io.obj
 0001:0000a0ac       ??_C@_0DB@OIMGFNOG@CmdThread?3?3OID_802_11_RX_ANTENNA@ 1000b0ac     wince_io.obj
 0001:0000a0e0       ??_C@_0BD@MHJIODPL@?$CB?$CB?$CB?5Radio?5Off?5?$CB?$CB?$CB?6?$AA@ 1000b0e0     wince_io.obj
 0001:0000a0f4       ??_C@_0BC@OGANFKK@?$CB?$CB?$CB?5Radio?5On?5?$CB?$CB?$CB?6?$AA@ 1000b0f4     wince_io.obj
 0001:0000a108       ??_C@_0BL@LBIJFMJL@?$CB?$CB?$CB?5RT_OID_CHECK_GPIO?5?$CB?$CB?$CB?6?$AA@ 1000b108     wince_io.obj
 0001:0000a124       ??_C@_09BBAMGPBN@Cmd?5?$DN?5?$CFx?6?$AA@ 1000b124     wince_io.obj
 0001:0000a130       ??_C@_0BJ@GILFBCBM@BBP?3ID?$FL0x?$CF02x?$FN?$DN?$FL0x?$CF02x?$FN?6?$AA@ 1000b130     wince_io.obj
 0001:0000a14c       ??_C@_0BN@DMNNPFEH@MAC?3Offset?$FL0x?$CF04x?$FN?$DN?$FL0x?$CF04x?$FN?6?$AA@ 1000b14c     wince_io.obj
 0001:0000a16c       ??_C@_0BC@OIOEAJAE@AGGREGATION?5?$DN?5?$CFd?6?$AA@ 1000b16c     wince_io.obj
 0001:0000a180       ??_C@_0BB@POPOLHKA@ACK?5policy?5?$DN?5?$CFs?6?$AA@ 1000b180     wince_io.obj
 0001:0000a194       ??_C@_09CFPFIELH@BLOCK?9ACK?$AA@ 1000b194     wince_io.obj
 0001:0000a1a0       ??_C@_0BA@HHLPELHL@NO?9EXPLICIT?9ACK?$AA@ 1000b1a0     wince_io.obj
 0001:0000a1b0       ??_C@_06PDABOHKG@NO?9ACK?$AA@ 1000b1b0     wince_io.obj
 0001:0000a1b8       ??_C@_06IOJAGNKJ@NORMAL?$AA@ 1000b1b8     wince_io.obj
 0001:0000a1c0       ??_C@_0CI@KOGDEBCE@turn?5off?5R17?5tuning?0?5restore?5to?5@ 1000b1c0     wince_io.obj
 0001:0000a1e8       ??_C@_0BE@FBOPCBNB@turn?5on?5R17?5tuning?6?$AA@ 1000b1e8     wince_io.obj
 0001:0000a200       ??_C@_0FB@JCNDEDAH@CmdThread?3?3RT_OID_802_11_SET_HAR@ 1000b200     wince_io.obj
 0001:0000a254       ??_C@_1CG@IDFJJPLL@?$AA?$DM?$AA?9?$AA?9?$AAU?$AAs?$AAb?$AAD?$AAe?$AAv?$AAi?$AAc?$AAe?$AAT?$AAe?$AAs?$AAt?$AA?$AN?$AA?6?$AA?$AA@ 1000b254     wince.obj
 0001:0000a27c       ??_C@_1CG@PDFDHLMN@?$AA?9?$AA?9?$AA?$DO?$AAU?$AAs?$AAb?$AAD?$AAe?$AAv?$AAi?$AAc?$AAe?$AAT?$AAe?$AAs?$AAt?$AA?$AN?$AA?6?$AA?$AA@ 1000b27c     wince.obj
 0001:0000a2a4       ??_C@_1CE@LKJAFLA@?$AAC?$AAl?$AAo?$AAs?$AAe?$AAP?$AAi?$AAp?$AAe?$AA?5?$AA0?$AAx?$AA?$CF?$AAx?$AA?$CB?$AA?$AN?$AA?6?$AA?$AA@ 1000b2a4     wince.obj
 0001:0000a2c8       ??_C@_1FE@POOGJMBH@?$AAR?$AAT?$AA2?$AA5?$AA0?$AA1?$AAU?$AAS?$AAB?$AA?3?$AA?5?$AAC?$AAl?$AAo?$AAs?$AAe?$AAP?$AAi?$AAp?$AAe@ 1000b2c8     wince.obj
 0001:0000a31c       ??_C@_1DG@NHDFGBIG@?$AA?$DM?$AA?$DN?$AA?$DN?$AA?$DN?$AA?5?$AAR?$AAe?$AAm?$AAo?$AAv?$AAe?$AAD?$AAe?$AAv?$AAi?$AAc?$AAe?$AAC?$AAo?$AAn@ 1000b31c     wince.obj
 0001:0000a354       ??_C@_1DM@KFGGBHHA@?$AAR?$AAT?$AA2?$AA5?$AA0?$AA1?$AAU?$AAS?$AAB?$AA?3?$AA?5?$AAI?$AAn?$AAv?$AAa?$AAl?$AAi?$AAd?$AA?5?$AAP@ 1000b354     wince.obj
 0001:0000a390       ??_C@_1DM@KIBIHFLC@?$AA?$DN?$AA?$DN?$AA?$DN?$AA?$DO?$AAR?$AAe?$AAm?$AAo?$AAv?$AAe?$AAD?$AAe?$AAv?$AAi?$AAc?$AAe?$AAC?$AAo?$AAn?$AAt@ 1000b390     wince.obj
 0001:0000a3cc       ??_C@_1BE@BMEIGAKF@?$AAR?$AAT?$AA2?$AA5?$AA0?$AA1?$AAU?$AAS?$AAB?$AA?$AA@ 1000b3cc     wince.obj
 0001:0000a3e0       ??_C@_1CM@KHKOFMAF@?$AA?5?$AA?$DM?$AA?$DN?$AA?$DN?$AAU?$AAs?$AAb?$AAD?$AAe?$AAv?$AAi?$AAc?$AAe?$AAN?$AAo?$AAt?$AAi?$AAf?$AAy?$AA?$AN@ 1000b3e0     wince.obj
 0001:0000a40c       ??_C@_1DM@KBFLPHO@?$AAR?$AAT?$AA2?$AA5?$AA0?$AA1?$AAU?$AAS?$AAB?$AA?3?$AA?5?$AAU?$AAn?$AAh?$AAa?$AAn?$AAd?$AAl?$AAe?$AAd@ 1000b40c     wince.obj
 0001:0000a448       ??_C@_1IG@KGNLPKIO@?$AAR?$AAT?$AA2?$AA5?$AAU?$AAS?$AAB?$AA?3?$AA?5?$AAW?$AAa?$AAr?$AAn?$AAi?$AAn?$AAg?$AA?0?$AA?5?$AAu?$AAn@ 1000b448     wince.obj
 0001:0000a4d0       ??_C@_1EC@NALAHCHI@?$AAR?$AAT?$AA2?$AA5?$AAU?$AAS?$AAB?$AA?3?$AA?5?$AAN?$AAd?$AAi?$AAs?$AAD?$AAe?$AAr?$AAe?$AAg?$AAi?$AAs@ 1000b4d0     wince.obj
 0001:0000a514       ??_C@_1BG@NGFFKKHI@?$AAR?$AAT?$AA2?$AA5?$AA0?$AA1?$AAU?$AAS?$AAB?$AA1?$AA?$AA@ 1000b514     wince.obj
 0001:0000a530       ??_C@_1HI@GFOENFGK@?$AAR?$AAT?$AA2?$AA5?$AA0?$AA1?$AAU?$AAS?$AAB?$AA?3?$AA?5?$AAU?$AAs?$AAb?$AAD?$AAe?$AAv?$AAi?$AAc?$AAe@ 1000b530     wince.obj
 0001:0000a5a8       ??_C@_1HG@DOFIFCAC@?$AAC?$AA?3?$AA?2?$AAW?$AAI?$AAN?$AAC?$AAE?$AA5?$AA0?$AA0?$AA?2?$AAP?$AAB?$AAW?$AAo?$AAr?$AAk?$AAs?$AAp@ 1000b5a8     wince.obj
 0001:0000a620       ??_C@_1FO@DNELDMBE@?$AAR?$AAT?$AA2?$AA5?$AA0?$AA1?$AAU?$AAS?$AAB?$AA?3?$AA?5?$AAU?$AAs?$AAb?$AAD?$AAe?$AAv?$AAi?$AAc?$AAe@ 1000b620     wince.obj
 0001:0000a680       ??_C@_1CK@GJGEIJOM@?$AA?$DN?$AA?$DN?$AA?$DO?$AAU?$AAs?$AAb?$AAD?$AAe?$AAv?$AAi?$AAc?$AAe?$AAN?$AAo?$AAt?$AAi?$AAf?$AAy?$AA?$AN?$AA?6@ 1000b680     wince.obj
 0001:0000a6ac       ??_C@_1DC@CKACOHDO@?$AAR?$AAT?$AA2?$AA5?$AA0?$AA1?$AAU?$AAS?$AAB?$AA?3?$AA?5?$AA?$DM?$AA?$DN?$AA?$DN?$AAD?$AAl?$AAl?$AAE?$AAn?$AAt@ 1000b6ac     wince.obj
 0001:0000a6e0       ??_C@_1EA@PAECMEML@?$AAR?$AAT?$AA2?$AA5?$AA0?$AA1?$AAU?$AAS?$AAB?$AA?3?$AA?5?$AAD?$AAL?$AAL?$AA_?$AAP?$AAR?$AAO?$AAC?$AAE@ 1000b6e0     wince.obj
 0001:0000a720       ??_C@_1EA@FMPHAKCD@?$AAR?$AAT?$AA2?$AA5?$AA0?$AA1?$AAU?$AAS?$AAB?$AA?3?$AA?5?$AAD?$AAL?$AAL?$AA_?$AAP?$AAR?$AAO?$AAC?$AAE@ 1000b720     wince.obj
 0001:0000a760       ??_C@_1DC@HDKJLDAL@?$AAR?$AAT?$AA2?$AA5?$AA0?$AA1?$AAU?$AAS?$AAB?$AA?3?$AA?5?$AA?$DN?$AA?$DN?$AA?$DO?$AAD?$AAl?$AAl?$AAE?$AAn?$AAt@ 1000b760     wince.obj
 0001:0000a794       ??_C@_0BN@BGKGACPE@?$DM?9?9?5RTUSBCE_InterfaceStart?$AN?6?$AA@ 1000b794     wince.obj
 0001:0000a7b8       ??_C@_1GC@NFKFFAMN@?$AAR?$AAT?$AA2?$AA5?$AA0?$AA1?$AAU?$AAS?$AAB?$AA?3?$AA?5?$AAR?$AAe?$AAg?$AAi?$AAs?$AAt?$AAe?$AAr?$AAN@ 1000b7b8     wince.obj
 0001:0000a820       ??_C@_1EC@BANDLFJ@?$AAR?$AAT?$AA2?$AA5?$AA0?$AA1?$AAU?$AAS?$AAB?$AA?3?$AA?5?$AAC?$AAr?$AAe?$AAa?$AAt?$AAe?$AAE?$AAv?$AAe@ 1000b820     wince.obj
 0001:0000a864       ??_C@_0CA@LKGGHNAN@RTUSBCE_ConfigureDevice?5failed?6?$AA@ 1000b864     wince.obj
 0001:0000a884       ??_C@_0CP@EJHHJEAK@?$EA?$EA?$EA?5RTUSBCE_InterfaceStart?5pAdap@ 1000b884     wince.obj
 0001:0000a8b4       ??_C@_0BN@BOIJNAED@?9?9?$DO?5RTUSBCE_InterfaceStart?$AN?6?$AA@ 1000b8b4     wince.obj
 0001:0000a8d4       ??_C@_0BG@LLCIHIEL@?$DN?$DN?$DOActivateDeviceEx?$AN?6?$AA@ 1000b8d4     wince.obj
 0001:0000a8f0       ??_C@_1EK@DHDNAADI@?$AAR?$AAT?$AA2?$AA5?$AA0?$AA1?$AAU?$AAS?$AAB?$AA?3?$AA?5?$AA?$DM?$AA?$DN?$AA?$DN?$AA?$DN?$AA?$DN?$AA?$DN?$AA?$DN?$AA?5?$AAU@ 1000b8f0     wince.obj
 0001:0000a940       ??_C@_1HG@BAFKOBAN@?$AAR?$AAT?$AA2?$AA5?$AA0?$AA1?$AAU?$AAS?$AAB?$AA?3?$AA?5?$AAW?$AAa?$AAr?$AAn?$AAi?$AAn?$AAg?$AA?0?$AA?5@ 1000b940     wince.obj
 0001:0000a9b8       ??_C@_1DI@EMPOLEJH@?$AAR?$AAT?$AA2?$AA5?$AA0?$AA1?$AAU?$AAS?$AAB?$AA?5?$AAR?$AAe?$AAg?$AAi?$AAs?$AAt?$AAe?$AAr?$AAA?$AAd@ 1000b9b8     wince.obj
 0001:0000a9f0       ??_C@_1IG@FFCFEGNK@?$AAR?$AAT?$AA2?$AA5?$AA0?$AA1?$AAU?$AAS?$AAB?$AA?3?$AA?5?$AAP?$AAa?$AAr?$AAs?$AAe?$AAU?$AAs?$AAb?$AAD@ 1000b9f0     wince.obj
 0001:0000aa78       ??_C@_1EG@GBCKFIFN@?$AAR?$AAT?$AA2?$AA5?$AA0?$AA1?$AAU?$AAS?$AAB?$AA?3?$AA?5?$AAo?$AAu?$AAr?$AA?5?$AAD?$AAe?$AAv?$AAi?$AAc@ 1000ba78     wince.obj
 0001:0000aac0       ??_C@_0CP@JNKLFFBE@RT2501USB?5?$DN?$DN?$DN?$DN?$DN?$DN?$DO?5USBDeviceAttac@ 1000bac0     wince.obj
 0001:0000aaf0       ??_C@_1CK@KOMMGCAN@?$AAC?$AAo?$AAm?$AAm?$AAa?$AAn?$AAd?$AAS?$AAt?$AAa?$AAt?$AAu?$AAs?$AAT?$AAi?$AAm?$AAe?$AAo?$AAu?$AAt@ 1000baf0     wince.obj
 0001:0000ab1c       ??_C@_1CI@IEJJCHBF@?$AAC?$AAo?$AAm?$AAm?$AAa?$AAn?$AAd?$AAB?$AAl?$AAo?$AAc?$AAk?$AAT?$AAi?$AAm?$AAe?$AAo?$AAu?$AAt?$AA?$AA@ 1000bb1c     wince.obj
 0001:0000ab44       ??_C@_1BK@GEBLDPB@?$AAR?$AAe?$AAs?$AAe?$AAt?$AAT?$AAi?$AAm?$AAe?$AAo?$AAu?$AAt?$AA?$AA@ 1000bb44     wince.obj
 0001:0000ab60       ??_C@_1EI@MDFHKBKD@?$AAD?$AAr?$AAi?$AAv?$AAe?$AAr?$AAs?$AA?2?$AAU?$AAS?$AAB?$AA?2?$AAC?$AAl?$AAi?$AAe?$AAn?$AAt?$AAD?$AAr@ 1000bb60     wince.obj
 0001:0000aba8       ??_C@_1EC@FNIBLCAL@?$AAR?$AAT?$AA2?$AA5?$AA0?$AA1?$AAU?$AAS?$AAB?$AA?3?$AA?5?$AA?$DM?$AA?$DN?$AA?$DN?$AAU?$AAS?$AAB?$AAI?$AAn?$AAs@ 1000bba8     wince.obj
 0001:0000abf0       ??_C@_1EC@HIBALCDH@?$AAR?$AAe?$AAg?$AAi?$AAs?$AAt?$AAe?$AAr?$AAC?$AAl?$AAi?$AAe?$AAn?$AAt?$AAS?$AAe?$AAt?$AAt?$AAi?$AAn@ 1000bbf0     wince.obj
 0001:0000ac38       ??_C@_1EC@LOMFNKAL@?$AAR?$AAe?$AAg?$AAi?$AAs?$AAt?$AAe?$AAr?$AAC?$AAl?$AAi?$AAe?$AAn?$AAt?$AAD?$AAr?$AAi?$AAv?$AAe?$AAr@ 1000bc38     wince.obj
 0001:0000ac80       ??_C@_1EC@FNBFDKOB@?$AAR?$AAT?$AA2?$AA5?$AA0?$AA1?$AAU?$AAS?$AAB?$AA?3?$AA?5?$AA?$DN?$AA?$DN?$AA?$DO?$AAU?$AAS?$AAB?$AAI?$AAn?$AAs@ 1000bc80     wince.obj
 0001:0000acc4       ??_C@_17DJMMGLBL@?$AAD?$AAl?$AAl?$AA?$AA@ 1000bcc4     wince.obj
 0001:0000acd0       ??_C@_1EM@DNHLPGAH@?$AAR?$AAT?$AA2?$AA5?$AA0?$AA1?$AAU?$AAS?$AAB?$AA?3?$AA?5?$AA?$DM?$AA?$DN?$AA?$DN?$AAU?$AAS?$AAB?$AAU?$AAn?$AAI@ 1000bcd0     wince.obj
 0001:0000ad20       ??_C@_1EG@CIIKAKLG@?$AAR?$AAT?$AA2?$AA5?$AA0?$AA1?$AAU?$AAS?$AAB?$AA?3?$AA?5?$AA?$DN?$AA?$DN?$AA?$DO?$AAU?$AAS?$AAB?$AAU?$AAn?$AAI@ 1000bd20     wince.obj
 0001:0000ad68       ??_C@_1DK@GAADKJGK@?$AA?$DM?$AA?$DN?$AA?$DN?$AAP?$AAa?$AAr?$AAs?$AAe?$AAU?$AAs?$AAb?$AAD?$AAe?$AAs?$AAc?$AAr?$AAi?$AAp?$AAt?$AAo@ 1000bd68     wince.obj
 0001:0000ada8       ??_C@_1EE@PIAABIBG@?$AA?$CK?$AA?$CK?$AA?$CK?$AA?5?$AAF?$AAo?$AAu?$AAn?$AAd?$AA?5?$AAi?$AAn?$AAt?$AAe?$AAr?$AAf?$AAa?$AAc?$AAe?$AA?5@ 1000bda8     wince.obj
 0001:0000adec       ??_C@_1CE@JMILGGBB@?$AAi?$AAI?$AAn?$AAt?$AAe?$AAr?$AAf?$AAa?$AAc?$AAe?$AA?3?$AA?5?$AA0?$AAx?$AA?$CF?$AAx?$AA?6?$AA?$AA@ 1000bdec     wince.obj
 0001:0000ae10       ??_C@_1DE@FHKOHACH@?$AAb?$AAI?$AAn?$AAt?$AAe?$AAr?$AAf?$AAa?$AAc?$AAe?$AAP?$AAr?$AAo?$AAt?$AAo?$AAc?$AAo?$AAl?$AA?3?$AA?5@ 1000be10     wince.obj
 0001:0000ae44       ??_C@_1DE@EBHIKONI@?$AAb?$AAI?$AAn?$AAt?$AAe?$AAr?$AAf?$AAa?$AAc?$AAe?$AAS?$AAu?$AAb?$AAC?$AAl?$AAa?$AAs?$AAs?$AA?3?$AA?5@ 1000be44     wince.obj
 0001:0000ae78       ??_C@_1CO@GFLHDDIN@?$AAb?$AAI?$AAn?$AAt?$AAe?$AAr?$AAf?$AAa?$AAc?$AAe?$AAC?$AAl?$AAa?$AAs?$AAs?$AA?3?$AA?5?$AA0?$AAx?$AA?$CF@ 1000be78     wince.obj
 0001:0000aea8       ??_C@_1CK@NGJMHMFB@?$AAb?$AAN?$AAu?$AAm?$AAE?$AAn?$AAd?$AAp?$AAo?$AAi?$AAn?$AAt?$AAs?$AA?3?$AA?5?$AA0?$AAx?$AA?$CF?$AAx?$AA?6@ 1000bea8     wince.obj
 0001:0000aed4       ??_C@_1DC@DBGDLPA@?$AAb?$AAA?$AAl?$AAt?$AAe?$AAr?$AAn?$AAa?$AAt?$AAe?$AAS?$AAe?$AAt?$AAt?$AAi?$AAn?$AAg?$AA?3?$AA?5?$AA0@ 1000bed4     wince.obj
 0001:0000af08       ??_C@_1DA@GGMGJBI@?$AAb?$AAI?$AAn?$AAt?$AAe?$AAr?$AAf?$AAa?$AAc?$AAe?$AAN?$AAu?$AAm?$AAb?$AAe?$AAr?$AA?3?$AA?5?$AA0?$AAx@ 1000bf08     wince.obj
 0001:0000af38       ??_C@_1DG@OAIIGBKE@?$AA?9?$AA?9?$AA?9?$AA?9?$AA?9?$AA?9?$AA?9?$AA?9?$AA?9?$AA?9?$AA?9?$AA?9?$AA?9?$AA?9?$AA?9?$AA?9?$AA?9?$AA?9?$AA?9?$AA?9@ 1000bf38     wince.obj
 0001:0000af70       ??_C@_1DO@KMENEDNE@?$AAU?$AAS?$AAB?$AA_?$AAI?$AAN?$AAT?$AAE?$AAR?$AAF?$AAA?$AAC?$AAE?$AA_?$AAD?$AAE?$AAS?$AAC?$AAR?$AAI@ 1000bf70     wince.obj
 0001:0000afb0       ??_C@_1CA@GDJPGJNE@?$AAC?$AAo?$AAn?$AAf?$AAi?$AAg?$AAI?$AAn?$AAd?$AAe?$AAx?$AA?3?$AA?$CF?$AAd?$AA?6?$AA?$AA@ 1000bfb0     wince.obj
 0001:0000afd0       ??_C@_1CA@GLOFNEKL@?$AAM?$AAa?$AAx?$AAP?$AAo?$AAw?$AAe?$AAr?$AA?3?$AA?5?$AA0?$AAx?$AA?$CF?$AAx?$AA?6?$AA?$AA@ 1000bfd0     wince.obj
 0001:0000aff0       ??_C@_1CI@GGILJLCD@?$AAb?$AAm?$AAA?$AAt?$AAt?$AAr?$AAi?$AAb?$AAu?$AAt?$AAe?$AAs?$AA?3?$AA?5?$AA0?$AAx?$AA?$CF?$AAx?$AA?6?$AA?$AA@ 1000bff0     wince.obj
 0001:0000b018       ??_C@_1CM@KBBCNADB@?$AAi?$AAC?$AAo?$AAn?$AAf?$AAi?$AAg?$AAu?$AAr?$AAa?$AAt?$AAi?$AAo?$AAn?$AA?3?$AA?5?$AA0?$AAx?$AA?$CF?$AAx@ 1000c018     wince.obj
 0001:0000b044       ??_C@_1DG@CEBLCJLI@?$AAb?$AAC?$AAo?$AAn?$AAf?$AAi?$AAg?$AAu?$AAr?$AAa?$AAt?$AAi?$AAo?$AAn?$AAV?$AAa?$AAl?$AAu?$AAe?$AA?3@ 1000c044     wince.obj
 0001:0000b07c       ??_C@_1CM@GOEKMKAL@?$AAb?$AAN?$AAu?$AAm?$AAI?$AAn?$AAt?$AAe?$AAr?$AAf?$AAa?$AAc?$AAe?$AAs?$AA?3?$AA?5?$AA0?$AAx?$AA?$CF?$AAx@ 1000c07c     wince.obj
 0001:0000b0a8       ??_C@_1CI@PEJIKDOG@?$AAw?$AAT?$AAo?$AAt?$AAa?$AAl?$AAL?$AAe?$AAn?$AAg?$AAt?$AAh?$AA?3?$AA?5?$AA0?$AAx?$AA?$CF?$AAx?$AA?6?$AA?$AA@ 1000c0a8     wince.obj
 0001:0000b0d0       ??_C@_1DO@LJAHMEFB@?$AA?9?$AA?9?$AA?9?$AA?9?$AA?9?$AA?9?$AA?9?$AA?9?$AA?9?$AA?9?$AA?9?$AA?9?$AA?9?$AA?9?$AA?9?$AA?9?$AA?9?$AA?9?$AA?9?$AA?9@ 1000c0d0     wince.obj
 0001:0000b110       ??_C@_1DO@PJJBMGJF@?$AAU?$AAS?$AAB?$AA_?$AAC?$AAO?$AAN?$AAF?$AAI?$AAG?$AAU?$AAR?$AAA?$AAT?$AAI?$AAO?$AAN?$AA_?$AAD?$AAE@ 1000c110     wince.obj
 0001:0000b150       ??_C@_13LBAGMAIH@?$AA?6?$AA?$AA@ 1000c150     wince.obj
 0001:0000b154       ??_C@_1DE@NDPKMAKH@?$AAb?$AAN?$AAu?$AAm?$AAC?$AAo?$AAn?$AAf?$AAi?$AAg?$AAu?$AAr?$AAa?$AAt?$AAi?$AAo?$AAn?$AAs?$AA?3?$AA?5@ 1000c154     wince.obj
 0001:0000b188       ??_C@_1CK@CKKPHHF@?$AAi?$AAS?$AAe?$AAr?$AAi?$AAa?$AAl?$AAN?$AAu?$AAm?$AAb?$AAe?$AAr?$AA?3?$AA?5?$AA0?$AAx?$AA?$CF?$AAx?$AA?6@ 1000c188     wince.obj
 0001:0000b1b4       ??_C@_1CA@FDMGGJK@?$AAi?$AAP?$AAr?$AAo?$AAd?$AAu?$AAc?$AAt?$AA?3?$AA?5?$AA0?$AAx?$AA?$CF?$AAx?$AA?6?$AA?$AA@ 1000c1b4     wince.obj
 0001:0000b1d4       ??_C@_1CK@PBGEDOII@?$AAi?$AAM?$AAa?$AAn?$AAu?$AAf?$AAa?$AAc?$AAt?$AAu?$AAr?$AAe?$AAr?$AA?3?$AA?5?$AA0?$AAx?$AA?$CF?$AAx?$AA?6@ 1000c1d4     wince.obj
 0001:0000b200       ??_C@_1CC@DBBKOFLL@?$AAb?$AAc?$AAd?$AAD?$AAe?$AAv?$AAi?$AAc?$AAe?$AA?3?$AA?5?$AA0?$AAx?$AA?$CF?$AAx?$AA?6?$AA?$AA@ 1000c200     wince.obj
 0001:0000b224       ??_C@_1CI@KHDNBKNK@?$AAi?$AAd?$AAP?$AAr?$AAo?$AAd?$AAu?$AAc?$AAt?$AA?3?$AA?5?$AA?$CF?$AAd?$AA?$DN?$AA0?$AAx?$AA?$CF?$AAx?$AA?6?$AA?$AA@ 1000c224     wince.obj
 0001:0000b24c       ??_C@_1CG@GCAMPMJL@?$AAi?$AAd?$AAV?$AAe?$AAn?$AAd?$AAo?$AAr?$AA?3?$AA?5?$AA?$CF?$AAd?$AA?$DN?$AA0?$AAx?$AA?$CF?$AAx?$AA?6?$AA?$AA@ 1000c24c     wince.obj
 0001:0000b274       ??_C@_1CO@EIKOAMMG@?$AAb?$AAM?$AAa?$AAx?$AAP?$AAa?$AAc?$AAk?$AAe?$AAt?$AAS?$AAi?$AAz?$AAe?$AA0?$AA?3?$AA?5?$AA0?$AAx?$AA?$CF@ 1000c274     wince.obj
 0001:0000b2a4       ??_C@_1CO@NIGOBFMD@?$AAb?$AAD?$AAe?$AAv?$AAi?$AAc?$AAe?$AAP?$AAr?$AAo?$AAt?$AAo?$AAc?$AAo?$AAl?$AA?3?$AA?5?$AA0?$AAx?$AA?$CF@ 1000c2a4     wince.obj
 0001:0000b2d4       ??_C@_1CO@MOLIMLDM@?$AAb?$AAD?$AAe?$AAv?$AAi?$AAc?$AAe?$AAS?$AAu?$AAb?$AAC?$AAl?$AAa?$AAs?$AAs?$AA?3?$AA?5?$AA0?$AAx?$AA?$CF@ 1000c2d4     wince.obj
 0001:0000b304       ??_C@_1CI@HPCIHJJG@?$AAb?$AAD?$AAe?$AAv?$AAi?$AAc?$AAe?$AAC?$AAl?$AAa?$AAs?$AAs?$AA?3?$AA?5?$AA0?$AAx?$AA?$CF?$AAx?$AA?6?$AA?$AA@ 1000c304     wince.obj
 0001:0000b32c       ??_C@_1BM@MCKMICOP@?$AAb?$AAc?$AAd?$AAU?$AAS?$AAB?$AA?3?$AA?5?$AA0?$AAx?$AA?$CF?$AAx?$AA?6?$AA?$AA@ 1000c32c     wince.obj
 0001:0000b348       ??_C@_1CO@BEMPIGAC@?$AAb?$AAD?$AAe?$AAs?$AAc?$AAr?$AAi?$AAp?$AAt?$AAo?$AAr?$AAT?$AAy?$AAp?$AAe?$AA?3?$AA?5?$AA0?$AAx?$AA?$CF@ 1000c348     wince.obj
 0001:0000b378       ??_C@_1BO@HCAHHBMN@?$AAb?$AAL?$AAe?$AAn?$AAg?$AAt?$AAh?$AA?3?$AA?5?$AA0?$AAx?$AA?$CF?$AAx?$AA?6?$AA?$AA@ 1000c378     wince.obj
 0001:0000b398       ??_C@_1DA@PPGHFICI@?$AA?9?$AA?9?$AA?9?$AA?9?$AA?9?$AA?9?$AA?9?$AA?9?$AA?9?$AA?9?$AA?9?$AA?9?$AA?9?$AA?9?$AA?9?$AA?9?$AA?9?$AA?9?$AA?9?$AA?9@ 1000c398     wince.obj
 0001:0000b3c8       ??_C@_1DA@BHAPFKON@?$AAU?$AAS?$AAB?$AA_?$AAD?$AAE?$AAV?$AAI?$AAC?$AAE?$AA_?$AAD?$AAE?$AAS?$AAC?$AAR?$AAI?$AAP?$AAT?$AAO@ 1000c3c8     wince.obj
 0001:0000b3f8       ??_C@_1DC@GNDMFOKL@?$AAG?$AAe?$AAt?$AAD?$AAe?$AAv?$AAi?$AAc?$AAe?$AAI?$AAn?$AAf?$AAo?$AA?5?$AAe?$AAr?$AAr?$AAo?$AAr?$AA?3@ 1000c3f8     wince.obj
 0001:0000b42c       ??_C@_1CK@NIDHICOA@?$AAI?$AAn?$AAv?$AAa?$AAl?$AAi?$AAd?$AA?5?$AAp?$AAa?$AAr?$AAa?$AAm?$AAe?$AAt?$AAe?$AAr?$AA?3?$AA?$AN?$AA?6@ 1000c42c     wince.obj
 0001:0000b458       ??_C@_1EA@LBCNPIEL@?$AAI?$AAn?$AAv?$AAa?$AAl?$AAi?$AAd?$AA?5?$AAp?$AAa?$AAr?$AAa?$AAm?$AAe?$AAt?$AAe?$AAr?$AA?3?$AAC?$AAo@ 1000c458     wince.obj
 0001:0000b498       ??_C@_1EC@BLMAJBLK@?$AAI?$AAn?$AAv?$AAa?$AAl?$AAi?$AAd?$AA?5?$AAp?$AAa?$AAr?$AAa?$AAm?$AAe?$AAt?$AAe?$AAr?$AA?3?$AAC?$AAu@ 1000c498     wince.obj
 0001:0000b4dc       ??_C@_1DK@KILCHDCF@?$AAI?$AAn?$AAv?$AAa?$AAl?$AAi?$AAd?$AA?5?$AAp?$AAa?$AAr?$AAa?$AAm?$AAe?$AAt?$AAe?$AAr?$AA?3?$AAU?$AAs@ 1000c4dc     wince.obj
 0001:0000b518       ??_C@_1DO@BDDPKKG@?$AAI?$AAn?$AAv?$AAa?$AAl?$AAi?$AAd?$AA?5?$AAp?$AAa?$AAr?$AAa?$AAm?$AAe?$AAt?$AAe?$AAr?$AA?3?$AAh?$AAU@ 1000c518     wince.obj
 0001:0000b558       ??_C@_0CA@CBBFBJML@?9?9?9?$DOUSBMSC?$DOParseUsbDescriptors?6?$AA@ 1000c558     wince.obj
 0001:0000b578       ??_C@_1DK@IDLOABHP@?$AA?$CK?$AA?$CK?$AA?$CK?$AA?5?$AAR?$AAe?$AAs?$AAe?$AAt?$AAE?$AAv?$AAe?$AAn?$AAt?$AA?5?$AAE?$AAR?$AAR?$AAO?$AAR@ 1000c578     wince.obj
 0001:0000b5b4       ??_C@_03OFAPEBGM@?$CFs?6?$AA@ 1000c5b4     wince.obj
 0001:0000b5b8       ??_C@_07BNCCFNNE@?$CF4?44x?5?5?$AA@ 1000c5b8     wince.obj
 0001:0000b5c0       ??_C@_0BB@JCEFLFJE@0123456789abcdef?$AA@ 1000c5c0     wince.obj
 0001:0000b5d8       ??_C@_1EA@DLNKEDK@?$AA?$CK?$AA?$CK?$AA?$CK?$AA?5?$AAA?$AAb?$AAo?$AAr?$AAt?$AAT?$AAr?$AAa?$AAn?$AAs?$AAf?$AAe?$AAr?$AA?5?$AAE?$AAR@ 1000c5d8     usbclient:usbclient.obj
 0001:0000b618       ??_C@_1EA@OEBLAPPP@?$AA?$CK?$AA?$CK?$AA?$CK?$AA?5?$AAC?$AAl?$AAo?$AAs?$AAe?$AAT?$AAr?$AAa?$AAn?$AAs?$AAf?$AAe?$AAr?$AA?5?$AAE?$AAR@ 1000c618     usbclient:usbclient.obj
 0001:0000b658       ??_C@_1GK@NFJEKGG@?$AA?$CK?$AA?$CK?$AA?$CK?$AA?5?$AAC?$AAl?$AAe?$AAa?$AAr?$AAO?$AAr?$AAS?$AAe?$AAt?$AAF?$AAe?$AAa?$AAt?$AAu?$AAr@ 1000c658     usbclient:usbclient.obj
 0001:0000b6c8       ??_C@_1EC@JIGPENPP@?$AA?$CK?$AA?$CK?$AA?$CK?$AA?5?$AAU?$AAn?$AAh?$AAa?$AAn?$AAd?$AAl?$AAe?$AAd?$AA?5?$AAW?$AAa?$AAi?$AAt?$AAR?$AAe@ 1000c6c8     usbclient:usbclient.obj
 0001:0000b710       ??_C@_1FO@EGDNIMLN@?$AAC?$AAl?$AAe?$AAa?$AAr?$AAO?$AAr?$AAS?$AAe?$AAt?$AAF?$AAe?$AAa?$AAt?$AAu?$AAr?$AAe?$AA?3?$AAW?$AAA@ 1000c710     usbclient:usbclient.obj
 0001:0000b770       ??_C@_1FE@GJFHKKL@?$AA?$CK?$AA?$CK?$AA?$CK?$AA?5?$AAD?$AAe?$AAf?$AAa?$AAu?$AAl?$AAt?$AAT?$AAr?$AAa?$AAn?$AAs?$AAf?$AAe?$AAr?$AAC@ 1000c770     usbclient:usbclient.obj
 0001:0000b7c4       ??_C@_1DG@KGMCLKFK@?$AA?$CK?$AA?$CK?$AA?$CK?$AA?5?$AAS?$AAe?$AAt?$AAE?$AAv?$AAe?$AAn?$AAt?$AA?5?$AAE?$AAR?$AAR?$AAO?$AAR?$AA?3?$AA?$CF@ 1000c7c4     usbclient:usbclient.obj
 0001:0000b800       ??_C@_1HC@OIDPFNDL@?$AA?$CK?$AA?$CK?$AA?$CK?$AA?5?$AAG?$AAe?$AAt?$AAS?$AAt?$AAa?$AAt?$AAu?$AAs?$AA?5?$AAo?$AAn?$AA?5?$AAe?$AAn?$AAd@ 1000c800     usbclient:usbclient.obj
 0001:0000b878       ??_C@_1EO@LLIJNJID@?$AAG?$AAe?$AAt?$AAS?$AAt?$AAa?$AAt?$AAu?$AAs?$AA?3?$AAW?$AAA?$AAI?$AAT?$AA_?$AAT?$AAI?$AAM?$AAE?$AAO@ 1000c878     usbclient:usbclient.obj
 0001:0000b8c8       ??_C@_1EI@EFFJOCFO@?$AA?$CK?$AA?$CK?$AA?$CK?$AA?5?$AAG?$AAe?$AAt?$AAT?$AAr?$AAa?$AAn?$AAs?$AAf?$AAe?$AAr?$AAS?$AAt?$AAa?$AAt?$AAu@ 1000c8c8     usbclient:usbclient.obj
 0001:0000b910       ??_C@_1HA@BBDFJFG@?$AAG?$AAe?$AAt?$AAT?$AAr?$AAa?$AAn?$AAs?$AAf?$AAe?$AAr?$AAS?$AAt?$AAa?$AAt?$AAu?$AAs?$AA?5?$AA?$CI?$AAB@ 1000c910     usbclient:usbclient.obj
 0001:0000b980       ??_C@_1JK@HKJHGPDC@?$AAI?$AAs?$AAs?$AAu?$AAe?$AAB?$AAu?$AAl?$AAk?$AAT?$AAr?$AAa?$AAn?$AAs?$AAf?$AAe?$AAr?$AA?5?$AAE?$AAR@ 1000c980     usbclient:usbclient.obj
 0001:0000ba20       ??_C@_1FA@COJHPOOL@?$AA?$CK?$AA?$CK?$AA?$CK?$AA?5?$AAI?$AAs?$AAs?$AAu?$AAe?$AAB?$AAu?$AAl?$AAk?$AAT?$AAr?$AAa?$AAn?$AAs?$AAf?$AAe@ 1000ca20     usbclient:usbclient.obj
 0001:0000ba70       ??_C@_1DI@EENFKOKJ@?$AA?$CF?$AAs?$AA?3?$AAW?$AAA?$AAI?$AAT?$AA_?$AAT?$AAI?$AAM?$AAE?$AAO?$AAU?$AAT?$AA?5?$AAo?$AAn?$AA?5?$AAh@ 1000ca70     usbclient:usbclient.obj
 0001:0000baa8       ??_C@_17HCEMPBGG@?$AAO?$AAU?$AAT?$AA?$AA@ 1000caa8     usbclient:usbclient.obj
 0001:0000bab0       ??_C@_15BNKBCKPG@?$AAI?$AAN?$AA?$AA@ 1000cab0     usbclient:usbclient.obj
 0001:0000bab8       ??_C@_1KE@HEHDFMIE@?$AAI?$AAs?$AAs?$AAu?$AAe?$AAI?$AAn?$AAt?$AAe?$AAr?$AAr?$AAu?$AAp?$AAt?$AAT?$AAr?$AAa?$AAn?$AAs?$AAf@ 1000cab8     usbclient:usbclient.obj
 0001:0000bb60       ??_C@_1FK@KGMBLFKM@?$AA?$CK?$AA?$CK?$AA?$CK?$AA?5?$AAI?$AAs?$AAs?$AAu?$AAe?$AAI?$AAn?$AAt?$AAe?$AAr?$AAr?$AAu?$AAp?$AAt?$AAT?$AAr@ 1000cb60     usbclient:usbclient.obj
 0001:0000bbc0       ??_C@_1JO@FNJJOIFN@?$AAI?$AAs?$AAs?$AAu?$AAe?$AAV?$AAe?$AAn?$AAd?$AAo?$AAr?$AAT?$AAr?$AAa?$AAn?$AAs?$AAf?$AAe?$AAr?$AA?5@ 1000cbc0     usbclient:usbclient.obj
 0001:0000bc60       ??_C@_1FI@ILPCPOCG@?$AA?$CK?$AA?$CK?$AA?$CK?$AA?5?$AAI?$AAs?$AAs?$AAu?$AAe?$AAV?$AAe?$AAn?$AAd?$AAo?$AAr?$AAT?$AAr?$AAa?$AAn?$AAs@ 1000cc60     usbclient:usbclient.obj
 0001:0000bcb8       ??_C@_1EM@GADAJNPB@?$AA?$CK?$AA?$CK?$AA?$CK?$AA?5?$AAI?$AAs?$AAD?$AAe?$AAf?$AAa?$AAu?$AAl?$AAt?$AAP?$AAi?$AAp?$AAe?$AAH?$AAa?$AAl@ 1000ccb8     usbclient:usbclient.obj
 0001:0000bd08       ??_C@_1EE@FGLFADDK@?$AA?$CK?$AA?$CK?$AA?$CK?$AA?5?$AAR?$AAe?$AAs?$AAe?$AAt?$AAD?$AAe?$AAf?$AAa?$AAu?$AAl?$AAt?$AAP?$AAi?$AAp?$AAe@ 1000cd08     usbclient:usbclient.obj
 0001:0000bd4c       ??_C@_1DG@LIHBBAAA@?$AAE?$AAn?$AAp?$AAo?$AAi?$AAn?$AAt?$AA?3?$AA0?$AAx?$AA?$CF?$AAx?$AA?5?$AAw?$AAS?$AAt?$AAa?$AAt?$AAu?$AAs@ 1000cd4c     usbclient:usbclient.obj
 0001:0000bd84       ??_C@_1DI@MOPNAAFE@?$AA?$CK?$AA?$CK?$AA?$CK?$AA?5?$AAR?$AAe?$AAs?$AAe?$AAt?$AAP?$AAi?$AAp?$AAe?$AA?5?$AAE?$AAR?$AAR?$AAO?$AAR?$AA?3@ 1000cd84     usbclient:usbclient.obj
 0001:0000be30       _MlmeInit                  1000ce30 f   mlme.obj
 0001:0000c040       _MlmeHandler               1000d040 f   mlme.obj
 0001:0000c400       _MlmeHalt                  1000d400 f   mlme.obj
 0001:0000c520       _MlmeSuspend               1000d520 f   mlme.obj
 0001:0000c7d0       _MlmeResume                1000d7d0 f   mlme.obj
 0001:0000c8c0       _MlmePeriodicExec          1000d8c0 f   mlme.obj
 0001:0000cac0       _STAMlmePeriodicExec       1000dac0 f   mlme.obj
 0001:0000d7c0       _LinkDownExec              1000e7c0 f   mlme.obj
 0001:0000d810       _MlmeAutoScan              1000e810 f   mlme.obj
 0001:0000d860       _MlmeAutoReconnectLastSSID 1000e860 f   mlme.obj
 0001:0000d920       _MlmeValidateSSID          1000e920 f   mlme.obj
 0001:0000d970       _MlmeValidateSetSSID       1000e970 f   mlme.obj
 0001:0000d9d0       _MlmeIsVisibleSSID         1000e9d0 f   mlme.obj
 0001:0000da30       _MlmeCheckForRoaming       1000ea30 f   mlme.obj
 0001:0000dbe0       _MlmeCheckForFastRoaming   1000ebe0 f   mlme.obj
 0001:0000de40       _MlmeCalculateChannelQuality 1000ee40 f   mlme.obj
 0001:0000e030       _MlmeDynamicTxRateSwitching 1000f030 f   mlme.obj
 0001:0000e9c0       _MlmeCheckPsmChange        1000f9c0 f   mlme.obj
 0001:0000ea60       _MlmeSetPsmBit             1000fa60 f   mlme.obj
 0001:0000eae0       _MlmeSetTxPreamble         1000fae0 f   mlme.obj
 0001:0000eb90       _MlmeUpdateTxRates         1000fb90 f   mlme.obj
 0001:0000f680       _MlmeRadioOff              10010680 f   mlme.obj
 0001:0000f910       _MlmeRadioOn               10010910 f   mlme.obj
 0001:0000fa10       _BssTableInit              10010a10 f   mlme.obj
 0001:0000fa60       _BssTableSearch            10010a60 f   mlme.obj
 0001:0000fb00       _BssSsidTableSearch        10010b00 f   mlme.obj
 0001:0000fbe0       _BssTableSearchWithSSID    10010be0 f   mlme.obj
 0001:0000fd20       _BssTableDeleteEntry       10010d20 f   mlme.obj
 0001:0000fe00       _BssEntrySet               10010e00 f   mlme.obj
 0001:00010060       _BssTableSetEntry          10011060 f   mlme.obj
 0001:000101c0       _BssTableSsidSort          100111c0 f   mlme.obj
 0001:00010630       _BssTableSortByRssi        10011630 f   mlme.obj
 0001:00010740       _BssCipherParse            10011740 f   mlme.obj
 0001:00010e60       _MacAddrRandomBssid        10011e60 f   mlme.obj
 0001:00010eb0       _MgtMacHeaderInit          10011eb0 f   mlme.obj
 0001:00010f70       _MakeOutgoingFrame         10011f70 f   mlme.obj
 0001:00010ff0       _MlmeQueueInit             10011ff0 f   mlme.obj
 0001:000110c0       _MlmeEnqueue               100120c0 f   mlme.obj
 0001:00011260       _MlmeEnqueueForRecv        10012260 f   mlme.obj
 0001:000114b0       _MlmeDequeue               100124b0 f   mlme.obj
 0001:00011560       _MlmeRestartStateMachine   10012560 f   mlme.obj
 0001:00011710       _MlmePostRestartStateMachine 10012710 f   mlme.obj
 0001:00011750       _MlmeQueueEmpty            10012750 f   mlme.obj
 0001:000117a0       _MlmeQueueFull             100127a0 f   mlme.obj
 0001:000117f0       _MlmeQueueDestroy          100127f0 f   mlme.obj
 0001:00011860       _MsgTypeSubst              10012860 f   mlme.obj
 0001:00011ad0       _StateMachineInit          10012ad0 f   mlme.obj
 0001:00011b60       _StateMachineSetAction     10012b60 f   mlme.obj
 0001:00011bb0       _StateMachinePerformAction 10012bb0 f   mlme.obj
 0001:00011bf0       _Drop                      10012bf0 f   mlme.obj
 0001:00011c00       _LfsrInit                  10012c00 f   mlme.obj
 0001:00011c30       _RandomByte                10012c30 f   mlme.obj
 0001:00011cc0       _AsicSwitchChannel         10012cc0 f   mlme.obj
 0001:000123b0       _AsicLockChannel           100133b0 f   mlme.obj
 0001:000123c0       _AsicAntennaSelect         100133c0 f   mlme.obj
 0001:000126e0       _AsicAntennaSetting        100136e0 f   mlme.obj
 0001:00012ed0       _AsicAdjustTxPower         10013ed0 f   mlme.obj
 0001:00013540       _AsicSleepThenAutoWakeup   10014540 f   mlme.obj
 0001:00013650       _AsicForceSleep            10014650 f   mlme.obj
 0001:000136d0       _AsicForceWakeup           100146d0 f   mlme.obj
 0001:00013750       _AsicSetBssid              10014750 f   mlme.obj
 0001:000137f0       _AsicDisableSync           100147f0 f   mlme.obj
 0001:00013850       _AsicEnableBssSync         10014850 f   mlme.obj
 0001:00013960       _AsicEnableIbssSync        10014960 f   mlme.obj
 0001:00013b60       _AsicSetEdcaParm           10014b60 f   mlme.obj
 0001:00014020       _AsicSetSlotTime           10015020 f   mlme.obj
 0001:00014150       _AsicBbpTuning             10015150 f   mlme.obj
 0001:000147d0       _AsicAddSharedKeyEntry     100157d0 f   mlme.obj
 0001:00014b50       _AsicRemoveSharedKeyEntry  10015b50 f   mlme.obj
 0001:00014c30       _AsicAddPairwiseKeyEntry   10015c30 f   mlme.obj
 0001:00014e20       _AsicRemovePairwiseKeyEntry 10015e20 f   mlme.obj
 0001:00014ed0       _RTMPCheckRates            10015ed0 f   mlme.obj
 0001:00014f90       _AsicSetRxAnt              10015f90 f   mlme.obj
 0001:000152b0       _AsicEvaluateSecondaryRxAnt 100162b0 f   mlme.obj
 0001:00015380       _AsicRxAntEvalTimeout      10016380 f   mlme.obj
 0001:000153b0       _AsicRxAntEvalAction       100163b0 f   mlme.obj
 0001:00015500       _StaQuickResponeForRateUpExec 10016500 f   mlme.obj
 0001:000157b0       _RadarDetectionStart       100167b0 f   mlme.obj
 0001:00015950       _RadarDetectionStop        10016950 f   mlme.obj
 0001:00015a10       _RadarChannelCheck         10016a10 f   mlme.obj
 0001:00015a90       _MlmeThread                10016a90 f   mlme.obj
 0001:00015ab0       _MlmeFreeMemory            10016ab0 f   mlme.obj
 0001:00015f00       _MlmeAllocateMemory        10016f00 f   mlme.obj
 0001:00016180       _MlmeInitMemoryHandler     10017180 f   mlme.obj
 0001:000163c0       _MlmeFreeMemoryHandler     100173c0 f   mlme.obj
 0001:00016490       _AironetStateMachineInit   10017490 f   aironet.obj
 0001:00016500       _AironetMsgAction          10017500 f   aironet.obj
 0001:00016940       _AironetRequestAction      10017940 f   aironet.obj
 0001:00016a90       _ChannelLoadRequestAction  10017a90 f   aironet.obj
 0001:00016cd0       _NoiseHistRequestAction    10017cd0 f   aironet.obj
 0001:00016f30       _BeaconRequestAction       10017f30 f   aironet.obj
 0001:00017390       _AironetReportAction       10018390 f   aironet.obj
 0001:000175a0       _AironetFinalReportAction  100185a0 f   aironet.obj
 0001:000177c0       _ChannelLoadReportAction   100187c0 f   aironet.obj
 0001:000179c0       _NoiseHistReportAction     100189c0 f   aironet.obj
 0001:00017cb0       _BeaconReportAction        10018cb0 f   aironet.obj
 0001:00017d00       _AironetAddBeaconReport    10018d00 f   aironet.obj
 0001:00018390       _AironetCreateBeaconReportFromBssTable 10019390 f   aironet.obj
 0001:000186d0       _Sniff2BytesFromNdisBuffer 100196d0 f   rtusb_data.obj
 0001:00018790       _RTMPSendPackets           10019790 f   rtusb_data.obj
 0001:00018960       _RTMPSendPacket            10019960 f   rtusb_data.obj
 0001:00018d60       _RTMPDeQueuePacket         10019d60 f   rtusb_data.obj
 0001:000190f0       _RTUSBFreeDescriptorRequest 1001a0f0 f   rtusb_data.obj
 0001:00019240       _RTUSBRejectPendingPackets 1001a240 f   rtusb_data.obj
 0001:00019370       _RTUSBSuspendMsduTransmission 1001a370 f   rtusb_data.obj
 0001:000193d0       _RTUSBResumeMsduTransmission 1001a3d0 f   rtusb_data.obj
 0001:000194b0       _RTUSBCalcDuration         1001a4b0 f   rtusb_data.obj
 0001:00019590       _RTUSBWriteTxDescriptor    1001a590 f   rtusb_data.obj
 0001:00019b70       _TxFrameIsAggregatible     1001ab70 f   rtusb_data.obj
 0001:00019bc0       _RTUSBHardTransmit         1001abc0 f   rtusb_data.obj
 0001:0001b5d0       _RTUSBRxPacket             1001c5d0 f   rtusb_data.obj
 0001:0001cc70       _RTUSBDequeueMLMEPacket    1001dc70 f   rtusb_data.obj
 0001:0001ce00       _RTUSBCleanUpMLMEWaitQueue 1001de00 f   rtusb_data.obj
 0001:0001cef0       _MiniportMMRequest         1001def0 f   rtusb_data.obj
 0001:0001d080       _RTMPSearchTupleCache      1001e080 f   rtusb_data.obj
 0001:0001d140       _RTMPUpdateTupleCache      1001e140 f   rtusb_data.obj
 0001:0001d450       _RTMPApplyPacketFilter     1001e450 f   rtusb_data.obj
 0001:0001d6b0       _RTMPCheckRxDescriptor     1001e6b0 f   rtusb_data.obj
 0001:0001da40       _RTMPReportMicError        1001ea40 f   rtusb_data.obj
 0001:0001db60       _RTUSBMlmeHardTransmit     1001eb60 f   rtusb_data.obj
 0001:0001dea0       _RTMPSendNullFrame         1001eea0 f   rtusb_data.obj
 0001:0001e0b0       _RTMPSendRTSCTSFrame       1001f0b0 f   rtusb_data.obj
 0001:0001e450       _RTMPCalcDuration          1001f450 f   rtusb_data.obj
 0001:0001e530       _RTMPCheckDHCPFrame        1001f530 f   rtusb_data.obj
 0001:0001e680       _InterlockedDecrement      1001f680 f i rtusb_data.obj
 0001:0001e6a0       _InterlockedIncrement      1001f6a0 f i rtusb_data.obj
 0001:0001e6c0       _RTMPAllocAdapterBlock     1001f6c0 f   rtmp_init.obj
 0001:0001e790       _NICInitTransmit           1001f790 f   rtmp_init.obj
 0001:0001ed10       _CreateThreads             1001fd10 f   rtmp_init.obj
 0001:0001ed30       _NICInitRecv               1001fd30 f   rtmp_init.obj
 0001:0001ee20       _RTMPInitAdapterBlock      1001fe20 f   rtmp_init.obj
 0001:0001f220       _ReleaseAdapter            10020220 f   rtmp_init.obj
 0001:0001f640       _RTMPFreeAdapter           10020640 f   rtmp_init.obj
 0001:0001f700       _NICReadRegParameters      10020700 f   rtmp_init.obj
 0001:00020030       _RTUSBWriteHWMACAddress    10021030 f   rtmp_init.obj
 0001:00020190       _NICReadEEPROMParameters   10021190 f   rtmp_init.obj
 0001:00020d30       _NICInitAsicFromEEPROM     10021d30 f   rtmp_init.obj
 0001:000210c0       _NICInitializeAsic         100220c0 f   rtmp_init.obj
 0001:000212d0       _NICIssueReset             100222d0 f   rtmp_init.obj
 0001:000212e0       _NICCheckForHang           100222e0 f   rtmp_init.obj
 0001:000212f0       _NICUpdateRawCounters      100222f0 f   rtmp_init.obj
 0001:00021620       _NICResetFromError         10022620 f   rtmp_init.obj
 0001:00021650       _NICLoadFirmware           10022650 f   rtmp_init.obj
 0001:00021a10       _RTMPEqualMemory           10022a10 f   rtmp_init.obj
 0001:00021a80       _RTMPCompareMemory         10022a80 f   rtmp_init.obj
 0001:00021b00       _RTMPZeroMemory            10022b00 f   rtmp_init.obj
 0001:00021b40       _RTMPFillMemory            10022b40 f   rtmp_init.obj
 0001:00021b80       _RTMPMoveMemory            10022b80 f   rtmp_init.obj
 0001:00021c10       _UserCfgInit               10022c10 f   rtmp_init.obj
 0001:000221c0       _BtoH                      100231c0 f   rtmp_init.obj
 0001:00022220       _AtoH                      10023220 f   rtmp_init.obj
 0001:000222b0       _RTMPPatchMacBbpBug        100232b0 f   rtmp_init.obj
 0001:000222c0       _RTMPInitTimer             100232c0 f   rtmp_init.obj
 0001:00022300       _RTMPSetTimer              10023300 f   rtmp_init.obj
 0001:00022390       _RTMPCancelTimer           10023390 f   rtmp_init.obj
 0001:000223f0       _RTMPSetLED                100233f0 f   rtmp_init.obj
 0001:00022600       _RTMPSetSignalLED          10023600 f   rtmp_init.obj
 0001:000226c0       _RTMPCckBbpTuning          100236c0 f   rtmp_init.obj
 0001:000227d0       _DriverEntry               100237d0 f   rtmp_main.obj
 0001:00022a30       _RTMPInitialize            10023a30 f   rtmp_main.obj
 0001:00022f60       _RTMPCheckForHang          10023f60 f   rtmp_main.obj
 0001:00022fd0       _RTMPHalt                  10023fd0 f   rtmp_main.obj
 0001:000232f0       _RTMPReset                 100242f0 f   rtmp_main.obj
 0001:00023330       _RTMPTransferData          10024330 f   rtmp_main.obj
 0001:000234e0       _RTMPPnPEventNotify        100244e0 f   rtmp_main.obj
 0001:00023700       _RTMPShutdown              10024700 f   rtmp_main.obj
 0001:00023740       _RTMPQueryInformation      10024740 f   rtmp_info.obj
 0001:000258b0       _RTMPSetInformation        100268b0 f   rtmp_info.obj
 0001:00026170       _STAQueryInformation       10027170 f   rtmp_info.obj
 0001:00027830       _STASetInformation         10028830 f   rtmp_info.obj
 0001:00029480       _RTMPWPAAddKeyProc         1002a480 f   rtmp_info.obj
 0001:000299d0       _RTMPWPARemoveKeyProc      1002a9d0 f   rtmp_info.obj
 0001:00029b80       _RTMPWPARemoveAllKeys      1002ab80 f   rtmp_info.obj
 0001:00029c40       _RTMPSetPhyMode            1002ac40 f   rtmp_info.obj
 0001:0002a070       _RTMPInitWepEngine         1002b070 f   rtmp_wep.obj
 0001:0002a160       _RTMPEncryptData           1002b160 f   rtmp_wep.obj
 0001:0002a1b0       _RTMPDecryptData           1002b1b0 f   rtmp_wep.obj
 0001:0002a3a0       _ARCFOUR_INIT              1002b3a0 f   rtmp_wep.obj
 0001:0002a480       _ARCFOUR_BYTE              1002b480 f   rtmp_wep.obj
 0001:0002a510       _ARCFOUR_DECRYPT           1002b510 f   rtmp_wep.obj
 0001:0002a560       _ARCFOUR_ENCRYPT           1002b560 f   rtmp_wep.obj
 0001:0002a5b0       _WPAARCFOUR_ENCRYPT        1002b5b0 f   rtmp_wep.obj
 0001:0002a630       _RTMP_CALC_FCS32           1002b630 f   rtmp_wep.obj
 0001:0002a680       _RTMPSetICV                1002b680 f   rtmp_wep.obj
 0001:0002a6c0       _RTMPTkipGetUInt32         1002b6c0 f   rtmp_tkip.obj
 0001:0002a710       _RTMPTkipPutUInt32         1002b710 f   rtmp_tkip.obj
 0001:0002a760       _RTMPTkipSetMICKey         1002b760 f   rtmp_tkip.obj
 0001:0002a7c0       _RTMPTkipAppendByte        1002b7c0 f   rtmp_tkip.obj
 0001:0002a900       _RTMPTkipAppend            1002b900 f   rtmp_tkip.obj
 0001:0002a940       _RTMPTkipGetMIC            1002b940 f   rtmp_tkip.obj
 0001:0002a9d0       _RTMPInitTkipEngine        1002b9d0 f   rtmp_tkip.obj
 0001:0002aa40       _RTMPInitMICEngine         1002ba40 f   rtmp_tkip.obj
 0001:0002aab0       _RTMPTkipCompareMICValue   1002bab0 f   rtmp_tkip.obj
 0001:0002ac70       _RTMPTkipCompareMICValueWithLLC 1002bc70 f   rtmp_tkip.obj
 0001:0002ae40       _RTMPCalculateMICValue     1002be40 f   rtmp_tkip.obj
 0001:0002af70       _tkip_sbox                 1002bf70 f   rtmp_tkip.obj
 0001:0002afe0       _rotr1                     1002bfe0 f   rtmp_tkip.obj
 0001:0002b020       _RTMPTkipMixKey            1002c020 f   rtmp_tkip.obj
 0001:0002b5d0       _construct_mic_header1     1002c5d0 f   rtmp_tkip.obj
 0001:0002b6c0       _construct_mic_header2     1002c6c0 f   rtmp_tkip.obj
 0001:0002b800       _construct_mic_iv          1002c800 f   rtmp_tkip.obj
 0001:0002b8f0       _bitwise_xor               1002c8f0 f   rtmp_tkip.obj
 0001:0002b930       _aes128k128d               1002c930 f   rtmp_tkip.obj
 0001:0002ba80       _construct_ctr_preload     1002ca80 f   rtmp_tkip.obj
 0001:0002bb80       _RTMPSoftDecryptTKIP       1002cb80 f   rtmp_tkip.obj
 0001:0002c080       _RTMPSoftDecryptAES        1002d080 f   rtmp_tkip.obj
 0001:0002c660       _AssocStateMachineInit     1002d660 f   assoc.obj
 0001:0002c8a0       _AssocTimeout              1002d8a0 f   assoc.obj
 0001:0002c910       _ReassocTimeout            1002d910 f   assoc.obj
 0001:0002c980       _DisassocTimeout           1002d980 f   assoc.obj
 0001:0002c9e0       _MlmeAssocReqAction        1002d9e0 f   assoc.obj
 0001:0002d4a0       _MlmeReassocReqAction      1002e4a0 f   assoc.obj
 0001:0002dc60       _MlmeDisassocReqAction     1002ec60 f   assoc.obj
 0001:0002dde0       _PeerAssocRspAction        1002ede0 f   assoc.obj
 0001:0002e020       _PeerReassocRspAction      1002f020 f   assoc.obj
 0001:0002e2a0       _AssocPostProc             1002f2a0 f   assoc.obj
 0001:0002e520       _PeerDisassocAction        1002f520 f   assoc.obj
 0001:0002e640       _AssocTimeoutAction        1002f640 f   assoc.obj
 0001:0002e690       _ReassocTimeoutAction      1002f690 f   assoc.obj
 0001:0002e6e0       _DisassocTimeoutAction     1002f6e0 f   assoc.obj
 0001:0002e730       _InvalidStateWhenAssoc     1002f730 f   assoc.obj
 0001:0002e790       _InvalidStateWhenReassoc   1002f790 f   assoc.obj
 0001:0002e7f0       _InvalidStateWhenDisassociate 1002f7f0 f   assoc.obj
 0001:0002e850       _Cls3errAction             1002f850 f   assoc.obj
 0001:0002e930       _SwitchBetweenWepAndCkip   1002f930 f   assoc.obj
 0001:0002ecb0       _AuthStateMachineInit      1002fcb0 f   auth.obj
 0001:0002ed90       _AuthTimeout               1002fd90 f   auth.obj
 0001:0002ee00       _MlmeAuthReqAction         1002fe00 f   auth.obj
 0001:0002f040       _PeerAuthRspAtSeq2Action   10030040 f   auth.obj
 0001:0002f400       _PeerAuthRspAtSeq4Action   10030400 f   auth.obj
 0001:0002f510       _MlmeDeauthReqAction       10030510 f   auth.obj
 0001:0002f660       _AuthTimeoutAction         10030660 f   auth.obj
 0001:0002f6b0       _InvalidStateWhenAuth      100306b0 f   auth.obj
 0001:0002f710       _Cls2errAction             10030710 f   auth.obj
 0001:0002f7f0       _AuthRspStateMachineInit   100307f0 f   auth_rsp.obj
 0001:0002f860       _PeerAuthSimpleRspGenAndSend 10030860 f   auth_rsp.obj
 0001:0002f930       _PeerDeauthAction          10030930 f   auth_rsp.obj
 0001:0002fa40       _SyncStateMachineInit      10030a40 f   sync.obj
 0001:0002fbf0       _BeaconTimeout             10030bf0 f   sync.obj
 0001:0002fc50       _ScanTimeout               10030c50 f   sync.obj
 0001:0002fcb0       _MlmeScanReqAction         10030cb0 f   sync.obj
 0001:0002ff60       _MlmeJoinReqAction         10030f60 f   sync.obj
 0001:000300e0       _MlmeStartReqAction        100310e0 f   sync.obj
 0001:00030430       _PeerBeaconAtScanAction    10031430 f   sync.obj
 0001:000308a0       _PeerBeaconAtJoinAction    100318a0 f   sync.obj
 0001:00030e90       _PeerBeacon                10031e90 f   sync.obj
 0001:00031da0       _PeerProbeReqAction        10032da0 f   sync.obj
 0001:000320f0       _BeaconTimeoutAtJoinAction 100330f0 f   sync.obj
 0001:00032140       _ScanTimeoutAction         10033140 f   sync.obj
 0001:000321c0       _ScanNextChannel           100331c0 f   sync.obj
 0001:000327b0       _InvalidStateWhenScan      100337b0 f   sync.obj
 0001:00032810       _InvalidStateWhenJoin      10033810 f   sync.obj
 0001:00032870       _InvalidStateWhenStart     10033870 f   sync.obj
 0001:000328d0       _EnqueuePsPoll             100338d0 f   sync.obj
 0001:00032910       _EnqueueBeaconFrame        10033910 f   sync.obj
 0001:00032a00       _EnqueueProbeRequest       10033a00 f   sync.obj
 0001:00032ae0       _BuildChannelList          10033ae0 f   sync.obj
 0001:00032ef0       _FirstChannel              10033ef0 f   sync.obj
 0001:00032f00       _NextChannel               10033f00 f   sync.obj
 0001:00032f60       _ChangeToCellPowerLimit    10033f60 f   sync.obj
 0001:00033020       _ConvertToRssi             10034020 f   sync.obj
 0001:00033230       _RTMPusecDelay             10034230 f i sync.obj
 0001:00033290       _MlmeCntlInit              10034290 f   connect.obj
 0001:000332b0       _MlmeCntlMachinePerformAction 100342b0 f   connect.obj
 0001:000334e0       _CntlIdleProc              100344e0 f   connect.obj
 0001:00033630       _CntlOidScanProc           10034630 f   connect.obj
 0001:000337b0       _CntlOidSsidProc           100347b0 f   connect.obj
 0001:00033cf0       _CntlOidRTBssidProc        10034cf0 f   connect.obj
 0001:00034240       _CntlMlmeRoamingProc       10035240 f   connect.obj
 0001:000342c0       _CntlWaitDisassocProc      100352c0 f   connect.obj
 0001:000343a0       _CntlWaitJoinProc          100353a0 f   connect.obj
 0001:00034530       _CntlWaitStartProc         10035530 f   connect.obj
 0001:00034670       _CntlWaitAuthProc          10035670 f   connect.obj
 0001:00034830       _CntlWaitAuthProc2         10035830 f   connect.obj
 0001:00034a10       _CntlWaitAssocProc         10035a10 f   connect.obj
 0001:00034ac0       _CntlWaitReassocProc       10035ac0 f   connect.obj
 0001:00034bb0       _LinkUp                    10035bb0 f   connect.obj
 0001:00035250       _LinkDown                  10036250 f   connect.obj
 0001:00035760       _MlmeCntlConfirm           10036760 f   connect.obj
 0001:00035780       _IterateOnBssTab           10036780 f   connect.obj
 0001:00035ac0       _IterateOnBssTab2          10036ac0 f   connect.obj
 0001:00035c00       _JoinParmFill              10036c00 f   connect.obj
 0001:00035c10       _AssocParmFill             10036c10 f   connect.obj
 0001:00035c60       _ScanParmFill              10036c60 f   connect.obj
 0001:00035ca0       _DisassocParmFill          10036ca0 f   connect.obj
 0001:00035cd0       _StartParmFill             10036cd0 f   connect.obj
 0001:00035d00       _AuthParmFill              10036d00 f   connect.obj
 0001:00035d40       _ComposePsPoll             10036d40 f   connect.obj
 0001:00035e00       _ComposeNullFrame          10036e00 f   connect.obj
 0001:00035ee0       _MakeIbssBeacon            10036ee0 f   connect.obj
 0001:00036340       _MlmeScanReqSanity         10037340 f   sanity.obj
 0001:00036420       _MlmeStartReqSanity        10037420 f   sanity.obj
 0001:00036480       _MlmeAssocReqSanity        10037480 f   sanity.obj
 0001:000364d0       _MlmeAuthReqSanity         100374d0 f   sanity.obj
 0001:00036560       _PeerAssocRspSanity        10037560 f   sanity.obj
 0001:00036a30       _PeerDisassocSanity        10037a30 f   sanity.obj
 0001:00036a70       _PeerDeauthSanity          10037a70 f   sanity.obj
 0001:00036ab0       _PeerAuthSanity            10037ab0 f   sanity.obj
 0001:00036c00       _PeerProbeReqSanity        10037c00 f   sanity.obj
 0001:00036d20       _PeerBeaconAndProbeRspSanity 10037d20 f   sanity.obj
 0001:00037810       _GetTimBit                 10038810 f   sanity.obj
 0001:00037940       _ChannelSanity             10038940 f   sanity.obj
 0001:00037990       _NetworkTypeInUseSanity    10038990 f   sanity.obj
 0001:00037a10       _PeerTxTypeInUseSanity     10038a10 f   sanity.obj
 0001:00037b10       _RTMPWPAWepKeySanity       10038b10 f   sanity.obj
 0001:00037c20       _RTMPRemoveKeySanity       10038c20 f   sanity.obj
 0001:00037e20       _md5_mac                   10038e20 f   md5.obj
 0001:00037e90       _hmac_md5                  10038e90 f   md5.obj
 0001:00038020       _MD5Init                   10039020 f   md5.obj
 0001:00038060       _MD5Update                 10039060 f   md5.obj
 0001:00038190       _MD5Final                  10039190 f   md5.obj
 0001:00038270       _MD5Transform              10039270 f   md5.obj
 0001:000390e0       _SHAInit                   1003a0e0 f   md5.obj
 0001:00039170       _SHAUpdate                 1003a170 f   md5.obj
 0001:00039570       _SHAFinal                  1003a570 f   md5.obj
 0001:000396d0       _aes_set_key               1003a6d0 f   md5.obj
 0001:00039e20       _aes_encrypt               1003ae20 f   md5.obj
 0001:0003af70       _aes_decrypt               1003bf70 f   md5.obj
 0001:0003c0d0       _WpaMsgTypeSubst           1003d0d0 f   wpa.obj
 0001:0003c160       _WpaPskStateMachineInit    1003d160 f   wpa.obj
 0001:0003c1a0       _WpaEAPOLKeyAction         1003d1a0 f   wpa.obj
 0001:0003c7a0       _WpaPairMsg1Action         1003d7a0 f   wpa.obj
 0001:0003cf50       _WpaPairMsg3Action         1003df50 f   wpa.obj
 0001:0003d520       _WpaGroupMsg1Action        1003e520 f   wpa.obj
 0001:0003dbd0       _WpaMacHeaderInit          1003ebd0 f   wpa.obj
 0001:0003dcb0       _WpaHardTransmit           1003ecb0 f   wpa.obj
 0001:0003e1c0       _HMAC_SHA1                 1003f1c0 f   wpa.obj
 0001:0003e340       _PRF                       1003f340 f   wpa.obj
 0001:0003e430       _CCKMPRF                   1003f430 f   wpa.obj
 0001:0003e500       _WpaCountPTK               1003f500 f   wpa.obj
 0001:0003e870       _GenRandom                 1003f870 f   wpa.obj
 0001:0003ea10       _AES_GTK_KEY_UNWRAP        1003fa10 f   wpa.obj
 0001:0003ebf0       _MD4Init                   1003fbf0 f   md4.obj
 0001:0003ec30       _MD4Update                 1003fc30 f   md4.obj
 0001:0003ed30       _MD4Final                  1003fd30 f   md4.obj
 0001:0003edd0       _MD4Transform              1003fdd0 f   md4.obj
 0001:0003f710       _Encode                    10040710 f   md4.obj
 0001:0003f7b0       _Decode                    100407b0 f   md4.obj
 0001:0003f830       _MD4_memcpy                10040830 f   md4.obj
 0001:0003f870       _MD4_memset                10040870 f   md4.obj
 0001:0003f8a0       _LeapMsgTypeSubst          100408a0 f   leap.obj
 0001:0003f8b0       _LeapMachinePerformAction  100408b0 f   leap.obj
 0001:0003fc40       _LeapMacHeaderInit         10040c40 f   leap.obj
 0001:0003fd20       _LeapStartAction           10040d20 f   leap.obj
 0001:0003fea0       _LeapIdentityAction        10040ea0 f   leap.obj
 0001:00040160       _LeapPeerChallengeAction   10041160 f   leap.obj
 0001:00040540       _LeapNakeResponse          10041540 f   leap.obj
 0001:00040810       _HashPwd                   10041810 f   leap.obj
 0001:000408c0       _PeerChallengeResponse     100418c0 f   leap.obj
 0001:00040930       _ParityKey                 10041930 f   leap.obj
 0001:000409b0       _DesKey                    100419b0 f   leap.obj
 0001:00040c10       _Des                       10041c10 f   leap.obj
 0001:00041b60       _DesEncrypt                10042b60 f   leap.obj
 0001:00041bc0       _LeapNetworkChallengeAction 10042bc0 f   leap.obj
 0001:00041ee0       _LeapNetworkChallengeResponse 10042ee0 f   leap.obj
 0001:000421c0       _HashpwdHash               100431c0 f   leap.obj
 0001:00042200       _ProcessSessionKey         10043200 f   leap.obj
 0001:000422b0       _LeapEapolKeyAction        100432b0 f   leap.obj
 0001:00042670       _RogueApTableInit          10043670 f   leap.obj
 0001:000426b0       _RogueApTableSearch        100436b0 f   leap.obj
 0001:00042700       _RogueApEntrySet           10043700 f   leap.obj
 0001:00042730       _RogueApTableSetEntry      10043730 f   leap.obj
 0001:00042810       _RogueApTableDeleteEntry   10043810 f   leap.obj
 0001:000428c0       _LeapAuthTimeout           100438c0 f   leap.obj
 0001:000429f0       _LeapSendRogueAPReport     100439f0 f   leap.obj
 0001:00043040       _CCKMAssocRspSanity        10044040 f   leap.obj
 0001:00043840       _CCXAdjacentAPReport       10044840 f   leap.obj
 0001:00043ea0       _CKIP_key_permute          10044ea0 f   rtmp_ckipmic.obj
 0001:00044090       _RTMPCkipMicInit           10045090 f   rtmp_ckipmic.obj
 0001:000440d0       _RTMPMicUpdate             100450d0 f   rtmp_ckipmic.obj
 0001:000441a0       _RTMPMicGetCoefficient     100451a0 f   rtmp_ckipmic.obj
 0001:00044250       _xor_128                   10045250 f   rtmp_ckipmic.obj
 0001:00044290       _RTMPCkipSbox              10045290 f   rtmp_ckipmic.obj
 0001:000442a0       _xor_32                    100452a0 f   rtmp_ckipmic.obj
 0001:000442e0       _next_key                  100452e0 f   rtmp_ckipmic.obj
 0001:000443f0       _byte_sub                  100453f0 f   rtmp_ckipmic.obj
 0001:00044430       _shift_row                 10045430 f   rtmp_ckipmic.obj
 0001:00044500       _mix_column                10045500 f   rtmp_ckipmic.obj
 0001:000446b0       _RTMPAesEncrypt            100456b0 f   rtmp_ckipmic.obj
 0001:00044800       _RTMPMicFinal              10045800 f   rtmp_ckipmic.obj
 0001:00044980       _RTMPCkipInsertCMIC        10045980 f   rtmp_ckipmic.obj
 0001:00044c40       _RTMPCkipDecrypt           10045c40 f   rtmp_ckipmic.obj
 0001:00044e50       _RTMGetPCkipPK             10045e50 f   rtmp_ckipmic.obj
 0001:00044f80       _RTUSBInitTxDesc           10045f80 f   wince_bulk.obj
 0001:00044f90       _RTUSBInitRxDesc           10045f90 f   wince_bulk.obj
 0001:00044fa0       _RTUSBUpdateTxD            10045fa0 f   wince_bulk.obj
 0001:000451c0       _RTUSBAggregationFrameExec 100461c0 f   wince_bulk.obj
 0001:000454a0       _RTUSBBulkOutDataPacket    100464a0 f   wince_bulk.obj
 0001:00045740       _RTUSBBulkOutDataPacketComplete 10046740 f   wince_bulk.obj
 0001:00045ac0       _RTUSBBulkOutNullFrame     10046ac0 f   wince_bulk.obj
 0001:00045c40       _RTUSBBulkOutNullFrameComplete 10046c40 f   wince_bulk.obj
 0001:00045ce0       _RTUSBBulkOutBeacon        10046ce0 f   wince_bulk.obj
 0001:00045e10       _RTUSBBulkOutBeaconComplete 10046e10 f   wince_bulk.obj
 0001:00045e90       _RTUSBBulkOutMLMEPacket    10046e90 f   wince_bulk.obj
 0001:00045fd0       _RTUSBBulkOutMLMEPacketComplete 10046fd0 f   wince_bulk.obj
 0001:00046100       _RTUSBBulkOutPsPoll        10047100 f   wince_bulk.obj
 0001:000461e0       _RTUSBBulkOutPsPollComplete 100471e0 f   wince_bulk.obj
 0001:00046270       _RTUSBBulkRxComplete       10047270 f   wince_bulk.obj
 0001:000462b0       _TransferNotify            100472b0 f   wince_bulk.obj
 0001:000462d0       _RTUSBBulkReceive          100472d0 f   wince_bulk.obj
 0001:000465a0       _RTUSBKickBulkOut          100475a0 f   wince_bulk.obj
 0001:00046c30       _RTUSBCleanUpDataBulkOutQueue 10047c30 f   wince_bulk.obj
 0001:00046d50       _RTUSBCleanUpMLMEBulkOutQueue 10047d50 f   wince_bulk.obj
 0001:00046e10       _RTUSBCancelPendingIRPs    10047e10 f   wince_bulk.obj
 0001:00046e30       _RTUSBCancelPendingBulkInIRP 10047e30 f   wince_bulk.obj
 0001:00046ea0       _RTUSBCancelPendingBulkOutIRP 10047ea0 f   wince_bulk.obj
 0001:00046ff0       _SetEvent                  10047ff0 f i wince_bulk.obj
 0001:00047010       _ResetEvent                10048010 f i wince_bulk.obj
 0001:00047030       _InterlockedExchange       10048030 f i wince_bulk.obj
 0001:00047040       _RTUSBFirmwareRun          10048040 f   wince_io.obj
 0001:00047070       _RTUSBSetLED               10048070 f   wince_io.obj
 0001:000470a0       _RTUSBSingleRead           100480a0 f   wince_io.obj
 0001:000470e0       _RTUSBSingleWrite          100480e0 f   wince_io.obj
 0001:00047110       _RTUSBMultiRead            10048110 f   wince_io.obj
 0001:00047150       _RTUSBMultiWrite           10048150 f   wince_io.obj
 0001:00047180       _RTUSBReadMACRegister      10048180 f   wince_io.obj
 0001:000471c0       _RTUSBWriteMACRegister     100481c0 f   wince_io.obj
 0001:000471f0       _RTUSBReadBBPRegister      100481f0 f   wince_io.obj
 0001:000473b0       _RTUSBWriteBBPRegister     100483b0 f   wince_io.obj
 0001:000474d0       _RTUSBWriteRFRegister      100484d0 f   wince_io.obj
 0001:00047590       _RTUSBReadEEPROM           10048590 f   wince_io.obj
 0001:000475d0       _RTUSBWriteEEPROM          100485d0 f   wince_io.obj
 0001:00047600       _RTUSBPutToSleep           10048600 f   wince_io.obj
 0001:00047630       _RTUSBWakeUp               10048630 f   wince_io.obj
 0001:00047660       _RTUSBInitializeCmdQ       10048660 f   wince_io.obj
 0001:00047690       _RTUSBEnqueueCmdFromNdis   10048690 f   wince_io.obj
 0001:00047850       _RTUSBEnqueueInternalCmd   10048850 f   wince_io.obj
 0001:000479f0       _RTUSBDequeueCmd           100489f0 f   wince_io.obj
 0001:00047a40       _RTUSB_VendorRequest       10048a40 f   wince_io.obj
 0001:00047cf0       _VenderTransferComplete    10048cf0 f   wince_io.obj
 0001:00047d00       _RTUSB_CallUSBD            10048d00 f   wince_io.obj
 0001:00047d10       _RTUSBCE_ConfigureDevice   10048d10 f   wince_io.obj
 0001:00048470       _RTUSB_InterfaceStop       10049470 f   wince_io.obj
 0001:000484b0       _RTUSBCE_ResetAllPipes     100494b0 f   wince_io.obj
 0001:000486a0       _RTUSB_ResetPipe           100496a0 f   wince_io.obj
 0001:000486c0       _RTUSB_ResetDevice         100496c0 f   wince_io.obj
 0001:000486e0       _RTUSBCmdThread            100496e0 f   wince_io.obj
 0001:0004a290       _RTUSBQueryHardWareRegister 1004b290 f   wince_io.obj
 0001:0004a370       _RTUSBSetHardWareRegister  1004b370 f   wince_io.obj
 0001:0004a6e0       _UsbDeviceTest             1004b6e0 f   wince.obj
 0001:0004a740       _ClosePipe                 1004b740 f   wince.obj
 0001:0004a7f0       _RemoveDeviceContext       1004b7f0 f   wince.obj
 0001:0004a960       _UsbDeviceNotify           1004b960 f   wince.obj
 0001:0004ac00       _DllEntry                  1004bc00 f   wince.obj
 0001:0004acf0       _RTUSBCE_InterfaceStart    1004bcf0 f   wince.obj
 0001:0004af50       _ActivateDeviceEx          1004bf50 f   wince.obj
 0001:0004afa0       _USBDeviceAttach           1004bfa0 f   wince.obj
 0001:0004b250       _USBInstallDriver          1004c250 f   wince.obj
 0001:0004b4d0       _USBUnInstallDriver        1004c4d0 f   wince.obj
 0001:0004b5f0       _ParseUsbDescriptors       1004c5f0 f   wince.obj
 0001:0004c0e0       _RTUSBCE_ResetEvent        1004d0e0 f   wince.obj
 0001:0004c170       _RxBulkPollingExec         1004d170 f   wince.obj
 0001:0004c180       _RTMPCopyUnicodeString     1004d180 f   wince.obj
 0001:0004c240       _DBGDumpHex                1004d240 f   wince.obj
 0001:0004c494       _NKDbgPrintfW              1004d494 f   Coredll:COREDLL.dll
 0001:0004c49a       _InitializeCriticalSection 1004d49a f   Coredll:COREDLL.dll
 0001:0004c4a0       _DeleteCriticalSection     1004d4a0 f   Coredll:COREDLL.dll
 0001:0004c4a6       _ResumeThread              1004d4a6 f   Coredll:COREDLL.dll
 0001:0004c4ac       _CeGetThreadPriority       1004d4ac f   Coredll:COREDLL.dll
 0001:0004c4b2       _CeSetThreadPriority       1004d4b2 f   Coredll:COREDLL.dll
 0001:0004c4b8       _memset                    1004d4b8 f   Coredll:COREDLL.dll
 0001:0004c4be       __allshr                   1004d4be f   Coredll:COREDLL.dll
 0001:0004c4c4       __allmul                   1004d4c4 f   Coredll:COREDLL.dll
 0001:0004c4ca       __aullshr                  1004d4ca f   Coredll:COREDLL.dll
 0001:0004c4d0       _LeaveCriticalSection      1004d4d0 f   Coredll:COREDLL.dll
 0001:0004c4d6       _EnterCriticalSection      1004d4d6 f   Coredll:COREDLL.dll
 0001:0004c4dc       _SetEventData              1004d4dc f   Coredll:COREDLL.dll
 0001:0004c4e2       _GetEventData              1004d4e2 f   Coredll:COREDLL.dll
 0001:0004c4e8       _EventModify               1004d4e8 f   Coredll:COREDLL.dll
 0001:0004c4ee       _WaitForSingleObject       1004d4ee f   Coredll:COREDLL.dll
 0001:0004c4f4       _Sleep                     1004d4f4 f   Coredll:COREDLL.dll
 0001:0004c4fa       _SetLastError              1004d4fa f   Coredll:COREDLL.dll
 0001:0004c500       _CloseHandle               1004d500 f   Coredll:COREDLL.dll
 0001:0004c506       _CreateThread              1004d506 f   Coredll:COREDLL.dll
 0001:0004c50c       _CreateEventW              1004d50c f   Coredll:COREDLL.dll
 0001:0004c512       _GetLastError              1004d512 f   Coredll:COREDLL.dll
 0001:0004c518       _DisableThreadLibraryCalls 1004d518 f   Coredll:COREDLL.dll
 0001:0004c51e       _RegisterDbgZones          1004d51e f   Coredll:COREDLL.dll
 0001:0004c524       _sprintf                   1004d524 f   Coredll:COREDLL.dll
 0001:0004c52a       _NdisAllocateSpinLock      1004d52a f   ndis:NDIS.dll
 0001:0004c530       _DbgPrint                  1004d530 f   ndis:NDIS.dll
 0001:0004c536       _NdisReleaseSpinLock       1004d536 f   ndis:NDIS.dll
 0001:0004c53c       _NdisAcquireSpinLock       1004d53c f   ndis:NDIS.dll
 0001:0004c542       _NdisFreeSpinLock          1004d542 f   ndis:NDIS.dll
 0001:0004c548       _NdisMSleep                1004d548 f   ndis:NDIS.dll
 0001:0004c54e       _NdisGetSystemUpTime       1004d54e f   ndis:NDIS.dll
 0001:0004c554       _NdisFreeMemory            1004d554 f   ndis:NDIS.dll
 0001:0004c55a       _NdisAllocateMemoryWithTag 1004d55a f   ndis:NDIS.dll
 0001:0004c560       _NdisQueryBuffer           1004d560 f   ndis:NDIS.dll
 0001:0004c566       _NdisQueryPacket           1004d566 f   ndis:NDIS.dll
 0001:0004c56c       _NdisInterlockedIncrement  1004d56c f   ndis:NDIS.dll
 0001:0004c572       _NdisFreeBufferPool        1004d572 f   ndis:NDIS.dll
 0001:0004c578       _NdisFreePacketPool        1004d578 f   ndis:NDIS.dll
 0001:0004c57e       _NdisCloseConfiguration    1004d57e f   ndis:NDIS.dll
 0001:0004c584       _NdisUnicodeStringToAnsiString 1004d584 f   ndis:NDIS.dll
 0001:0004c58a       _NdisReadConfiguration     1004d58a f   ndis:NDIS.dll
 0001:0004c590       _NdisOpenConfiguration     1004d590 f   ndis:NDIS.dll
 0001:0004c596       _NdisCloseFile             1004d596 f   ndis:NDIS.dll
 0001:0004c59c       _NdisUnmapFile             1004d59c f   ndis:NDIS.dll
 0001:0004c5a2       _NdisMapFile               1004d5a2 f   ndis:NDIS.dll
 0001:0004c5a8       _NdisOpenFile              1004d5a8 f   ndis:NDIS.dll
 0001:0004c5ae       _NdisInitializeString      1004d5ae f   ndis:NDIS.dll
 0001:0004c5b4       _NdisMInitializeTimer      1004d5b4 f   ndis:NDIS.dll
 0001:0004c5ba       _NdisSetTimer              1004d5ba f   ndis:NDIS.dll
 0001:0004c5c0       _NdisMSetPeriodicTimer     1004d5c0 f   ndis:NDIS.dll
 0001:0004c5c6       _NdisMCancelTimer          1004d5c6 f   ndis:NDIS.dll
 0001:0004c5cc       _NdisTerminateWrapper      1004d5cc f   ndis:NDIS.dll
 0001:0004c5d2       _NdisMRegisterMiniport     1004d5d2 f   ndis:NDIS.dll
 0001:0004c5d8       _NdisInitializeWrapper     1004d5d8 f   ndis:NDIS.dll
 0001:0004c5de       _NdisInterlockedDecrement  1004d5de f   ndis:NDIS.dll
 0001:0004c5e4       _NdisMGetDeviceProperty    1004d5e4 f   ndis:NDIS.dll
 0001:0004c5ea       _NdisMSetAttributesEx      1004d5ea f   ndis:NDIS.dll
 0001:0004c5f0       _NdisGetCurrentSystemTime  1004d5f0 f   ndis:NDIS.dll
 0001:0004c5f6       _NdisStallExecution        1004d5f6 f   ndis:NDIS.dll
 0001:0004c5fc       _NdisDeregisterAdapter     1004d5fc f   ndis:NDIS.dll
 0001:0004c602       _NdisRegisterAdapter       1004d602 f   ndis:NDIS.dll
 0001:0004c608       _RegisterClientSettings    1004d608 f   usbd:USBD.dll
 0001:0004c60e       _RegisterClientDriverID    1004d60e f   usbd:USBD.dll
 0001:0004c614       _UnRegisterClientDriverID  1004d614 f   usbd:USBD.dll
 0001:0004c61a       _UnRegisterClientSettings  1004d61a f   usbd:USBD.dll
 0001:0004c620       _AbortTransfer             1004d620 f   usbclient:usbclient.obj
 0001:0004c690       _CloseTransferHandle       1004d690 f   usbclient:usbclient.obj
 0001:0004c700       _ClearOrSetFeature         1004d700 f   usbclient:usbclient.obj
 0001:0004c900       _DefaultTransferComplete   1004d900 f   usbclient:usbclient.obj
 0001:0004c9b0       _GetStatus                 1004d9b0 f   usbclient:usbclient.obj
 0001:0004cba0       _GetTransferStatus         1004dba0 f   usbclient:usbclient.obj
 0001:0004cc80       _IssueBulkTransfer         1004dc80 f   usbclient:usbclient.obj
 0001:0004cf50       _IssueInterruptTransfer    1004df50 f   usbclient:usbclient.obj
 0001:0004d220       _IssueVendorTransfer       1004e220 f   usbclient:usbclient.obj
 0001:0004d4f0       _ResetDefaultEndpoint      1004e4f0 f   usbclient:usbclient.obj
 0001:0004d5d0       _ResetBulkEndpoint         1004e5d0 f   usbclient:usbclient.obj
 0001:0004d720       _ResetPipe                 1004e720 f   usbclient:usbclient.obj
 0001:0004d7a0       __ResetEvent               1004e7a0 f i usbclient:usbclient.obj
 0001:0004d804       __IMPORT_DESCRIPTOR_COREDLL 1004e804     Coredll:COREDLL.dll
 0001:0004d818       __IMPORT_DESCRIPTOR_NDIS   1004e818     ndis:NDIS.dll
 0001:0004d82c       __IMPORT_DESCRIPTOR_USBD   1004e82c     usbd:USBD.dll
 0001:0004d840       __NULL_IMPORT_DESCRIPTOR   1004e840     Coredll:COREDLL.dll
 0002:00000000       __imp__NKDbgPrintfW        1004f000     Coredll:COREDLL.dll
 0002:00000004       __imp__InitializeCriticalSection 1004f004     Coredll:COREDLL.dll
 0002:00000008       __imp__DeleteCriticalSection 1004f008     Coredll:COREDLL.dll
 0002:0000000c       __imp__ResumeThread        1004f00c     Coredll:COREDLL.dll
 0002:00000010       __imp__CeGetThreadPriority 1004f010     Coredll:COREDLL.dll
 0002:00000014       __imp__CeSetThreadPriority 1004f014     Coredll:COREDLL.dll
 0002:00000018       __imp__memset              1004f018     Coredll:COREDLL.dll
 0002:0000001c       __imp___allshr             1004f01c     Coredll:COREDLL.dll
 0002:00000020       __imp___allmul             1004f020     Coredll:COREDLL.dll
 0002:00000024       __imp___aullshr            1004f024     Coredll:COREDLL.dll
 0002:00000028       __imp__LeaveCriticalSection 1004f028     Coredll:COREDLL.dll
 0002:0000002c       __imp__EnterCriticalSection 1004f02c     Coredll:COREDLL.dll
 0002:00000030       __imp__SetEventData        1004f030     Coredll:COREDLL.dll
 0002:00000034       __imp__GetEventData        1004f034     Coredll:COREDLL.dll
 0002:00000038       __imp__EventModify         1004f038     Coredll:COREDLL.dll
 0002:0000003c       __imp__WaitForSingleObject 1004f03c     Coredll:COREDLL.dll
 0002:00000040       __imp__Sleep               1004f040     Coredll:COREDLL.dll
 0002:00000044       __imp__SetLastError        1004f044     Coredll:COREDLL.dll
 0002:00000048       __imp__CloseHandle         1004f048     Coredll:COREDLL.dll
 0002:0000004c       __imp__CreateThread        1004f04c     Coredll:COREDLL.dll
 0002:00000050       __imp__CreateEventW        1004f050     Coredll:COREDLL.dll
 0002:00000054       __imp__GetLastError        1004f054     Coredll:COREDLL.dll
 0002:00000058       __imp__DisableThreadLibraryCalls 1004f058     Coredll:COREDLL.dll
 0002:0000005c       __imp__RegisterDbgZones    1004f05c     Coredll:COREDLL.dll
 0002:00000060       __imp__sprintf             1004f060     Coredll:COREDLL.dll
 0002:00000064       \177COREDLL_NULL_THUNK_DATA 1004f064     Coredll:COREDLL.dll
 0002:00000068       __imp__NdisAllocateSpinLock 1004f068     ndis:NDIS.dll
 0002:0000006c       __imp__DbgPrint            1004f06c     ndis:NDIS.dll
 0002:00000070       __imp__NdisReleaseSpinLock 1004f070     ndis:NDIS.dll
 0002:00000074       __imp__NdisAcquireSpinLock 1004f074     ndis:NDIS.dll
 0002:00000078       __imp__NdisFreeSpinLock    1004f078     ndis:NDIS.dll
 0002:0000007c       __imp__NdisMSleep          1004f07c     ndis:NDIS.dll
 0002:00000080       __imp__NdisGetSystemUpTime 1004f080     ndis:NDIS.dll
 0002:00000084       __imp__NdisFreeMemory      1004f084     ndis:NDIS.dll
 0002:00000088       __imp__NdisAllocateMemoryWithTag 1004f088     ndis:NDIS.dll
 0002:0000008c       __imp__NdisQueryBuffer     1004f08c     ndis:NDIS.dll
 0002:00000090       __imp__NdisQueryPacket     1004f090     ndis:NDIS.dll
 0002:00000094       __imp__NdisInterlockedIncrement 1004f094     ndis:NDIS.dll
 0002:00000098       __imp__NdisFreeBufferPool  1004f098     ndis:NDIS.dll
 0002:0000009c       __imp__NdisFreePacketPool  1004f09c     ndis:NDIS.dll
 0002:000000a0       __imp__NdisCloseConfiguration 1004f0a0     ndis:NDIS.dll
 0002:000000a4       __imp__NdisUnicodeStringToAnsiString 1004f0a4     ndis:NDIS.dll
 0002:000000a8       __imp__NdisReadConfiguration 1004f0a8     ndis:NDIS.dll
 0002:000000ac       __imp__NdisOpenConfiguration 1004f0ac     ndis:NDIS.dll
 0002:000000b0       __imp__NdisCloseFile       1004f0b0     ndis:NDIS.dll
 0002:000000b4       __imp__NdisUnmapFile       1004f0b4     ndis:NDIS.dll
 0002:000000b8       __imp__NdisMapFile         1004f0b8     ndis:NDIS.dll
 0002:000000bc       __imp__NdisOpenFile        1004f0bc     ndis:NDIS.dll
 0002:000000c0       __imp__NdisInitializeString 1004f0c0     ndis:NDIS.dll
 0002:000000c4       __imp__NdisMInitializeTimer 1004f0c4     ndis:NDIS.dll
 0002:000000c8       __imp__NdisSetTimer        1004f0c8     ndis:NDIS.dll
 0002:000000cc       __imp__NdisMSetPeriodicTimer 1004f0cc     ndis:NDIS.dll
 0002:000000d0       __imp__NdisMCancelTimer    1004f0d0     ndis:NDIS.dll
 0002:000000d4       __imp__NdisTerminateWrapper 1004f0d4     ndis:NDIS.dll
 0002:000000d8       __imp__NdisMRegisterMiniport 1004f0d8     ndis:NDIS.dll
 0002:000000dc       __imp__NdisInitializeWrapper 1004f0dc     ndis:NDIS.dll
 0002:000000e0       __imp__NdisInterlockedDecrement 1004f0e0     ndis:NDIS.dll
 0002:000000e4       __imp__NdisMGetDeviceProperty 1004f0e4     ndis:NDIS.dll
 0002:000000e8       __imp__NdisMSetAttributesEx 1004f0e8     ndis:NDIS.dll
 0002:000000ec       __imp__NdisGetCurrentSystemTime 1004f0ec     ndis:NDIS.dll
 0002:000000f0       __imp__NdisStallExecution  1004f0f0     ndis:NDIS.dll
 0002:000000f4       __imp__NdisDeregisterAdapter 1004f0f4     ndis:NDIS.dll
 0002:000000f8       __imp__NdisRegisterAdapter 1004f0f8     ndis:NDIS.dll
 0002:000000fc       \177NDIS_NULL_THUNK_DATA   1004f0fc     ndis:NDIS.dll
 0002:00000100       __imp__RegisterClientDriverID 1004f100     usbd:USBD.dll
 0002:00000104       __imp__UnRegisterClientDriverID 1004f104     usbd:USBD.dll
 0002:00000108       __imp__UnRegisterClientSettings 1004f108     usbd:USBD.dll
 0002:0000010c       __imp__RegisterClientSettings 1004f10c     usbd:USBD.dll
 0002:00000110       \177USBD_NULL_THUNK_DATA   1004f110     usbd:USBD.dll
 0002:00000118       _ReasonString              1004f118     mlme.obj
 0002:00000160       _BasicRateMask             1004f160     mlme.obj
 0002:00000190       _BROADCAST_ADDR            1004f190     mlme.obj
 0002:00000198       _RssiSafeLevelForTxRate    1004f198     mlme.obj
 0002:000001a8       _Phy11BNextRateDownward    1004f1a8     mlme.obj
 0002:000001ac       _Phy11BNextRateUpward      1004f1ac     mlme.obj
 0002:000001b0       _Phy11BGNextRateDownward   1004f1b0     mlme.obj
 0002:000001bc       _Phy11BGNextRateUpward     1004f1bc     mlme.obj
 0002:000001c8       _Phy11ANextRateDownward    1004f1c8     mlme.obj
 0002:000001d4       _Phy11ANextRateUpward      1004f1d4     mlme.obj
 0002:000001e0       _RateUpPER                 1004f1e0     mlme.obj
 0002:000001f8       _RateDownPER               1004f1f8     mlme.obj
 0002:00000210       _RateIdToMbps              1004f210     mlme.obj
 0002:00000220       _RateIdTo500Kbps           1004f220     mlme.obj
 0002:0000023c       _SupRateIe                 1004f23c     mlme.obj
 0002:0000023d       _ExtRateIe                 1004f23d     mlme.obj
 0002:0000023e       _ErpIe                     1004f23e     mlme.obj
 0002:0000023f       _DsIe                      1004f23f     mlme.obj
 0002:00000240       _TimIe                     1004f240     mlme.obj
 0002:00000241       _WpaIe                     1004f241     mlme.obj
 0002:00000242       _Wpa2Ie                    1004f242     mlme.obj
 0002:00000243       _IbssIe                    1004f243     mlme.obj
 0002:00000244       _Ccx2Ie                    1004f244     mlme.obj
 0002:00000248       _SES_OUI                   1004f248     mlme.obj
 0002:00000250       _RF2528RegTable            1004f250     mlme.obj
 0002:00000368       _RF5226RegTable            1004f368     mlme.obj
 0002:00000958       _AntStr                    1004f958     mlme.obj
 0002:00000968       _CISCO_OUI                 1004f968     aironet.obj
 0002:0000096c       _SNAP_802_1H               1004f96c     rtusb_data.obj
 0002:00000974       _SNAP_BRIDGE_TUNNEL        1004f974     rtusb_data.obj
 0002:0000097c       _SNAP_AIRONET              1004f97c     rtusb_data.obj
 0002:00000984       _CKIP_LLC_SNAP             1004f984     rtusb_data.obj
 0002:0000098c       _EAPOL_LLC_SNAP            1004f98c     rtusb_data.obj
 0002:00000994       _EAPOL                     1004f994     rtusb_data.obj
 0002:00000998       _IPX                       1004f998     rtusb_data.obj
 0002:0000099c       _APPLE_TALK                1004f99c     rtusb_data.obj
 0002:000009a0       _RateIdToPlcpSignal        1004f9a0     rtusb_data.obj
 0002:000009ac       _OfdmSignalToRateId        1004f9ac     rtusb_data.obj
 0002:000009bc       _default_cwmin             1004f9bc     rtusb_data.obj
 0002:000009c0       _default_cwmax             1004f9c0     rtusb_data.obj
 0002:000009c4       _default_sta_aifsn         1004f9c4     rtusb_data.obj
 0002:000009c8       _MapUserPriorityToAccessCategory 1004f9c8     rtusb_data.obj
 0002:000009d0       _BIT8                      1004f9d0     rtmp_init.obj
 0002:000009d8       _BIT32                     1004f9d8     rtmp_init.obj
 0002:00000a58       _CipherName                1004fa58     rtmp_init.obj
 0002:00000a78       _NICRegTable               1004fa78     rtmp_init.obj
 0002:00000ef8       _BBPRegTable               1004fef8     rtmp_init.obj
 0002:00000f30       _MACRegTable               1004ff30     rtmp_init.obj
 0002:00000fc8       _FirmwareImage             1004ffc8     rtmp_init.obj
 0002:00001628       _RTDebugLevel              10050628     rtmp_main.obj
 0002:00001630       _Wpa2AuthEncryptPairs      10050630     rtmp_info.obj
 0002:000016a0       _STASupportedOids          100506a0     rtmp_info.obj
 0002:000018f8       _FCSTAB_32                 100508f8     rtmp_wep.obj
 0002:00001cf8       _WEPKEY                    10050cf8     rtmp_wep.obj
 0002:00001d08       _Tkip_Sbox_Lower           10050d08     rtmp_tkip.obj
 0002:00002108       _Tkip_Sbox_Upper           10051108     rtmp_tkip.obj
 0002:00002508       _CipherWpaTemplate         10051508     assoc.obj
 0002:00002520       _CipherWpa2Template        10051520     assoc.obj
 0002:00002538       _Ccx2IeInfo                10051538     assoc.obj
 0002:00002540       _A_BAND_REGION_0_CHANNEL_LIST 10051540     sync.obj
 0002:00002550       _A_BAND_REGION_1_CHANNEL_LIST 10051550     sync.obj
 0002:00002564       _A_BAND_REGION_2_CHANNEL_LIST 10051564     sync.obj
 0002:0000256c       _A_BAND_REGION_3_CHANNEL_LIST 1005156c     sync.obj
 0002:00002574       _A_BAND_REGION_4_CHANNEL_LIST 10051574     sync.obj
 0002:0000257c       _A_BAND_REGION_5_CHANNEL_LIST 1005157c     sync.obj
 0002:00002580       _A_BAND_REGION_6_CHANNEL_LIST 10051580     sync.obj
 0002:00002584       _A_BAND_REGION_7_CHANNEL_LIST 10051584     sync.obj
 0002:0000259c       _CipherSuiteWpaNoneTkip    1005159c     connect.obj
 0002:000025b2       _CipherSuiteWpaNoneTkipLen 100515b2     connect.obj
 0002:000025b4       _CipherSuiteWpaNoneAes     100515b4     connect.obj
 0002:000025ca       _CipherSuiteWpaNoneAesLen  100515ca     connect.obj
 0002:000025cc       _WPA_OUI                   100515cc     sanity.obj
 0002:000025d0       _RSN_OUI                   100515d0     sanity.obj
 0002:000025d4       _WME_INFO_ELEM             100515d4     sanity.obj
 0002:000025dc       _WME_PARM_ELEM             100515dc     sanity.obj
 0002:000025e4       _Ccx2QosInfo               100515e4     sanity.obj
 0002:000025e8       _RALINK_OUI                100515e8     sanity.obj
 0002:000025ec       _NIC_VENDOR_DESC           100515ec     oem.obj
 0002:00002610       _NIC_VENDOR_DESC_LEN       10051610     oem.obj
 0002:00002614       _NIC_VENDOR_DRIVER_VERSION 10051614     oem.obj
 0002:00002618       _LINKNAME_STRING           10051618     oem.obj
 0002:0000263c       _NTDEVICE_STRING           1005163c     oem.obj
 0002:00004e84       _CipherWpaPskTkip          10053e84     wpa.obj
 0002:00004e9c       _CipherWpaPskTkipLen       10053e9c     wpa.obj
 0002:00004ea0       _CipherWpaPskAes           10053ea0     wpa.obj
 0002:00004eb8       _CipherWpaPskAesLen        10053eb8     wpa.obj
 0002:00004ebc       _CipherSuiteCiscoCCKM      10053ebc     wpa.obj
 0002:00004ed4       _CipherSuiteCiscoCCKMLen   10053ed4     wpa.obj
 0002:00004ed8       _CipherSuiteCiscoCCKM24    10053ed8     wpa.obj
 0002:00004ef2       _CipherSuiteCiscoCCKM24Len 10053ef2     wpa.obj
 0002:00004ef4       _CipherSuiteCiscoCCKMTkip  10053ef4     wpa.obj
 0002:00004f0c       _CipherSuiteCiscoCCKMTkipLen 10053f0c     wpa.obj
 0002:00004f10       _CipherSuiteCiscoCCKMTkip24 10053f10     wpa.obj
 0002:00004f2a       _CipherSuiteCiscoCCKMTkip24Len 10053f2a     wpa.obj
 0002:00004f2c       _CipherSuiteCCXTkip        10053f2c     wpa.obj
 0002:00004f44       _CipherSuiteCCXTkipLen     10053f44     wpa.obj
 0002:00004f48       _CCX_LLC_HDR               10053f48     wpa.obj
 0002:00004f50       _LLC_NORMAL                10053f50     wpa.obj
 0002:00004f58       _EAPOL_FRAME               10053f58     wpa.obj
 0002:00004f60       _PADDING                   10053f60     md4.obj
 0002:00004fa0       _EAP_HEADER                10053fa0     leap.obj
 0002:00004fa8       _SNAP_LEAP_ROGUEAP_HDR     10053fa8     leap.obj
 0002:00004fb0       _Spbox                     10053fb0     leap.obj
 0002:000057b0       _pc1                       100547b0     leap.obj
 0002:000057e8       _totrot                    100547e8     leap.obj
 0002:000057f8       _pc2                       100547f8     leap.obj
 0002:00005848       _SboxTable                 10054848     rtmp_ckipmic.obj
 0002:00005948       _vvenderid                 10054948     wince.obj
 0002:00005974       _pproductid                10054974     wince.obj
 0002:000059a0       _dpCurSettings             100549a0     wince.obj
 0002:00005e00       _ZERO_MAC_ADDR             10054e00     mlme.obj
 0002:00005e06       _SsidIe                    10054e06     mlme.obj
 0002:00005e08       _ZeroSsid                  10054e08     mlme.obj
 0002:00006e28       _Asmversion                10055e28     leap.obj
 0002:00006e30       _GUsbFuncs                 10055e30     <common>
 0002:00006e34       _GhDevice                  10055e34     <common>
 0002:00006e38       _GUsbInterface             10055e38     <common>
 0002:00006e40       _LocalStrings              10055e40     <common>
 0002:000071f8       _PPURB_BULK_OR_INTERRUPT_TRANSFER 100561f8     <common>
 0002:000071fc       _PURB_BULK_OR_INTERRUPT_TRANSFER 100561fc     <common>

 entry point at        0001:0004ac00

 Static symbols

 0001:00039290       _SHAHashBlock              1003a290 f   md5.obj
